:100000000C9449120C9468120C9468120C946812A7
:100010000C9468120C9488140C941E160C9468129C
:100020000C9468120C94EC1A0C9468120C946812DC
:100030000C9468120C9468120C9400300C946812A2
:100040000C9468120C94AB170C942F170C944C144E
:100050000C9468120C94A5230C9468120C946812EA
:100060000C9468120C9468120C9468120C94681228
:100070000C9468120C94472F0C94B7160C94DD1551
:100080000C9468120C940F810C946812322E322E4C
:100090003300696E636F6D70617469626C652048CE
:1000A000570020202530325800204D430045617311
:1000B00079436F6E74726F6C005F03AF01D7006B92
:1000C00000470035001A001100010203171804054B
:1000D00006151107080916120A000B0C13100F0E53
:1000E0000D14040E1F0E0E0E0E000E0E0E0E1F0E21
:1000F0000400040E1F001F0E04000004040400107E
:10010000081300100B1300130B1300010219000158
:100110001A1900191A19080C1E1F1E0C08000206D5
:100120000F1F0F0602000E11111F1B1B1F001F0ABD
:100130000A0A0A0A1F001C101810160505050C17DC
:10014000141714170C00040A110A0A0E00001C10E0
:100150001812160202071C101816110204071C10B0
:100160001816110201061C101815150701010000D0
:1001700000171515151712121212120000000000B8
:1001800000171117141717111311170000000000A2
:100190000015151711111714171117000000070586
:1001A00005050505050707070707070707070305EF
:1001B00009121418100003070F1E1C181000000667
:1001C00009121412090600060917170906001F1163
:1001D0001F001F111F001F111F001F1F1F001F1FC7
:1001E0001F001F111F001F1F1F001F1F1F00040ED5
:1001F0001F04041F0E04010101050D1F0C0411044E
:100200000A11111F1100110E111111110E000A0017
:10021000111111110E000E11111611111610001CE2
:100220001F1F1F131010001C13111D131010001896
:10023000171119171010001F11111F101010C303F0
:10024000F333CF0FFF3F00C030F00CCC3CFC03C3B6
:1002500033F30FCF3FFFAAC08030F0B020E0A00CF6
:10026000CC8C3CFCBC2CECAC08C88838F8B828E82E
:10027000A803C38333F3B323E3A30FCF8F3FFFBFA1
:100280002FEFAF0BCB8B3BFBBB2BEBAB02C2823216
:10029000F2B222E2A20ECE8E3EFEBE2EEEAE0ACA12
:1002A0008A3AFABA2AEA0040609770486858784457
:1002B0006454744C6C5C7C426252724A6A5A7A464C
:1002C0006656764E6E5E7E41615171496959794537
:1002D000659F754D6D5D7D436353734B6B5B7B47D2
:1002E0006757774F6F5F7F1018141C121A161E1174
:1002F00019151D131B171FD0D8D4DCD2DAD6DED1C6
:10030000D9D5DDD3DBD7DF9098949C929A969E91B5
:1003100099959D939B505504060507C4C6C5C7848F
:1003200086858734363537F4F6F5F7B4B6B5B72495
:10033000262527E4E6E5E7A4A6A5A701C18131F1BA
:10034000B121E1A10DCD8D3DFDBD2DEDAD09C989D9
:1003500039F9B929E9A9206D332020200000204D6A
:100360004D4920200000204D4D0220200000204457
:100370004343202000002053544F50200000534896
:100380004F52542100002048414C542000002020AE
:100390002020202000002050524F472000005245CE
:1003A000534554200000202054504D20000055504B
:1003B00044415445000020202020002533640025BE
:1003C0002D31312E31317300252D35640025632FF9
:1003D00025632025630025630046253032643D25D2
:1003E000630020200102202020202020200025332F
:1003F000640025336400252D3564002D2D2D2D201E
:1004000020004144523A20256C64202020202020E6
:100410002020202000232D007E0E0E0E0E1B1B1C04
:100420000E1B1B7E0E0E0E0E0D5D00435645520038
:100430004D52535400504D004D465800535755509F
:1004400044415445005243520052430054504D0021
:1004500043464753595300434647414343004346AD
:100460004744554D50004D415044554D5000545255
:100470004B434C4541520054524B4144440054526A
:100480004B44554D50004C4F43434C454152004C5A
:100490004F43414444004C4F4344554D50004C534E
:1004A000005054574C005054524C00505457420086
:1004B000505452420050545744005054524400503B
:1004C00054575000505452500050545752005054FA
:1004D00052520050410050440043410043560053E3
:1004E0004F00420040400053450053530053520018
:1004F0004D5400560059005400464D0046580046E1
:10050000004C43004C0048414C5400474F00210030
:1005100053544F50002E00484600485400484C00A9
:1005200048003F005A7A41004D4320696E205354E1
:100530004F50004D4320696E2048414C5400696C77
:100540006C6567616C207475726E6F757420616480
:1005500072657373006C6F6B2062757379006E6FD8
:1005600020736C6F7420617661696C61626C6500E8
:100570006E6F206461746100636F6D6D616E6420E5
:1005800071756575652066756C6C007475726E6F3B
:1005900075742071756575652066756C6C00706F7B
:1005A000776572206973204F66660062616420700F
:1005B0006172616D657465722076616C7565007538
:1005C0006E6B6E6F776E20636F6D6D616E6400454C
:1005D00052524F523A20005741524E494E473A200C
:1005E000002A454E442A002564203F0D00322E3259
:1005F0002E3300432025642025530D00256400255B
:10060000630025642025642025642E25642E25643E
:10061000004552524F52002530386C580052435218
:10062000202575202564202575005243202564006F
:100630004D4D004D4D00444343004D4D004D4D0088
:100640002A454E442A0042415544524154452025F2
:10065000750D004D41474D415854494D4520256485
:100660000D004D41474D494E54494D452025640DDF
:10067000007338384D4F44554C45532025640D00C8
:1006800053484F525454494D452025640D0044456C
:100690004641554C54444343004E45474154495606
:1006A0004553484F5254004C4F4E475041555345C7
:1006B000005B53595354454D5D0D00444343004D79
:1006C0004D0025642C20005B414343464D545D0D95
:1006D000005B46554E434D4150535D0D005B5452F7
:1006E000414B54494F4E535D0D005B4C4F434F5DA2
:1006F0000D0053455249414C20256C750D004D436A
:10070000552041544D6567613132380D00484152E2
:10071000445741524520485725640D00322E322E51
:10072000330056455253494F4E20005B494E464FC9
:100730005D0D0025732564002025642C25640025AB
:1007400064006E6F00796573002C202573004D33B3
:1007500000444343004D4D32004D4D31002C2000EC
:1007600025642C202564002A454E442A002A454E43
:10077000442A004D3300444343004D4D32004D4D5B
:1007800031002A454E442A0054696D656F75740026
:100790004269742072656164206572726F72004EE6
:1007A0006F2070616765004E6F2061636B004E6F54
:1007B000206465636F6465720053686F7274210012
:1007C0004275737921004E6F00596573004572724E
:1007D0006F72004F6B002564002564203D202425A6
:1007E000303258203D200050410050580050410008
:1007F00041646472202575203D2024253034582022
:10080000203D3E202043563137203D2025642028BE
:100810002425303258292C202043563138203D20C1
:1008200025642028242530325829004C6F6E67201B
:1008300041646472203D2025750025640025640014
:100840000D5D0025750035373630300053452025C5
:1008500064004D6F64756C65202325642028696EE3
:1008600070757420312E2E38202620392E2E3136E8
:1008700029203D20005352202564004D542025643A
:10088000202564000D5365724E722E2025386C753C
:1008900000322E322E33004D432052657669736943
:1008A0006F6E200052455345540054504D207072D5
:1008B0006F6772616D004443432070726F677261AD
:1008C0006D00507772206F6E0048616C7465642112
:1008D00000507772206F66660054202564202563DF
:1008E00020256400464D2025752025752C256400A3
:1008F0002025642C256400464D202575004658208F
:100900002575004620257500444343004D6F746FE4
:10091000726F6C61204E6577004D6F746F726F6CF3
:1009200061204F6C64006D3300756E7573656400F3
:100930004C202575202575202563202563000002A5
:100940000C151D263039434C565F69727F00020733
:100950000C10151A1E23282C31363A3F44484D52AC
:10096000565B6064696E73797F0002070B1014197F
:100970001D22262B3035393F43484C51565B5F646E
:10098000696D72767B7F48616C746564210D5D00D2
:1009900046207B4C6F6B232C205B46315D2C205B0B
:1009A00046325D2C205B46335D2C205B46345D2C4B
:1009B000205B46355D2C205B46365D2C205B463740
:1009C0005D2C205B46385D7D0054207B54726E7434
:1009D000232C205B436F6C6F725D2C205B53746122
:1009E0007475735D7D004C207B4C6F6B232C205BFA
:1009F00053706565645D2C205B464C5D2C205B4428
:100A000069725D2C205B46315D2C205B46325D2C8B
:100A1000205B46335D2C205B46345D7D00485420CE
:100A200048656C7020666F72207475726E6F757495
:100A300020636F6D6D616E64730048462048656C7D
:100A40007020666F722066756E6374696F6E2063C6
:100A50006F6D6D616E64730D00484C2048656C705D
:100A600020666F72206C6F6B20636F6D6D616E64BA
:100A7000730D002530386C75004B75727A20283163
:100A80002E356D7329202000004C616E67202834BC
:100A90002E3032356D732900004D6F746F726F6C9C
:100AA000610000000000000000444343202020209B
:100AB0002000000000000000004D4D20000000005C
:100AC000000000000000000000444343000000005C
:100AD000000000000000000000706F736974697608
:100AE00020284D4D29000000006E6567617469760D
:100AF000202844434329000000303A2061757320C8
:100B0000202020202020202000313A205461696CD0
:100B1000626974732020202000323A202B2049641F
:100B20004E6F74696679202000333A202B20416390
:100B3000636573736F72792000416E6C6167656ED7
:100B40007A757374616E642000416E6C6167656EC6
:100B50007A757374616E64200057696564657268A4
:100B600065727374656C6C6E00537065696368655B
:100B7000726E202020202020002077696564657235
:100B800068657273742E2020002073706569636835
:100B900065726E202020202000436F75727420281B
:100BA000312E356D73292000004C6F6E672028347C
:100BB0002E3032356D732900004D6F746F726F6C7B
:100BC000610000000000000000444343202020207A
:100BD0002000000000000000004D4D20000000003B
:100BE000000000000000000000444343000000003B
:100BF000000000000000000000706F7369746976E7
:100C00006520284D4D290000006E65676174697686
:100C1000652028444343290000303A206F6666204F
:100C2000202020202020202000313A205461696CAF
:100C3000626974732020202000323A202B204964FE
:100C40004E6F74696679202000333A202B2041636F
:100C5000636573736F727920005265737461757286
:100C60006174696F6E20202000456E72656769733C
:100C70007472656D656E742000526573746175726F
:100C80006174696F6E20202000456E72656769731C
:100C90007472656D656E7420002045746174205215
:100CA00065736561752E20200020457461742052A3
:100CB00065736561752E2020004B6F72722028319C
:100CC0002E356D7329202000004C616E672028347A
:100CD0002E3032356D732900004D6F746F726F6C5A
:100CE0006100000000000000004443432020202059
:100CF0002000000000000000004D4D20000000001A
:100D00000000000000000000004443430000000019
:100D1000000000000000000000506F7369746965F6
:100D20006620284D4D290000004E65676174696595
:100D3000662028444343290000303A206F6666202D
:100D4000202020202020202000313A205461696C8E
:100D5000626974732020202000323A202B204964DD
:100D60004E6F74696679202000333A202B2041634E
:100D7000636573736F727920004D6F64656C626197
:100D8000616E7369742E2020004D6F64656C626122
:100D9000616E7369742E2020004865727374656CEF
:100DA0006C656E2020202020004F70736C61616E96
:100DB0002020202020202020002068657273746588
:100DC0006C6C656E2020202000206F70736C616158
:100DD0006E202020202020200073686F727420284D
:100DE000312E356D73292000006C6F6E672028341A
:100DF0002E3032356D732900004D6F746F726F6C39
:100E00006100000000000000004443432020202037
:100E10002000000000000000004D4D2000000000F8
:100E200000000000000000000044434300000000F8
:100E3000000000000000000000706F7369746976A4
:100E40006520284D4D290000006E65676174697644
:100E5000652028444343290000303A206F6666200D
:100E6000202020202020202000313A205461696C6D
:100E7000626974732020202000323A202B204964BC
:100E80004E6F74696679202000333A202B2041632D
:100E9000636573736F72792000526573746F726546
:100EA0002020202020202020005361766520202053
:100EB000202020202020202000526573746F72654E
:100EC0002020202020202020005361766520202033
:100ED000202020202020202000206C61796F757454
:100EE000207374617475732000206C61796F757460
:100EF0002073746174757320005B756E6B6E6F7711
:100F00006E207374617475735D00696E6B6F6D70C4
:100F100061742E20466F726D617400466F726D6150
:100F20007420696E636F6D7061742E00496E636F1B
:100F30006D702E20466F726D6174202000696E63A3
:100F40006F6D7061742E20466F726D6174005B75F9
:100F50006E6B6E6F776E206572726F725D002E2EF3
:100F60002E2077617274656E202E2E2E2020002395
:100F70003D4CF6736368656E0000000000000000E1
:100F8000286B65696E2045696E747261672900007F
:100F900000202E2E2E206CF673636865202E2E2ED8
:100FA0002000204665686C657200000000000000AB
:100FB000000000206E75722066FC722044434321BD
:100FC00020202000206572737420474F206472FC3B
:100FD000636B656E002A3D41626272756368000052
:100FE0000000000000002050726F6772616D6D6933
:100FF0006572756E6700002D2D204B75727A7363D4
:10100000686C75DF202D2D00204E617469762028D4
:10101000313A31292020202000204C696E65617210
:101020002028323A3129202020002050726F677228
:1010300065737369762031202020002050726F671D
:10104000726573736976203220202000204143208E
:101050004D6F647573202020202020200020444301
:10106000204D6F6475732020202020202000204117
:1010700075746F5374657020202020202020002A72
:101080006C6573656E000000000000000000000049
:101090002A736368722E0000000000000000000048
:1010A000002E2E2073636872656962656E202E2E95
:1010B00000002E2E2E206C6573656E202E2E2E20A5
:1010C000200000212121204665686C6572202121C5
:1010D00021200000204F4B202020202020202020F5
:1010E00020202000002E2E207370656963686572D1
:1010F0006E202E2E000077696564657268657273D4
:1011000074656C6C656E00233D4CF6736368656EA8
:10111000202A3D4162627200233D4A61202A3D41FE
:10112000626272756368000000206CF67363686524
:101130006E20202020202020200041555300000058
:1011400000000000000000000000002A2A206B655B
:10115000696E65204C6F6B202A2A20002A2A204BBA
:1011600075727A7363686C75DF202A2A002A205A08
:10117000656974FC626572736368722E2A00576534
:1011800069636865202534642F2534640000004BB2
:101190006F6E66696775726174696F6E20202000DA
:1011A000204B6F6E66696775726174696F6E20207F
:1011B0000050617469656E74657A0000000000007B
:1011C0000000233D7375707072696D6572000000D8
:1011D0000000007669646500000000000000000067
:1011E000000000005375707072657373696F6E0054
:1011F000000000000020457272657572000000005A
:101200000000000000002044434320756E697175A2
:10121000656D656E74200020707265737320474F92
:1012200020666972737400002A3D4162616E646FCA
:101230006E00000000000000002050726F677261B5
:101240006D6D6174696F6E0000002D436F7572746F
:101250002D636972637569742D2000206E61746955
:1012600076652028313A312920202000206C696ED3
:101270006561722028323A312920202000207072C6
:101280006F67726573736976652031202000207066
:10129000726F677265737369766520322020002053
:1012A0004143204D6F646520202020202020200015
:1012B000204443204D6F64652020202020202020E2
:1012C00000204175746F5374657020202020202009
:1012D00020002A4C6563742E00000000000000000E
:1012E0000000002A456372697400000000000000DD
:1012F000000000002E2E2E20456372697475726501
:10130000202E2E2E002E2E2E204C656374757265B5
:10131000202E2E2E2000212121204572726575720B
:1013200020212121202000204F4B20202020202080
:10133000202020202020200020456E7265676973E0
:101340007472656D656E74200020526573746175EA
:10135000726174696F6E20202000233D5375707098
:1013600072202A3D4162616E642E00233D4F7569F3
:10137000202A3D4162616E646F6E200020537570BB
:101380007072696D657220202020202000496E61F6
:1013900063746966202020202020202020002A203D
:1013A000506173206465206C6F636F202A20002ACF
:1013B00020436F7572742D636972637569742000C0
:1013C0002A2054656D7073206465706173736520A5
:1013D0000041696775696C2E2534642F25346400DB
:1013E0000000456E72656769737472656D656E7431
:1013F000202000526573746175726174696F6E208C
:10140000202020002E2E2E207761636874656E20C8
:101410002E2E2E2000233D77697373656E00000029
:10142000000000000000286765656E20696E766F19
:1014300065722900000000202E2E2E20776973731C
:10144000656E202E2E2E000020666F757400000041
:1014500000000000000000000020416C6C65656E1B
:1014600020444343212020202000207072657373A4
:1014700020474F20666972737400002A3D416662FE
:1014800072656B656E000000000000002050726FF6
:101490006772616D6D6572656E000000002D2D4BE9
:1014A0006F7274736C756974696E672D2D00206E90
:1014B00061746976652028313A3129202020002086
:1014C0006C696E6561722028323A31292020200033
:1014D0002070726F677265737369766520312020A2
:1014E000002070726F6772657373697665203220B1
:1014F0002000204143204D6F6465202020202020C3
:10150000202000204443204D6F64652020202020AF
:1015100020202000204175746F53746570202020B6
:1015200020202020002A4C657A656E000000000013
:101530000000000000002A53636872690000000088
:10154000000000000000002E2E2073636872696A9C
:1015500076656E202E2E00002E2E2E206C657A656C
:101560006E202E2E2E202000002021212120466FCB
:1015700075742021212120200000204F4B202020A5
:1015800020202020202020202000002E2E2E204F42
:1015900070736C61616E202E2E2E00004865727390
:1015A00074656C6C656E20202020200000233D7740
:1015B000697373656E202A3D616662720000233D87
:1015C0004A61202A3D41666272656B656E2000208B
:1015D00077697373656E2020202020202020200052
:1015E0005549540000000000000000000000000009
:1015F000002A2A2A206765656E204C6F63202A2AFC
:101600002A002A2A6B6F7274736C756974696E672D
:101610002A2A002A2054696A646F766572736368A7
:10162000722E2A0057697373656C732534642F25F5
:101630003464000000436F6E66696720202020201C
:1016400020202020200020436F6E66696720202024
:10165000202020202020002E2E2E20776169746902
:101660006E67202E2E2E2000233D64656C65746508
:10167000000000000000000000286E6F20656E74FE
:10168000727929000000000000002E2E2E206465D3
:101690006C6574696E67202E2E2E00206661756C55
:1016A00074000000000000000000000020444343DC
:1016B000206F6E6C79212020202020200020707265
:1016C00065737320474F20666972737400002A3D6A
:1016D00043616E63656C00000000000000000020A4
:1016E00070726F6772616D696E67000000000000C4
:1016F0002D73686F727420636972637569742D202D
:1017000000206E61746976652028313A31292020E5
:101710002000206C696E6561722028323A312920E0
:101720002020002070726F67726573736976652080
:10173000312020002070726F67726573736976655F
:101740002032202000204143204D6F64652020205E
:10175000202020202000204443204D6F646520205D
:1017600020202020202000204175746F5374657064
:1017700020202020202020002A72656164200000A3
:101780000000000000000000002A77726974650004
:10179000000000000000000000002E2E2E207772B6
:1017A0006974696E67202E2E2E20002E2E2E207238
:1017B000656164696E67202E2E2E20002121212074
:1017C0006661756C742021212120202000204F4B60
:1017D00020202020202020202020202020002E2E0D
:1017E0002E20736176696E67202E2E2E2020002E0B
:1017F0002E20726573746F72696E67202E2E200022
:10180000233D44656C2E202A3D43616E63656C2048
:1018100000233D596573202A3D43616E63656C204A
:10182000200020636F6E66696775726174696F6E00
:101830002020004F4646000000000000000000008D
:10184000000000002A2A2A206E6F20547261696EFF
:10185000202A2A2A002A2073686F72742063697212
:101860006375697420002A2A2A2074696D65206FC7
:101870007574202A2A2A00506F696E74202025343E
:10188000642F253464000000436F6E6669677572CB
:101890006174696F6E2020200020636F6E66696737
:1018A00075726174696F6E2020005B6E6F206D65CC
:1018B00073736167655D0025642A2A2A20464149C1
:1018C0004C555245202A2A2A0025643A2030782592
:1018D00030386C58002532642030782530386C5808
:1018E00020202000204D3320656E61626C656420ED
:1018F00020202020003D2535640030782530386CCC
:10190000580020253564002534646D730025336448
:101910002C25647300202E2E2E2E20202020202007
:10192000202020002564206D7300202532640031C2
:101930003200003234000034380000393600003103
:101940003434003139320033383400353736003022
:101950003020426175640025346400202D2D2D0057
:101960002020202020202000204F4B20202020005D
:10197000253364002D2D2D002534643A20002536B2
:101980006400202D2D2D2D2D0025346400202D2DBB
:101990002D0043563A253464204269743A25643D4B
:1019A0000043563A20202020204269743A203D20EE
:1019B0000025357500202D2D2D2D00414243444535
:1019C000464748494A4B4C4D4E4F5051525354553F
:1019D000565758595A303132333435363738392E14
:1019E0002C3A2D2B232F3D3C7C3E20004D4D204991
:1019F0002020313420004D4D204920203237610015
:101A00004D4D20492020323762004D4D20022020CC
:101A1000313420004D4D20022020323761004D4DE1
:101A200020022020323762004443432020203134FA
:101A300020004443432020203238200044434320E8
:101A40002031323820006D33202020313238200000
:101A50003A2000253575005365724E722E202538C8
:101A60006C7500322E322E3300536F6674772E2041
:101A70005600253364004E723A202532642020003F
:101A80004C6F6B204D656EFC0000000000000000F4
:101A90004443432D50726F6772616D6D672E000075
:101AA0006D332050726F6772616D6D672E0000009C
:101AB000416E6C6167656E7A757374616E64000067
:101AC00045696E7374656C6C756E67656E000000B9
:101AD000536F667477617265205570646174650038
:101AE0004C43442042656C6575636874756E67008D
:101AF0004D6173746572436F6E74726F6C00000099
:101B0000457869740000000000000000000000003B
:101B100041757377E4686C656E200000000000007A
:101B2000446174656E666F726D6174000000000040
:101B30004E616D6520202020202000000000000064
:101B400045696E747261672020200000000000006B
:101B500043562028627974652900000000000000C7
:101B6000435620286269742900000000000000002C
:101B700042617369732D416472657373650000007F
:101B80006C616E6765204164726573736500000067
:101B90005265676973746572000000000000000000
:101BA000506167652D4D6F64650000000000000006
:101BB0004861757074676C6569730000000000000F
:101BC0005261696C436F6D204356000000000000B5
:101BD0003132384653204D6F64650000000000002C
:101BE0005265676C65726D6F64757300000000006C
:101BF0007338382D45696E7374656C6C756E67004B
:101C00004B6F6E66696775726174696F6E00000074
:101C1000426F6F73746572000000000000000000E6
:101C2000496E746572666163652042617564000087
:101C30005765696368656E000000000000000000E1
:101C40004C6F6B666F726D617400000000000000E5
:101C50004D4D2D5369676E616C2050617573650041
:101C60005261696C436F6D20537570706F727400B0
:101C70007338382D4D6F64756C65000000000000EE
:101C80007338382D4D6F64756C7465737400000083
:101C90004B75727A7363686C2E2D506F6C2E00003A
:101CA0004B75727A7363686C2E2D456D70662E00CD
:101CB000616C6C65205765696368656E00000000A3
:101CC0005765696368656E666F726D6174000000C8
:101CD0006D696E2E20536368616C747A6569740057
:101CE0006D61782E20536368616C747A6569740045
:101CF0006D3320416472657373650000000000005D
:101D00004D656E75204C6F636F0000000000000091
:101D100050726F6772616D2E2044434300000000D3
:101D20006D332050726F6772616D6D672E00000019
:101D300045746174205265736561752E0000000062
:101D40005265676C61676573000000000000000069
:101D50004D414A206C6F67696369656C0000000043
:101D60004C756D696E6F736974650000000000004A
:101D70004D6173746572436F6E74726F6C00000016
:101D800045786974000000000000000000000000B9
:101D900053656C656374696F6E200000000000007D
:101DA000466F726D617420646F6E6E6565730000BE
:101DB0004E6F6D2020202020202000000000000019
:101DC0005361697369652020202000000000000035
:101DD0004356202862797465290000000000000045
:101DE00043562028626974290000000000000000AA
:101DF0004164726573736520646520626173650078
:101E000041647265737365206C6F6E677565000061
:101E1000526567697374657200000000000000007D
:101E2000506167652D4D6F64650000000000000083
:101E3000566F6965207072696E636970616C6500C8
:101E40005261696C436F6D20435600000000000032
:101E50003132384653204D6F6465000000000000A9
:101E60004A6F676469616C204D6F64650000000013
:101E70005265676C616765207338380000000000A8
:101E8000436F6E66696775726174696F6E000000FA
:101E9000426F6F7374657200000000000000000064
:101EA000496E746572666163652042617564000005
:101EB000436F6E662E2041696775696C6C612E00F8
:101EC000466F726D6174206C6F636F0000000000DC
:101ED0005061757365207369676E616C204D4D00AC
:101EE0005261696C436F6D20537570706F7274002E
:101EF0004D6F64756C657320733838000000000006
:101F000054657374206D6F64756C65207338380088
:101F1000506F6C2E6372742D6369726375697400FF
:101F200053656E732E206372742D6369726374003F
:101F3000746F75732061696775696C6C612E000040
:101F4000466F726D61742061696775696C6C2E00F3
:101F5000547073206D696E2E696D70756C732E00F0
:101F6000547073206D61782E696D70756C732E00DE
:101F700041647265737365206D33000000000000DA
:101F80004C6F636D656E750000000000000000007E
:101F90004443432D70726F6772616D6D2E000000B7
:101FA0006D332D70726F6772616D6D672E0000006A
:101FB0004D6F64656C6261616E7369742E00000020
:101FC000496E7374656C6C696E67656E0000000025
:101FD000536F667477617265205570646174650033
:101FE0004C4344207665726C69636874696E67005F
:101FF0004D6173746572436F6E74726F6C00000094
:102000004578697400000000000000000000000036
:102010004B69657A656E200000000000000000003A
:1020200044617461666F726D6174000000000000AD
:102030004E61616D20202020202000000000000063
:10204000496E766F6572202020200000000000009D
:1020500043562028627974652900000000000000C2
:102060004356202862697429000000000000000027
:10207000426173697361647265730000000000005F
:102080004C616E672061647265730000000000009F
:1020900052656769737465720000000000000000FB
:1020A000506167652D4D6F64650000000000000001
:1020B000486F6F666473706F6F72000000000000FD
:1020C0005261696C436F6D204356000000000000B0
:1020D0003132384653204D6F646500000000000027
:1020E0004A6F676469616C204D6F64650000000091
:1020F0007338382D696E7374656C6C696E67656EC4
:10210000436F6E66696775726174696500000000EF
:10211000426F6F73746572000000000000000000E1
:10212000496E746572666163652042617564000082
:1021300057697373656C0000000000000000000028
:102140004C6F63666F726D617400000000000000E8
:102150004D4D207369676E61616C7061757A6500C1
:102160005261696C436F6D20537570706F727400AB
:102170007338382D6D6F64756C65000000000000C9
:102180007338382D6D6F64756C65746573740000F9
:102190004B6F7274736C2E20706F6C2E00000000F9
:1021A0004B6F7274736C2E206765762E00000000F2
:1021B000616C6C652057697373656C730000000077
:1021C00057697373656C666F726D6174000000000F
:1021D0004D696E2E736368616B656C74696A640027
:1021E0004D61782E736368616B656C74696A640015
:1021F0006D33206164726573000000000000000010
:102200004C6F636F6D6F74697665206D656E7500D8
:102210004443432070726F6772616D6D696E670031
:102220006D332070726F6772616D6D696E6700004B
:102230004C61796F7574207374617475730000005C
:1022400053657474696E677300000000000000003D
:10225000536F6674776172652055706461746500B0
:102260004C4344206261636B6C69676874000000D2
:102270004D6173746572436F6E74726F6C00000011
:1022800045786974000000000000000000000000B4
:1022900053656C65637420000000000000000000BE
:1022A0004461746120666F726D617400000000000B
:1022B0004E616D65202020202020000000000000DD
:1022C000456E74727920202020200000000000005C
:1022D0004356202862797465290000000000000040
:1022E00043562028626974290000000000000000A5
:1022F0005072696D617279206164647265737300F4
:10230000457874656E642E20616464726573730031
:102310005265676973746572000000000000000078
:10232000506167652D4D6F6465000000000000007E
:102330004D61696E20747261636B000000000000E3
:102340005261696C436F6D2043560000000000002D
:102350003132384653204D6F6465000000000000A4
:102360004A6F676469616C204D6F6465000000000E
:102370007338382073657474696E677300000000E9
:1023800044656C65746500000000000000000000FA
:10239000426F6F737465720000000000000000005F
:1023A000496E746572666163652042617564000000
:1023B000506F696E747300000000000000000000A0
:1023C0004C6F632E20666F726D6174000000000018
:1023D0004D4D207369676E616C2070617573650087
:1023E0005261696C436F6D20537570706F72740029
:1023F000733838206D6F64756C65730000000000E1
:10240000733838206D6F64756C6520746573740063
:1024100053686F727420632E20706F6C2E00000062
:1024200053686F727420632E2073656E732E0000E4
:10243000616C6C20506F696E7473000000000000C6
:10244000506F696E747320666F726D617400000066
:102450006D696E2E7377697463682E74696D65009B
:102460006D61782E7377697463682E74696D650089
:102470006D332061646472657373000000000000B6
:10248000446F776E6C6F6164202E2E2E20202020EA
:10249000000011241FBECFEFD0E1DEBFCDBF12E0A0
:1024A000A0E0B1E0EEEBFBE501E00BBF02C007905E
:1024B0000D92A637B107D9F71EE0A6E7B2E001C03A
:1024C0001D92AE3BB107E1F70E94C5120C94DDAD41
:1024D0000C94000080917602089581E08093770249
:1024E000089580E00E94746881E00E9474680E94F0
:1024F000AC780E94C88E0E94B03F809177028823FA
:1025000011F40E94C41EA8950895982F8091760218
:102510008917C9F18630B9F1853011F4963099F5F3
:1025200090937602892F8250823010F0973059F4C0
:102530000E946C371092D80780917602823029F47D
:102540000E945C3902C00E946B3280917602863014
:1025500011F40E94C36C80917602813011F482E004
:1025600003C0882321F481E064E00E94719184E03B
:1025700064E00E947191809176020E94657A81E008
:1025800080937702089580E00895EF92FF920F9371
:102590001F93CF93DF930E94926F0E94D3130E94E8
:1025A000F63A0E94168D0E94E9300E947F6C68E026
:1025B0004EE421E00E94011487E068E04EE421E04F
:1025C0000E9490150E94991878940E946A1C0E949B
:1025D0007C6CDC0114968C910E94BF1E82E06DEA37
:1025E00070E00E941C210E949E6C8130D9F482E030
:1025F00069EA70E00E941C2181E060E00E94481FAF
:1026000082E066E50E94422082E06CE870E00E9471
:102610001C210E947C6CEC0181E00E94401D8823FB
:1026200049F125C00E949E6C00D000D00F92EDB7FA
:10263000FEB7319692E0ADB7BEB711969C9322EAF1
:1026400030E032832183838314820E94C2200F9062
:102650000F900F900F900F9081E060E00E94481F54
:1026600082E062E970E00E941C21A895FECF81E023
:102670000E943E6F82E00E94401D882319F080E096
:102680000E943E6F83E00E94401D882319F082E083
:102690000E943E6F84E00E94401D882319F083E071
:1026A0000E943E6F80E00E94851285E10E94401DDD
:1026B000882311F00E94641D81E00E94B68080E0B2
:1026C0000E94401D882319F088E10E948BA60E9479
:1026D000EA848FEF60E240E050E00E94BE7080E04C
:1026E0000E94DB6B81E00E94DB6B0E94F69002C0CF
:1026F0000E9471128091DA079091DB07A091DC07AC
:10270000B091DD07805D9740A040B04088F3E09035
:10271000DA07F090DB070091DC071091DD0784E613
:1027200090E0A0E0B0E0E80EF91E0A1F1B1F96988B
:102730008E9A02C00E9471128091DA079091DB0795
:10274000A091DC07B091DD078E159F05A007B107AA
:1027500088F38E98969A89859A85009749F060E06B
:1027600070E040E050E00E941A86BC01009711F42E
:102770006A817B818FEF0E94CA6E81E011C00E9446
:102780000C460E947E1DAFEF8F3F9A07C1F70E9453
:102790007112809177028823A1F31092770280E072
:1027A0000E94DB40EECF8FE78ABB1BBA80E187BB7C
:1027B00018BA80EF84BB8FEF85BB8BEB81BB8CECB1
:1027C00082BB82E082B987EF83B987E7809361009B
:1027D00081EE8093620087E18093640089E18093B9
:1027E00065000E94068110926A001ABE8AB78A604C
:1027F0008ABF0E946619A89588E181BD8EE081BDDF
:102800000895109294079091940790939307909154
:1028100093079093B6079091B6079093B50791E010
:102820009093D7078C9A119A92B19E7E92B9199A79
:1028300093B19E7E93B992E09BB99498883008F04A
:1028400087E0E82FF0E0EE0FFF1FE754FF4FA59160
:10285000B491653010F465E003C0693008F068E0B9
:102860004F7D6550660F453411F4606203C04F34EC
:1028700009F46063223008F068608B2F992787FD88
:102880009A958F7080939000A9B96093950088EB1A
:102890008AB980E090E008951F920F920FB60F92D0
:1028A0000BB60F9211248F939F93EF93FF93909108
:1028B000B5078091B607981761F088B7806188BF27
:1028C0000C9B09C08091D70780FF05C089B7806144
:1028D00089BF559812C0E091B607F0E0ED56F84F69
:1028E00084A18CB98091B6078F5F8093B6078091E1
:1028F000B607803210F01092B607FF91EF919F91CA
:102900008F910F900BBE0F900FBE0F901F901895D8
:102910001F920F920FB60F9211248F9389B78F7E5B
:1029200089BF559A8F910F900FBE0F901F901895E9
:1029300027E0813D9207C0F12FE0813A920710F421
:1029400081E01EC023E28932920710F482E018C0B1
:1029500026E3813B920710F483E012C026E4813520
:10296000920710F484E00CC028E8893B920710F429
:1029700085E006C0895D964D10F087E001C086E0D5
:10298000789420E030E05E9902C020E030E02F5FD4
:102990003F4FA89597E220313907A8F368E04EE44D
:1029A00021E00E940114089580E0EACF8330C9F04D
:1029B000843028F4813061F0823080F40CC085309E
:1029C000B1F0853088F08630A9F08730C9F415C0A1
:1029D00020E639E017C020EB34E014C020EC32E1EF
:1029E00011C020E835E20EC020E438E30BC020E03F
:1029F0003BE408C020E036E905C020E031EE02C02B
:102A000020E030E0C901089539B120919000922F63
:102A100080E0232F30E0282B392B49EB50E060E099
:102A2000FA01859194918217930729F06F5F4E5FA9
:102A30005F4F6830A9F7862F0E94D6140895482F5B
:102A4000A89503C0559A7894A8952091B5078091D0
:102A5000B60730E090E001972817390799F3809185
:102A6000B5078F3121F48091B607882359F3E0919F
:102A7000B507F0E0ED56F84F44A39FB7F894809166
:102A8000B5078F5F8093B5078091B507803210F04E
:102A90001092B5079FBF559A80E090E00895F89492
:102AA0008091930790919407282F30E0291B3109DA
:102AB000789437FF02C0205E3F4F2031310534F457
:102AC0009498232B19F42FEF3FEF15C0E091940752
:102AD000F0E0ED56F84F9281F894809194078F5F63
:102AE0008093940780919407803210F0109294079D
:102AF000292F30E07894C90108959091D707882351
:102B000031F08091D70781608093D70706C080910C
:102B1000D7078E7F8093D707559A892F81700895A4
:102B200010924F0790914F0790934E0790914E0748
:102B300090937107909171079093700791E0909333
:102B4000920791B3986291BB8A981598939A92983C
:102B50001D9892E090939B009598883008F087E04C
:102B6000E82FF0E0EE0FFF1FE754FF4FA591B4915F
:102B7000653010F465E003C0693008F068E04F7D0F
:102B80006550660F8B2F992787FD9A958F708093DC
:102B90009800A0939900453411F4606203C04F344B
:102BA00009F46063223008F0686060939D0088EB50
:102BB00080939A0080E090E008951F920F920FB6E4
:102BC0000F920BB60F9211248F939F93EF93FF9365
:102BD0009091700780917107981761F088B78062B3
:102BE00088BF0D9B0DC08091920780FF09C089B7F7
:102BF000806289BF80919A008F7D80939A0013C074
:102C0000E0917107F0E0E25BF84F84A180939C00B3
:102C1000809171078F5F8093710780917107803277
:102C200010F010927107FF91EF919F918F910F908B
:102C30000BBE0F900FBE0F901F9018951F920F9212
:102C40000FB60F920BB60F9211248F93EF93FF9351
:102C500089B78F7D89BFEAE9F0E080818062808357
:102C6000FF91EF918F910F900BBE0F900FBE0F90C1
:102C70001F901895482FA89507C080919A008062F0
:102C800080939A007894A89520917007809171079D
:102C900030E090E001972817390779F380917007A9
:102CA0008F3121F480917107882339F3E091700707
:102CB000F0E0E25BF84F44A39FB7F894809170076F
:102CC0008F5F8093700780917007803210F01092B0
:102CD00070079FBF80919A00806280939A0080E085
:102CE00090E00895F89480914E0790914F07282F17
:102CF00030E0291B3109789437FF02C0205E3F4F36
:102D00002031310534F49598232B19F42FEF3FEF40
:102D100015C0E0914F07F0E0E25BF84F9281F89424
:102D200080914F078F5F80934F0780914F078032CC
:102D300010F010924F07292F30E07894C9010895C0
:102D40009091D707882331F080919207816080931A
:102D500092070AC0809192078E7F8093920780919C
:102D60009A00806280939A00892F817008951F9243
:102D70000F920FB60F920BB60F9211242F933F9321
:102D80004F935F936F937F938F939F93AF93BF9373
:102D9000EF93FF9320914E0780914F0730E090E032
:102DA00001972817390741F080914E078F3179F448
:102DB00080914F07882359F480914F078F5F80934C
:102DC0004F0780914F07803210F010924F0780918B
:102DD0009B00E0914E07F0E090919C00E25BF84F81
:102DE0009283928184FD0CC080914E078F5F809307
:102DF0004E0780914E07803278F010924E070CC03B
:102E0000992351F410924F0780914F0780934E07FA
:102E1000959881E00E94DB6B80914E0790914F075F
:102E2000282F30E0291B310937FF02C0205E3F4FB9
:102E3000213131050CF0959AFF91EF91BF91AF913F
:102E40009F918F917F916F915F914F913F912F91C2
:102E50000F900BBE0F900FBE0F901F9018951F92F2
:102E60000F920FB60F920BB60F9211242F933F9330
:102E70004F935F936F937F938F939F93AF93BF9382
:102E8000EF93FF93209193078091940730E090E0B7
:102E900001972817390741F0809193078F3179F412
:102EA00080919407882359F4809194078F5F8093D1
:102EB000940780919407803210F0109294078BB1A0
:102EC000E0919307F0E09CB1ED56F84F9283928128
:102ED00084FD0CC0809193078F5F8093930780914E
:102EE00093078032A8F01092930712C0992381F4BF
:102EF000109294078091940780939307949880E0B0
:102F00000E94DB6B81E068E04EE421E00E94011446
:102F10008091930790919407282F30E0291B310965
:102F200037FF02C0205E3F4F213131050CF0949AEB
:102F3000FF91EF91BF91AF919F918F917F916F9191
:102F40005F914F913F912F910F900BBE0F900FBE4D
:102F50000F901F90189578941F920F920FB60F92B2
:102F60000BB60F9211248F939F93EF93FF938FB122
:102F7000E0917802F0E0E858FD4F8283809178027A
:102F80008F5F8093780280917802803410F01092E5
:102F900078029091790280917802981759F4809183
:102FA00079028F5F8093790280917902803410F0EA
:102FB000109279029091BB028091BA02981711F495
:102FC0006F981DC0E091BB02F0E0E454FD4FE0813A
:102FD000E7FDC09A8091BB028F5F8093BB02809116
:102FE000BB02803210F01092BB0280E000000000B3
:102FF000000000008F5F8A30C9F7C098EFB9FF91D9
:10300000EF919F918F910F900BBE0F900FBE0F907D
:103010001F9018958091BB029091BA02282F30E042
:10302000215E3F4F291B31092032310514F0205217
:103030003040C9010895482F6F9934C0C0988EB1AF
:103040008FB16F9A9091BA028091BB02981711F4D8
:103050004FB94BC0E091BB02F0E0E454FD4F8081DA
:103060008FB98091BB028F5F8093BB028091BB02BE
:103070008032C0F01092BB0215C06F9913C0E0916E
:10308000BB02F0E0E454FD4F80818FB98091BB0218
:103090008F5F8093BB028091BB02803210F0109250
:1030A000BB026F9A8091BA022091BB0290E0019618
:1030B00030E08217930709F38091BA028F3121F42F
:1030C0008091BB028823C9F2E091BA02F0E0E45497
:1030D000FD4F40838091BA028F5F8093BA02809146
:1030E000BA02803210F01092BA0280E090E00895A7
:1030F0004FB7F8949091780280917902981719F45B
:103100002FEF3FEF13C0E0917902F0E0E858FD4F58
:103110008281282F30E0809179028F5F809379023D
:1031200080917902803410F0109279024FBFC9016A
:10313000089587B3876087BBBB9888B3896088BBD5
:1031400084E6E8E7F2E0DF011D928A95E9F71DB811
:103150008EB18FB187E78DB90895882311F0DD9A7C
:103160000895DD980895882351F08091650084606A
:103170008093650000000000000000000895809129
:1031800065008B7F8093650008950F931F93DF93F5
:10319000CF930F92CDB7DEB7182F8AB3807F8ABB4B
:1031A00080E00E94B3188091650082608093650082
:1031B000112321F080916500816003C0809165003A
:1031C0008E7F809365000000000081E00E94B318AC
:1031D00009B380E00E94B31810E084E0000F111FD3
:1031E0008A95E1F7000000000000000081E00E94E5
:1031F000B31899B39F70902B80E099830E94B31805
:103200008AB38F608ABB9981892F0F90CF91DF910C
:103210001F910F91089580E00E94C518982F87FF95
:1032200011C08091DF029091E00228E08130920786
:1032300014F080E0089501969093E0028093DF02FD
:1032400081E008958091E602882319F49F77909396
:10325000E7021092E0021092DF0280E008959B01E5
:10326000AC018091DA079091DB07A091DC07B09167
:10327000DD0782179307A407B50798F08091DA0756
:103280009091DB07A091DC07B091DD0760E0821B25
:10329000930BA40BB50B80509041A040B040A0F41C
:1032A00012C08091DA079091DB07A091DC07B09102
:1032B000DD0760E0281B390B4A0B5B0B2050304FB9
:1032C0004F4F5F4F08F061E0862F089510927D0008
:1032D00080B7877F80BF17BE11BE89E683BF8BE0B2
:1032E00085BD8FE183BD87B7806887BF82EF8FBDC3
:1032F0003AE13EBD4FEC50E057BD46BD85EB90E056
:103300009BBD8ABD99BD88BD22EC20938B00309374
:103310008A005093810040938000909387008093AF
:1033200086000895EF92FF920F931F932091DA0782
:103330003091DB074091DC075091DD077C0100E014
:1033400010E0E20EF31E041F151F01C0A895C8016E
:10335000B7010E942F198823C9F31F910F91FF9085
:10336000EF900895FF920F931F93082F162FF42EBE
:10337000809165008D7F8093650080E00E94B31886
:103380008AB38F608ABB8BB3902F92959F70807F9A
:10339000982B9BBB112321F080916500816003C0B5
:1033A000809165008E7F8093650081E00E94B31854
:1033B00080E00E94B318FF2029F088E090E00E948E
:1033C00092190FC08BB30F70807F802B8BBB0000D6
:1033D00000000000000081E00E94B31880E00E941D
:1033E000B3181F910F91FF900895EF92FF920F93E2
:1033F0001F932091DA073091DB074091DC07509151
:10340000DD077C0100E010E0E20EF31E041F151F33
:1034100002C00E947112C801B7010E942F198823AF
:10342000C1F31F910F91FF90EF9008950F931F9399
:10343000282F8091E502893018F48F5F8093E50290
:103440008091E5028430B1F0853048F4823009F48F
:10345000C0C0833008F0BAC08130E9F409C08630BA
:10346000B1F0863090F08730A1F08830A1F4B1C07F
:10347000DC9AAFC01092E4021092E30280E090E880
:103480009093E2028093E10206C0DD9AA2C0DD982B
:10349000A0C0DC989EC0222309F098C06091E3028E
:1034A0007091E4022091E1023091E202CF9B3CC096
:1034B000FB01EE0FFF1FEC5AF24F808191818223B6
:1034C0009323892B61F488E49DE00E9458926091D7
:1034D000E3027091E4028EE49DE00E945892E09134
:1034E000E302F091E4022091E1023091E202EE0F5A
:1034F000FF1FDF01A152B34F8D919C911197822B39
:10350000932B8D939C93DF01A958B34F8D919C9180
:103510001197822B932B8D939C93EC5AF24F8081C1
:103520009181822B932B29C0FB01EE0FFF1FEC5AD8
:10353000F24F8081918182239323892B61F088E46B
:103540009DE00E9458926091E3027091E4028EE443
:103550009DE00E945892E091E302F091E402EE0FA8
:10356000FF1FEC5AF24F8091E1029091E2028095A8
:103570009095208131818223932391838083809150
:10358000E1029091E202969587959093E2028093F2
:10359000E102892BE9F40091E3021091E4020F5F4C
:1035A0001F4F1093E4020093E3020E947C6CFC0125
:1035B000808590E00817190710F01092E50280E06E
:1035C00090E89093E2028093E10202C0DE9A01C08B
:1035D000DE981F910F9108951F920F920FB60F92D0
:1035E0000BB60F9211241F932F933F934F935F932A
:1035F0006F937F938F939F93AF93BF93EF93FF93BB
:103600008091DC02882309F051C181E08093DC02C3
:10361000789480E00E94161A8091DE028F5F80937A
:10362000DE028091DE0290E083709070813091051F
:1036300019F1823091051CF4892B41F0E5C08230EC
:10364000910561F1039709F0DFC065C08091DA0749
:103650009091DB07A091DC07B091DD070196A11DD9
:10366000B11D8093DA079093DB07A093DC07B0933A
:10367000DD070E944C1DC8C08091DA079091DB07DE
:10368000A091DC07B091DD0781709070892B19F053
:103690000E949A1DB9C00E94041DB6C00E946A1201
:1036A000833049F00E946A12823029F00E946A1227
:1036B000873009F0A9C00E94CA302091D807309104
:1036C000D9078823E9F02E5F3F4F3093D907209325
:1036D000D8070E947C6CFC019681992309F494C060
:1036E0008AE0989FC00111242091D8073091D90712
:1036F0002817390708F488C081E00E94851284C029
:103700002115310509F480C0215030403093D9078C
:103710002093D80779C00E946A12833059F184300F
:1037200028F4813061F0823008F513C08730D9F178
:10373000883009F448C0843009F061C024C0809109
:10374000DA079091DB07A091DC07B091DD0786FFD7
:1037500004C080916200816003C0809162008E7F0E
:1037600080936200809162008F7E4CC080916200E5
:10377000816148C080916200806180936200809185
:1037800062008E7F3FC0809162008E7F80936200D6
:103790008091DA079091DB07A091DC07B091DD07FB
:1037A00090FFE0CF1FC0809162008E7F8093620007
:1037B0008091DA079091DB07A091DC07B091DD07DB
:1037C00091FFD0CF0FC08091DA079091DB07A091D5
:1037D000DC07B091DD0787FF09C0809162008E7F12
:1037E000809362008091620080610CC080916200D1
:1037F0008F7E8093620080916200816003C080911F
:1038000062008E7E809362008091DD02882321F029
:103810000E940B198093DD028091DD02882309F05C
:1038200040C09091DE078091DF079817B9F1809131
:10383000DF07E82FF0E0E252F84F9281182F1F5F68
:10384000103108F010E0903801F58091DE07811703
:1038500029F1E12FF0E0E252F84F92819F3F19F4F5
:103860009091E702906897FF02C01092E602892FBC
:10387000807C803419F481E08093E6021F5F103170
:1038800008F010E0892F60E002C0892F61E040E07D
:103890000E94B2191093DF0781E001C080E080939D
:1038A000DD0281E00E94161A1092DC02FF91EF9176
:1038B000BF91AF919F918F917F916F915F914F9148
:1038C0003F912F911F910F900BBE0F900FBE0F9045
:1038D0001F901895CF93DF9388E290E00E94921991
:1038E00080E360E041E00E94B21980E360E041E0E3
:1038F0000E94B21980E360E041E00E94B21980E2C8
:1039000060E041E00E94B21988E20E94321F80E428
:103910000E94321F8AE00E94FF1E89E20E94321F2D
:103920008CE10E94321F82E50E94321F89E60E94CC
:10393000321F84E70E94321F80E40E94321F85E11B
:103940000E94FF1E88E20E94321F80E40E94321F04
:103950000E943C3EEC0101C0A8959091DE07809149
:10396000DF079817C9F70E940B198823A9F781E090
:103970000E94C5188A3019F481E089AB01C019AAE8
:1039800088E00E94321F81E00E94321F86E00E9480
:10399000321F8CE00E94321F80E060E00E94481FCE
:1039A00080E062EE70E00E94292081E066E271E032
:1039B0000E94292082E06EE271E00E94292083E0CB
:1039C0006EE371E00E942920DF91CF9108959091DC
:1039D000EA02E92FF0E0E651FD4F82839F5F90936A
:1039E000EA02983010F01092EA029091EB02809176
:1039F000EA02981741F4892F8F5F8093EB02883099
:103A000010F01092EB02089531B12091E902220FDB
:103A100036FD2160822F83708150823028F424FF8C
:103A200002C02E6001C0217F2093E9029091E8023C
:103A3000990F37FD9160892F83708150823028F46F
:103A400094FF02C09E6001C0917F9093E802207CA9
:103A5000892F807C203831F4882341F0803C79F430
:103A60008AE105C0203459F4803C21F489E10E94A8
:103A7000E71C0895882319F48AE10E94E71C089541
:103A8000893110F080E00895E82FF0E0EB50FD4F11
:103A90008081811181E0089530912703343029F429
:103AA00085B3806F85BB97980895979A25B380E179
:103AB00090E002C0880F991F3A95E2F78095807FC9
:103AC0002F70822B85BB089581E08093F4020895C6
:103AD0008091F402882389F08091DA079091DB07C6
:103AE000A091DC07B091DD0789589341A040B04018
:103AF00020F00E946C6F1092F40208950E94681DDD
:103B00009091EB028091EA02891719F42FEF3FEFB1
:103B10000FC0E92FF0E0E651FD4F8281282F30E001
:103B2000892F8F5F8093EB02883010F01092EB02A8
:103B3000C90108958F929F92AF92BF92CF92DF9268
:103B4000EF92FF920F931F93CF93DF930E946A121D
:103B5000982F80912803981729F09093280382E2E8
:103B60000E94E71C83B3E1B0EE0CEE0C90E1E92279
:103B70008F70E82ACC24DD2495E0A92E81E0882EE0
:103B8000912CBB24B394E0912703EA9DF00111240A
:103B9000EC0DFD1DE753FF4FF49088E18F1508F4FD
:103BA00097C00E2D08250170CF2DD0E0FE01E25FF9
:103BB000FC4F1081110F0E949E6C803819F4002375
:103BC00071F009C001111160812F90E08171907036
:103BD0008131910511F41F6103C0892B09F4107E16
:103BE000812F90E0807690708034910519F41F71D8
:103BF00082E00CC08032910519F4106E81E006C09D
:103C00008036910511F080E001C083E0FE01E25FA3
:103C1000FC4F1083823091F0833099F1813009F0AC
:103C200057C096E1F91621F480910A03882319F40C
:103C30008F2D0E94E71CCB50DD4F3DC0CB50DD4F98
:103C400018828F2D80680E94E71C0E946A128530BE
:103C500091F485E1F81629F480910B03882341F053
:103C60000DC096E1F916A1F580910A03882381F52C
:103C700086E00E94851285E1F81651F51092F40253
:103C800027C0FE01EB50FD4F80818F5F808388232A
:103C900009F4B08295E1F916D8F086E18F1568F441
:103CA00097E1F916A9F4CB50DD4F8881853680F075
:103CB00081E20E94E71CB8820BC080910A03893719
:103CC00038F080910B03893718F085E00E94851247
:103CD0000894C11CD11C85E0C816D10411F0E694EB
:103CE00052CF809127038F5F80932703853010F098
:103CF00010922703DF91CF911F910F91FF90EF90CA
:103D0000DF90CF90BF90AF909F908F900895909349
:103D10000B0880930A08892B89F170930908609336
:103D200008088091DA079091DB07A091DC07B09139
:103D3000DD079B0140E050E0280F391F4A1F5B1F41
:103D40002093040830930508409306085093070811
:103D5000809103088E7F809303082115310541056A
:103D6000510561F481E090E0A0E0B0E080930408A8
:103D700090930508A0930608B0930708089581332F
:103D800008F080E381BF089580910A0890910B08A4
:103D9000892BA1F1609104087091050880910608B3
:103DA000909107080E942F19882341F18091030800
:103DB000E0910A08F0910B08817009958091030841
:103DC00091E08927809303082091DA073091DB077F
:103DD0004091DC075091DD07809108089091090817
:103DE000A0E0B0E0820F931FA41FB51F80930408CA
:103DF00090930508A0930608B093070808951F93B1
:103E0000182F09C080E00E94746881E00E947468E5
:103E10000E94AC78A8952091DE078091DF0730E002
:103E200090E001972817390769F38091DE078F30FA
:103E300021F48091DF07882329F3F894E091DE07CD
:103E4000F0E0E252F84F12838091DE078F5F80939B
:103E5000DE078091DE07803110F01092DE07789443
:103E60001F9108951F93182F80E80E94FF1E812F35
:103E70000E94FF1E1F91089510920B0810920A08CD
:103E800081E00E94321F08958CE00E94321F089545
:103E90008295880F880F807C860F80680E94321F71
:103EA0000895BF92CF92DF92EF92FF920F931F93EC
:103EB000CF93DF93C82EB62E8A0110920B08109272
:103EC0000A0821E02817A0F13FE0361788F14115D4
:103ED000510571F1FA0101900020E9F73197DE2ECA
:103EE000D41A80E18D1510F490E1D92E8C2D6B2D14
:103EF0000E94481FE80180EFE82E87E0F82E08C0F6
:103F00008881F70181937F01699182E00E944220BC
:103F10009E01201B2D15A0F3C0920008B09201084D
:103F2000D09202088BEC9FE164EF71E00E94871E43
:103F3000DF91CF911F910F91FF90EF90DF90CF9085
:103F4000BF900895DF93CF93CDB7DEB7A0970FB69C
:103F5000F894DEBF0FBECDBFDE0111969E01205E3C
:103F60003F4F04C09D93A217B30731F0FA014F5F92
:103F70005F4F94919923B1F71C92AE014F5F5F4F51
:103F80000E94511FA0960FB6F894DEBF0FBECDBFA2
:103F9000CF91DF9108950F931F93CF93DF93082F55
:103FA00080910008609101080E94481F10E0C0EF56
:103FB000D7E009C0002311F460E201C0699182E0FA
:103FC0000E9442201F5F80910208181798F3DF912A
:103FD000CF911F910F9108950E94481F8EE00E947B
:103FE000321F0895EF92FF920F931F93CF93DF93A9
:103FF000382F7B01122F883028F5483018F5842F90
:1040000090E0820F911D099714F018E0141B330FF4
:10401000330F330F340F832F80640E94321FC0E0B0
:10402000D0E0012F10E008C0F701EC0FFD1FE49174
:104030008E2F0E94FF1E2196C017D107ACF38FEF81
:104040000E94321FDF91CF911F910F91FF90EF904F
:10405000089540E028E00E94F21F0895813069F041
:10406000813040F0833019F02FEF3FEF09C00E94FC
:104070007E1D05C00E944F1502C00E9472169C0151
:10408000C90108951F93162F813009F465C081304E
:1040900008F45EC0823009F062C067FF55C00E941C
:1040A0003C3EFC0181A98823E1F0143E11F414E8A0
:1040B0004BC0163F11F414E947C01C3F11F411E83E
:1040C00043C0143C11F41EE83FC0163D11F419E939
:1040D0003BC01C3D11F41AE937C0113F69F51BE9DB
:1040E00033C0143E11F411EE2FC0163F11F41FEE31
:1040F0002BC01C3F11F415EF27C0113F11F41EEE29
:1041000023C0143C39F484E06EEF71E00E94292052
:1041100014E01AC0163D39F485E066E072E00E94B2
:10412000292015E011C01C3D39F486E06EE072E0F4
:104130000E94292016E008C01F3D31F487E066E1A7
:1041400072E00E94292017E0812F0E94FF1E07C005
:10415000862F0E941F1503C0862F0E943A161F91BA
:1041600008951F93CF93DF93182FEB0104C021967E
:10417000812F0E94422068816623C9F7DF91CF9189
:104180001F9108950F931F93DF93CF93CDB7DEB7A1
:10419000C055D0400FB6F894DEBF0FBECDBF9E0114
:1041A000265A3F4F8E010F5F1F4FC8016A966EADB2
:1041B0007FAD6A97A9010E94BAAA68968FAD6897E9
:1041C000B8010E94B120C05BDF4F0FB6F894DEBF8C
:1041D0000FBECDBFCF91DF911F910F9108950F9327
:1041E0001F93DF93CF93CDB7DEB7C055D0400FB646
:1041F000F894DEBF0FBECDBF9E01265A3F4F8E0101
:104200000F5F1F4FC8016A966EAD7FAD6A97A90117
:104210000E9491AA68968FAD6897B8010E94B1205C
:10422000C05BDF4F0FB6F894DEBF0FBECDBFCF919E
:10423000DF911F910F9108951F93CF93DF93182F54
:10424000EB0104C0812F0E9442202196FE0164915F
:104250006623C1F7DF91CF911F910895582F5F70AA
:104260005F3011F45EE001C051115F5F442311F42F
:1042700090E001C098E0623061F0633018F4613082
:1042800069F405C0633039F0643041F406C09360CE
:1042900005C0946003C0966001C09760951739F41B
:1042A000442319F4592F95E002C0592F9AE080E079
:1042B00020E030E0880F880F50FD826090FD816023
:1042C0002F5F3F4F2430310519F056959695F2CF68
:1042D00090E00895962F9F709F3011F491E002C0F6
:1042E00091119F5F8370813071F480E020E030E0B5
:1042F000880F880F90FD83602F5F3F4F243031057A
:1043000001F19695F5CF67FD06C0983010F44DE0A9
:1043100007C045E005C0983010F042E001C04AE017
:1043200080E020E030E0880F880F90FD826040FD43
:1043300081602F5F3F4F2430310519F096954695E7
:10434000F2CF90E008959C01FB018038910520F4A4
:104350008F77808388E00895832F806C818320830A
:1043600080E10895F90108969C0153E03695279560
:104370005A95E1F72F73206821839C012095309591
:1043800095E0369527959A95E1F720778770282B49
:104390002083662319F0216020830BC0822F806860
:1043A0008083442311F028682083808191E089274D
:1043B000808380E108950F93CF93DF93EC01A62FC4
:1043C000A695A695A695862F877078E0781B04C0E1
:1043D000220F331F441F551F8A95D2F712C0FE01CA
:1043E000EA0FF11D8081822B8083872F071708F445
:1043F000802F680F081B232F342F452F5527AF5FC1
:1044000078E0002361F7862FDF91CF910F91089517
:104410000F93E42F8038910530F491609C0140E0C7
:1044200050E009E01AC022E08030920730F49C602E
:104430009C0140E050E00CE010C028E08030920782
:1044400030F490679C0140E050E00FE006C09C0112
:1044500040E050E0306C436002E1CB016E2F0E94DF
:10446000DB210F9108956FB7F89440910C0880916B
:104470000D08242F30E090E001972817390749F004
:104480004F3011F050E006C080910D0850E08823B5
:1044900009F451E06FBF6FB7F8944091BA0880916A
:1044A000BB08242F30E090E001972817390749F026
:1044B0004F3011F090E006C08091BB0890E0882357
:1044C00009F491E06FBF892F852B0895AF92BF92B9
:1044D000CF92DF92EF92FF920F931F93CF93DF93D0
:1044E000EC015A01122F80916803882309F057C00C
:1044F000013009F054C08981282F30E08881482F8D
:1045000050E03BC0808191818617970761F58281D9
:1045100093818A159B0539F58481813021F5868147
:104520009781A085B1850097A105B105E1F0F9015A
:1045300083E0EE0FFF1F8A95E1F7220F331FE20F92
:10454000F31FEC0FFD1F84899589A689B7898C1507
:104550009D05AE05BF0509F48FC0C48AD58AE68AD9
:10456000F78A138B89C0C90101963A9620E030E0A2
:104570008031910514F49C010EC0F901EE0FFF1F6C
:10458000C901A3E0880F991FAA95E1F7E80FF91F69
:104590003E96EC0FFD1F2417350709F0B3CFEFB798
:1045A000F8943881A32FB0E0898190E00197A81793
:1045B000B90741F03F3011F090E005C0898190E0EB
:1045C000882309F491E0EFBF992311F080E055C0F2
:1045D000FD0193E0EE0FFF1F9A95E1F7AA0FBB1FB5
:1045E000EA0FFB1FEC0FFD1F77876687888190E03D
:1045F000FC0163E0EE0FFF1F6A95E1F7880F991F3A
:10460000E80FF91FEC0FFD1FB18AA08A888190E0A6
:10461000FC0143E0EE0FFF1F4A95E1F7880F991F59
:10462000E80FF91FEC0FFD1F138B888190E0FC0150
:1046300023E0EE0FFF1F2A95E1F7880F991FE80F7F
:10464000F91FEC0FFD1F028B888190E0FC01B3E0A5
:10465000EE0FFF1FBA95E1F7880F991FE80FF91FBA
:10466000EC0FFD1FC48AD58AE68AF78A88818F5F9E
:104670008883803108F0188281E0DF91CF911F910B
:104680000F91FF90EF90DF90CF90BF90AF90089583
:1046900080916C0990E0833009F491E0892F0895AE
:1046A000FC01009729F1818590E083709070833040
:1046B000910534F48130910534F4892B61F018C0F0
:1046C0000397B1F404C080916703816007C08091B3
:1046D0006703826003C080916703846080936703EF
:1046E0008091670390E08770873019F091E001C0F6
:1046F00090E0892F0895809369030895809167035E
:1047000080720895809167038F7D80936703109274
:10471000800310927F03089590937E0380937D031E
:104720001092800310927F0308958FB7F8948FBF83
:1047300080917B0390917C0308958FB7F8948FBF8D
:1047400080917F0390918003089578941F920F9237
:104750000FB60F920BB60F9211242F933F938F93A6
:104760009F93EF93FF9380917A03883010F010921B
:104770007A0324B135B18091670384FF34C08091FE
:104780007A03E82FF0E0EE0FFF1FE659FC4F31836C
:1047900020838F5F80937A03EAE6F3E020E030E045
:1047A00081919191280F391F83E0EA37F807C1F70B
:1047B00030937C0320937B0380917F03909180034F
:1047C0008217930724F43093800320937F03809112
:1047D0007D0390917E03821793072CF480916703E9
:1047E000806280936703FF91EF919F918F913F913A
:1047F0002F910F900BBE0F900FBE0F901F9018952A
:10480000982F03C0892F862311F4990FD9F7892F88
:104810000895DC0152962C915297243009F04CC037
:1048200053969C915397292F215053962C9353972D
:1048300058968C915897813009F497C0843009F4C8
:1048400094C0803209F491C0803809F48EC082305F
:10485000E9F457968C915797883030F057961C9210
:10486000579753969C9325C0822F8695869586955B
:10487000FD01E80FF11D808190E0277002C0959541
:1048800087952A95E2F780FD09C011C0803179F043
:10489000803469F0883011F4223048F457968C91B6
:1048A00057978F5F57968C9323E330E063C05796FA
:1048B0001C922FEF3FEF5EC054968C915497882343
:1048C000C1F555968C915597882399F553963C914F
:1048D0005397932F915053969C935397233089F479
:1048E0005C968C915C97882361F49770973049F4BB
:1048F00081E05C968C935C9753963C93539790E041
:1049000019C05C961C925C9753962C915397822FFA
:10491000869586958695FD01E80FF11D808190E0D2
:10492000277002C0959587952A95E2F7982F917088
:1049300001C091E052968C91823029F0833099F039
:104940008130B1F408C0992319F420E130E012C09D
:104950002CE530E00FC0992319F42CE130E00AC0B7
:104960002EEB30E007C0992319F427E630E002C0AF
:104970002BE330E0C9010895CF93DF93DC01529619
:104980009C915297943009F0F2C058968C915897A8
:10499000813039F0843029F0803219F0803809F004
:1049A00051C083E0A932B80761F45C968C915C97A2
:1049B000882319F08FB58F7A02C08FB580658FBDBF
:1049C0000EC05C968C915C97882321F080918B00BF
:1049D0008F7A03C080918B00806580938B00539603
:1049E0008C91539780FD03C0C7E6D0E00CC090E0E7
:1049F0005C968C915C97882309F491E05C969C937B
:104A00005C97CAE9D0E053968C9153978823A1F420
:104A100058968C915897803879F483E0A932B8077A
:104A200021F48FB580658FBD05C080918B008065B6
:104A300080938B00CD5ED94F809167038F7E8093EA
:104A4000670351C083E0A932B807C1F488B599B5AE
:104A50008736910540F090E080914503882309F462
:104A600091E09093450380914503882319F08FB519
:104A70008F7A02C08FB580658FBD1FC08091860080
:104A8000909187008736910550F090E05C968C916C
:104A90005C97882309F491E05C969C935C975C9604
:104AA0008C915C97882321F080918B008F7A03C0D2
:104AB00080918B00806580938B0058968C915897DD
:104AC000803111F0803441F48091670380618093DC
:104AD0006703CDE4D8E107C0809167038F7E8093A0
:104AE0006703C7E6D0E053968C915397882309F06B
:104AF000D3C058969C915897923041F457968C9118
:104B00005797883018F0C7E6D0E0C6C059962C9168
:104B1000599703C0892F822311F4990FD9F758961A
:104B20009C93589757961C9257979031D1F091319A
:104B300040F4943091F0983091F0923009F0ACC08C
:104B400008C0903471F0903871F0903209F0A4C030
:104B500006C050968C91509707C08CE205C084E047
:104B600003C081E001C088E053968C9395C083E038
:104B7000A932B80721F48FB580658FBD05C080913B
:104B80008B00806580938B0054968C91549788237A
:104B900031F455968C915597882331F40BC0815090
:104BA00054968C93549704C0815055968C93559786
:104BB00081E01CC0933039F45C968C915C9788231B
:104BC00011F080E013C053962C915397822F869555
:104BD00086958695FD01E80FF11D808190E0277094
:104BE00002C0959587952A95E2F7817052969C911F
:104BF0005297923019F0933019F503C0CBE6D0E00C
:104C000021C0882319F4CEECD0E002C0C7E7D0E081
:104C100053968C9153978823A9F45B968C915B975C
:104C2000882381F48091690380FD02C082E001C085
:104C300086E055968C93559781E05B968C932CC0BB
:104C4000C7EDD0E053968C915397882329F555965C
:104C50008C915597882301F551968C91882399F46E
:104C60008091670380FF18C0809168038823A1F4B6
:104C700081E00E94896C882319F0C35BDF4E0CC071
:104C8000CD5ED94F09C0913029F0923029F4C85730
:104C9000DD4F02C0C05FDA4FCE01DF91CF910895A2
:104CA000FC018089838B8189823010F482E0818BC2
:104CB00082898330D1F0843018F48130C0F00AC08A
:104CC0008430A9F482E0868B91E0908F81898823DB
:104CD00009F4918B81E00E94896C882319F423E107
:104CE00036E007C02DE430E104C080E1848B22E38C
:104CF00030E0C901089580E1EAE6F3E0DF011D92AA
:104D00008A95E9F710927A0310927C0310927B0344
:104D10008FEF9FE790937E0380937D0308952F92FA
:104D20003F924F925F926F927F928F929F92AF923B
:104D3000BF92CF92DF92EF92FF920F931F93CF9388
:104D4000DF935C014B01442428E06A3B720711F4B5
:104D500044244394D40111969C9111978C91891706
:104D600009F036C1442029F480916703886080935C
:104D7000670380916803813041F4C40160E070E012
:104D800040E050E022E000E882C080916803823079
:104D900071F4C0906503D0906603EE24FF24C40133
:104DA00060E070E040E050E021E000EC0FC1809155
:104DB000690382FF27C0F40182819381A481B581B8
:104DC0000097A105B105F1F4C40160E070E040E096
:104DD00050E022E00EE8CC24DD2476010E94662219
:104DE0008091DA079091DB07A091DC07B091DD0795
:104DF00088519C4FAF4FBF4FF40182839383A483AC
:104E0000B583E6C08091690381FF30C0F4018681DB
:104E10009781A085B1850097A105B10539F5C40139
:104E200060E070E040E050E021E00FE8CC24DD24B9
:104E300076010E946622C40160E070E040E050E02C
:104E400021E000E90E9466228091DA079091DB0759
:104E5000A091DC07B091DD078854944FAF4FBF4F4E
:104E6000F40186839783A087B187B2C0442019F0EC
:104E70000E946A3802C00E948B3AEC01009759F4F4
:104E8000C40160E070E040E050E021E001E0CC24AB
:104E9000DD2476019BC0898590E08370907082301C
:104EA000910541F0833091050CF469C0039709F036
:104EB0008FC051C0C8840E94673865E00E9467A80F
:104EC000923029F1933030F4992351F0913009F068
:104ED0007FC011C0933039F1943009F079C02FC0F0
:104EE00068817981DD24EE24FF24C40140E050E094
:104EF00021E001E06BC068817981CC80DD80EE80AB
:104F0000FF80C40140E050E021E001E45FC068811F
:104F10007981CC80DD80EE80FF80C40140E050E0EC
:104F200021E002E453C068817981CC80DD80EE808D
:104F3000FF80C40140E050E021E003E447C0688105
:104F40007981CC80DD80EE80FF80C40140E050E0BC
:104F500021E004E43BC00E94673890E083709070C9
:104F60008130910581F0823091051CF4892B39F054
:104F70002FC08230910599F0039751F51CC06881CC
:104F80007981C884AFCF68817981CC80DD80EE8063
:104F9000FF80C40140E050E021E004E017C06881D8
:104FA0007981CC80DD80EE80FF80C40140E050E05C
:104FB00021E005E00BC068817981CC80DD80EE8046
:104FC000FF80C40140E050E021E006E00E9466223C
:104FD000D40111962C911197822F90E0FC0153E09F
:104FE000EE0FFF1F5A95E1F7880F991FE80FF91F81
:104FF000E80DF91DC685D78511962C911197822F42
:1050000090E0FC0133E0EE0FFF1F3A95E1F7880FC7
:10501000991FE80FF91FE80DF91D208831881196B6
:105020002C911197822F90E0FC0103E0EE0FFF1FFF
:105030000A95E1F7880F991FE80FF91FE80DF91D90
:10504000028911962C91822F90E0FC01B3E0EE0FC3
:10505000FF1FBA95E1F7880F991FE80FF91FE80DB8
:10506000F91DC488D588E688F788802F8C50823057
:1050700008F05BC0442049F18091DA079091DB078A
:10508000A091DC07B091DD078093710990937209BC
:10509000A0937309B093740980917109909172097A
:1050A000A0917309B09174090097A105B105A9F504
:1050B00081E090E0A0E0B0E08093710990937209E4
:1050C000A0937309B093740928C08091DA07909176
:1050D000DB07A091DC07B091DD0780936D09909309
:1050E0006E09A0936F09B093700980916D0990913A
:1050F0006E09A0916F09B09170090097A105B105E3
:1051000061F481E090E0A0E0B0E080936D099093BD
:105110006E09A0936F09B0937009CE010E94508D63
:10512000582E6624772410E040C0809168038130B7
:1051300009F443C080916803823041F4209709F458
:105140008FC6CE010E94B8383C018CC6CE010E94A9
:10515000B8383C01009731F01C2DFC015184F3E07C
:105160005F2221C0802F90E0807C90708038910574
:1051700039F0803C910561F08034910561F404C000
:1051800010E0E3E05E2E0FC010E0552453940BC0F6
:1051900010E0552408C0D5011C9201E010E0552410
:1051A0005394C0E0D0E041101078552001F582E022
:1051B0000E94896C8823C9F006C073E0572E6624CC
:1051C000772410E014C0F40182859385A485B58509
:1051D0000097A105B10511F0552409C08091650320
:1051E000909166036C0100EC69C155245394D4017D
:1051F00011963C91832F90E0FC0163E0EE0FFF1FBE
:105200006A95E1F7880F991FE80FF91FE80DF91D5E
:1052100023892150832F90E0FC0143E0EE0FFF1F14
:105220004A95E1F7880F991FE80FF91FE80DF91D5E
:10523000238B222309F035C180916D0990916E096D
:10524000A0916F09B09170090097A105B105C1F057
:1052500060916D0970916E0980916F09909170094C
:10526000685D7F4F8F4F9F4F0E942F19882341F019
:1052700010926D0910926E0910926F0910927009C8
:105280008091710990917209A0917309B09174098C
:105290000097A105B105C1F0609171097091720983
:1052A0008091730990917409685D7F4F8F4F9F4F74
:1052B0000E942F19882341F01092710910927209EF
:1052C0001092730910927409F401628173818481D0
:1052D0009581611571058105910559F00E942F197D
:1052E000882339F0D40112961D921D921D921C92B2
:1052F0001597F40166817781808591856115710527
:105300008105910559F00E942F19882339F0D401A5
:1053100016961D921D921D921C921997F40162859A
:10532000738584859585611571058105910559F011
:105330000E942F19882339F0D4011A961D921D92CC
:105340001D921C921D97442039F580916C0980FDB7
:1053500088C080916D0990916E09A0916F09B091FC
:1053600070090097A105B10509F07BC080916C0917
:10537000816080936C098091DA079091DB07A0919E
:10538000DC07B091DD0780936D0990936E09A093BF
:105390006F09B093700926C080916C0981FD61C0CE
:1053A0008091710990917209A0917309B09174096B
:1053B0000097A105B10509F054C080916C09826085
:1053C00080936C098091DA079091DB07A091DC074C
:1053D000B091DD078093710990937209A0937309CE
:1053E000B0937409F40121814091680950916909D1
:1053F000822F90E0FC01B3E0EE0FFF1FBA95E1F7BA
:10540000880F991FE80FF91FE80DF91D5787468788
:10541000D40111962C91119730916A09822F90E056
:10542000FC0173E0EE0FFF1F7A95E1F7880F991FDB
:10543000E80FF91FE80DF91D328B11962C91309170
:105440006B09822F90E0FC0153E0EE0FFF1F5A958D
:10545000E1F7880F991FE80FF91FE80DF91D338B4D
:1054600020C0F4012181822F90E0FC0123E0EE0FA7
:10547000FF1F2A95E1F7880F991FE80FF91FE80D24
:10548000F91D128AD40111968C9111978F5F119694
:105490008C93119711968C911197803110F0119681
:1054A0001C92B2E0B51528F0E1E05E1608F097C155
:1054B00005C0F3E05F1609F0D7C4B3C2809167035B
:1054C00084608093670384E0D50152968C935A2CB4
:1054D0004B2C80E1D5011D928A95E9F791E0F50109
:1054E000918B83E8818F908F013C09F48FC0023C3F
:1054F00078F40330D1F0043020F4013009F047C1D2
:1055000018C0043009F445C0003C09F040C155C042
:10551000033C09F4C9C0033C08F49FC0043C09F4EF
:10552000E8C0053C09F033C110C1D30118961C91A5
:105530001F67812F90E08F779070009731F08F3741
:10554000910511F4117801C01F5FF30124813581A9
:1055500040E050E04760852D942D68E004E10E9412
:10556000DB21682FD50150968C931058212F30E005
:105570003160442737FD4095542F852D942D0BE045
:105580000E94DB21482FF501808BCE01652D742D03
:105590000EC0960140E050E04760C50168E004E1BC
:1055A0000E94DB21482FF501808BCE01B5010E94BE
:1055B0000822D50150968C93EAC08091DA07909129
:1055C000DB07A091DC07B091DD078051954FAF4F0D
:1055D000BF4FF40182879387A487B587960140E087
:1055E00050E0C50168E000E10E94DB21682FC501A1
:1055F00024E332E140E050E000E20E94DB21682F2A
:10560000C5012DE330E040E050E047C09E0140E09E
:1056100050E0A90133272227C101A0E0B0E0282BE8
:10562000392B4A2B5B2BC50168E000E20E94DB218D
:10563000682F2C2D30E040E050E0C50106E00E94CC
:10564000DB21682FC5012AE330E040E050E00E94F2
:10565000DB21482F80E090E044C09E0140E050E014
:10566000A90133272227C101A0E0B0E0282B392B64
:105670004A2B5B2BC50168E000E20E94DB21682F0A
:10568000960140E050E0C5010EE00E94DB21682F4A
:10569000C5012BE330E040E050E006E00E94DB2152
:1056A000482F80E090E082CF9E0140E050E0A901C9
:1056B00033272227C101A0E0B0E0282B392B4A2B49
:1056C0005B2BC50168E000E20E94DB21682FC50169
:1056D0002CE330E040E050E006E00E94DB21482F60
:1056E000C601B5010E940822F501808B8FEF818FE2
:1056F0004EC0222D30E040E050E02F7730704070F7
:10570000507072E0220F331F441F551F7A95D1F756
:10571000386080E090E0A0E0B0E0CC2021F081E0B3
:1057200090E0A0E0B0E0282B392B4A2B5B2B852D95
:10573000942D68E00CE00E94DB21482FD5015096A3
:105740008C93CE01652D742D1EC0910140E050E078
:105750006AE0220F331F441F551F6A95D1F7546E1C
:105760008C2D90E0A0E0B0E0282B392B4A2B5B2B4E
:10577000C50168E000E20E94DB21482FD501509668
:105780008C93CE01B5010E940822F501808BD501D2
:1057900050962C91222309F467C3422F41503FE7D2
:1057A00067E051E017C0832F330F87FD3627842F22
:1057B000869586958695F501E80FF11D808190E02C
:1057C000242F277002C0959587952A95E2F780FDD2
:1057D000352741504F3F39F7F501308345C380915C
:1057E0006703816080936703D4011A961D921D920E
:1057F0001D921C921D97802F8C508230B0F482E055
:10580000F501828BFE0133E0F695E7953A95E1F7D5
:10581000F070319621E0E030F20711F4E0E0F0E0C2
:10582000EA5AFD4F949184E00FC081E0F501828B2C
:10583000CF3FD10521F018F0E0E0F0E001C0FE011B
:10584000EA5AFD4F949182E0D50151968C93892FAD
:105850008295869586958370F5018283990F990FBD
:10586000918382E1808B6114710409F44AC0043091
:1058700041F0013431F0023421F0033411F00434EA
:1058800091F4C60181709070892B39F0D501119681
:105890008C911197836011968C93F30110854420AD
:1058A00051F0107808C0D30114968C9180FF03C08A
:1058B0009360F5019183812F90E08F779070892B11
:1058C00001F1D30119968C910E94253E0F97CCF0DF
:1058D0001F5FF30181850E943B38892B51F410FF33
:1058E00008C0D50111968C91119791E089271196E6
:1058F0008C93812F90E08F7190709595879510789B
:10590000182B0E3070F40C30F8F4043030F4023000
:1059100070F5013009F0A8C225C0043009F0A4C216
:1059200021C00234D1F1033430F40034D9F0013411
:1059300009F09AC229C0043409F44BC00434C8F1F8
:10594000053409F091C255C0C770D070C25CDD4FFC
:10595000FE012491D5012C930C3009F085C22C7FD7
:105960002C9382C2852D612F0E946A213FC0D301F2
:1059700018966C9160786F60852D0E946A21F50100
:10598000808384E0818B70C2F694E794D794C794A7
:105990004C2D4170812F61E017C0B2E0F694E7947E
:1059A000D794C794BA95D1F74C2D4170812F62E0FE
:1059B0001BC0A3E0F694E794D794C794AA95D1F7B7
:1059C0004C2D4170812F63E00E942E21D5018C93D4
:1059D0004BC2F4E0F694E794D794C794FA95D1F7C4
:1059E0004C2D4170812F64E00E942E21F5018083AF
:1059F0003BC2D50111968C911197836011968C93BF
:105A0000119782E052968C935297F694E794D7942C
:105A1000C794F601EF70F070EA5BFD4FE491EC93F0
:105A200023C280916703826080936703F40112862A
:105A3000138614861586D50152965C92529781E0A2
:105A400051968C93519788E150968C93063818F5AF
:105A5000033808F049C1063009F4D0C0073078F4A3
:105A60000330F1F1043020F4013009F0E1C139C014
:105A7000043009F495C0053009F0DAC1ADC0023830
:105A800008F02AC1003808F013C1802F8C508230F2
:105A900008F0CEC119C0013950F40F3808F09DC18B
:105AA0000E3808F094C1083808F05AC141C10239D3
:105AB00009F4AFC0023908F4ABC1033909F4B6C028
:105AC000043909F0B5C1C8C040E00D3009F441E027
:105AD00095012F5F3F4FCE0160E00E94B221A8C127
:105AE0001F67F30181858C70883099F48FE3D501AD
:105AF00012968C93812F90E08F779070009731F001
:105B00008F37910511F4117801C01F5FF5011183E2
:105B1000B8C017FF04C080E6F501818304C080E4AB
:105B2000D50111968C93F30181850E94253E212F8A
:105B300030E00F97E4F0C9018F779070009731F053
:105B40008F37910511F412E001C01D5F912F9695DA
:105B50009F70D50111968C911197982B11969C935B
:105B6000119710FF46C0906111969C9342C0C901E5
:105B70008F779070009731F08F37910511F411E015
:105B800001C01F5F212F2F70F5018181282B2183F8
:105B9000D30114968C9180FF2CC02061218329C0F1
:105BA000D701C601B695A795979587958F708068A0
:105BB000D50111968C93C60181709070892BC9F024
:105BC000F30181850E94253E0F979CF0D501119627
:105BD0008C91119780610BC065E0F694E794D7949F
:105BE000C7946A95D1F78C2D8F70806BD501119673
:105BF0008C93B5016E5F7F4FCE016BC059E0F69478
:105C0000E794D794C7945A95D1F78C2D8F70806AFA
:105C1000EDCF4DE0F694E794D794C7944A95D1F729
:105C2000D5011196CC9211978EED0CC035E1F6940A
:105C3000E794D794C7943A95D1F7D5011196CC92B1
:105C400011978FED12968C93B5016D5F7F4FCE014A
:105C50000E94A321885EEAC0822D8F77D50111961C
:105C60008C931197C114D104E104F10419F08068F8
:105C700011968C93B0E82B16310470F48DEDF5017C
:105C80008283B5016D5F7F4FCE010E94A321885EA4
:105C9000D50150968C93CCC0F50181818283220C72
:105CA000232C221C33083194218280EC838387C00B
:105CB000F501118295012E5F3F4F013841F4CE016D
:105CC000816060E040E00E94B221805FE1CFCE01C0
:105CD000B9010E94A321A9C08FEFD50112968C9320
:105CE000129711961C92A4C0053811F488E708C0D9
:105CF000043829F484E7D50113968C9303C08CE70C
:105D0000F50183834E01992D9370D50113968C91E3
:105D10001397892B13968C9313971296CC93129703
:105D20001196CC92119780E250968C93509714C0A4
:105D300080E7F5018283063811F488E782839E01AB
:105D40002770D50112969C911297922B12969C93D4
:105D500012971196CC9211978AE051968C9368C055
:105D6000802F8B58833030F4832D8370846EF5013F
:105D7000838306C0832D83708C6ED50113968C931C
:105D8000F5012282C182093811F00C3851F49501D5
:105D90002C5F3F4FCE01816060E040E00E94B22165
:105DA00014C00A3811F00D3851F495012C5F3F4FA3
:105DB000CE0161E040E00E94B221805E37C0B501B3
:105DC0006C5F7F4FCE010E94A321805E61CF8FEB7D
:105DD000F50182838FE081832BC00E94906C8FEF4E
:105DE000D50115968C93159714968C9314978EE382
:105DF00013968C93139712967C93129711966C932B
:105E00001197003919F48FE714968C9380E30EC034
:105E10008C2D8F71D50111968C9395012E5F3F4F7C
:105E2000CE0161E040E00E94B221805FF501808BED
:105E3000D50150969C919695969596959150E92FFF
:105E4000FF27E7FDF095EA0DFB1D20E004C08081EF
:105E50002827915031971916D4F3F501208304C0F7
:105E60006624772410E0A3C9DF91CF911F910F9191
:105E7000FF90EF90DF90CF90BF90AF909F908F906A
:105E80007F906F905F904F903F902F9008951F925A
:105E90000F920FB60F920BB60F9211240F931F9310
:105EA0002F933F934F935F936F937F938F939F9322
:105EB000AF93BF93EF93FF93809164038823B1F076
:105EC0008091670380FD07C08BE390E0909387008B
:105ED0008093860004C0109287001092860087E7A6
:105EE00090E0909381008093800075C087E493E0F8
:105EF0000E94BC24AC012091880030918900059754
:105F00002817390728F4509381004093800017C068
:105F10008091880090918900C2969093810080932F
:105F20008000009188001091890087E493E00E942E
:105F30005026080F191F1093810000938000809154
:105F40005A03882309F03FC080915C038823D9F568
:105F500080915F038823B9F580915803882399F4D1
:105F600081E08093640380917C00846080937C0056
:105F70001FB7789487E493E06AEB78E00E948F265D
:105F80001FBF10926403809158038150809358037F
:105F90008091570380935A0390915903933021F4D1
:105FA00080E180935B0309C0943029F481E0809301
:105FB0005F0390935A0310925B0310925C0310925C
:105FC00063031092620387E493E00E940924909394
:105FD000870080938600FF91EF91BF91AF919F91D1
:105FE0008F917F916F915F914F913F912F911F9171
:105FF0000F910F900BBE0F900FBE0F901F90189532
:106000001F920F920FB60F920BB60F9211240F939F
:106010001F932F933F934F935F936F937F938F9330
:106020009F93AF93BF93EF93FF938091680388236F
:1060300031F08091670385FF02C010923A0380918E
:1060400046038823A1F08091670380FD05C08BE3A0
:1060500090E099BD88BD02C019BC18BC8BE390E0EC
:106060009BBD8ABD87E790E097BD86BD70C089E281
:1060700093E00E94BC24AC012CB53DB505972817D0
:10608000390718F457BD46BD0FC08CB59DB5C296F3
:1060900097BD86BD0CB51DB589E293E00E945026E0
:1060A000080F191F17BD06BD80913C03882309F016
:1060B00044C080913E03882309F03FC08091410392
:1060C0008823D9F580913A03882389F481E080936D
:1060D000460386B7846086BF1FB7789489E293E051
:1060E0006CE078E00E948F261FBF109246038091DB
:1060F0003A03815080933A038091390380933C03A3
:1061000090913B03933051F480916803882311F000
:1061100084E101C080E180933D0309C0943029F4FB
:1061200081E08093410390933C0310923D031092D1
:106130003E03109245031092440389E293E00E94CB
:1061400009249BBD8ABD8AB59BB599BD88BDFF91C9
:10615000EF91BF91AF919F918F917F916F915F91DF
:106160004F913F912F911F910F910F900BBE0F9068
:106170000FBE0F901F9018950E946A12833020F076
:10618000853020F0873011F081E008958091670319
:10619000887008950E947C6CFC01808182FF0DC094
:1061A00096B3809163009095991F9927991F8695C2
:1061B000869586958095817009C086B3909163001D
:1061C000969596959695909591708078982B892FB5
:1061D00008950E947C6CFC01808182FF02C0C79AF6
:1061E0000895C79808959C0180916C09833011F03F
:1061F00080E008953093690920936809662311F0BF
:106200008DE001C08CE080936A0983E080936B0984
:1062100010926C090E947C6CFC01808186FF05C095
:1062200080916C09816080936C09808187FD02C038
:1062300081E0089580916C09826080936C0981E00F
:1062400008952F923F924F925F926F927F928F921A
:106250009F92AF92BF92CF92DF92EF92FF920F93F5
:106260001F93CF93DF93EC012B013A01222E302EA6
:1062700046015701009731F48AEB98E00E942131E2
:10628000CCE0D8E080916803882321F088E0CA3B05
:10629000D80701F10E946A128230E0F0853010F0D8
:1062A0008730C1F41FB7F894CE01B201A301222DAB
:1062B000032D750164010E9466221FBF882329F403
:1062C00085E090E00E949219E5CF80916703877F77
:1062D00080936703DF91CF911F910F91FF90EF9013
:1062E000DF90CF90BF90AF909F908F907F906F90F6
:1062F0005F904F903F902F900895CF92DF92EF9252
:10630000FF920F93982F809168038823E9F59923D2
:10631000D9F110920D0880910D0880930C088EE140
:10632000E9E2F3E0DF011D928A95E9F70E946A1223
:10633000873031F48091670381608093670311C0D7
:1063400080E593E20E9445388CE098E060E070E0E0
:1063500040E050E02AE002E8CC24DD2476010E94EF
:1063600021318BE390E099BD88BD88B599B59BBD7F
:106370008ABD87E790E097BD86BD1DBC1CBC87B772
:10638000846087BFBE9A05C0BE98C69887B78B7FCA
:1063900087BF0F91FF90EF90DF90CF900895CF923D
:1063A000DF92EF92FF920F93982F809168038823DA
:1063B00099F5992389F11092BB088091BB088093CD
:1063C000BA088EE1E7E4F3E0DF011D928A95E9F770
:1063D0008AEB98E060E070E040E050E022E002E804
:1063E000CC24DD2476010E9421318BE390E0909350
:1063F00087008093860087E790E0909381008093E8
:106400008000109289001092880080917D00846045
:1064100080937D00139A07C013981B9880917D008C
:106420008B7F80937D000F91FF90EF90DF90CF9056
:1064300008951F93182F8823E1F180E00E947D3199
:1064400080E00E94CF3181E064E00E9471918091F0
:1064500062008B7F809362008EE1E9E2F3E0DF016E
:106460001D928A95E9F782E08093670383E0809329
:106470003B038FEF809329038BE390E099BD88BDA8
:1064800088B599B59BBD8ABD87E790E097BD86BD6D
:1064900010920D0880910D0880930C0810936803EA
:1064A000BD9A87B7846087BF82E090E00E94F519AB
:1064B00007C087B78B7F87BF10926803BD98C598C8
:1064C0001F91089581E00E941932809167038061D5
:1064D00080936703089580E00E941932E2E6F0E0BD
:1064E00080818B7F808380E00E947D3180E00E94EC
:1064F000CF3181E064E00E9471910895CF92DF92E4
:10650000EF92FF920F93009711F485EA90E0909339
:106510006603809365036C01EE24FF248CE098E011
:1065200060E070E040E050E024E000EC0E942131A7
:106530000F91FF90EF90DF90CF90089582E00E943E
:106540001932809167038F7E809367038091DA0709
:106550009091DB07A091DC07B091DD0790E00E94ED
:106560007E320895CF92DF92EF92FF920F931F93A6
:106570008B019C016A01A90166277727EE24FF247D
:106580008CE098E0BA01A80122E003EC0E942131DE
:1065900081E01F910F91FF90EF90DF90CF900895D1
:1065A000CF92DF92EF92FF920F931F938B019C018A
:1065B0006A01A90166277727EE24FF248CE098E082
:1065C000BA01A80122E002EC0E94213181E01F9172
:1065D0000F91FF90EF90DF90CF900895CF92DF92D0
:1065E000EF92FF920F931F938B019C01C42EAC017D
:1065F00066277727DD24EE24FF248CE098E0BA019B
:10660000A80122E001EC0E94213181E01F910F914D
:10661000FF90EF90DF90CF900895CF92DF92EF92AE
:10662000FF920F93FC01613091F0613018F06230FD
:1066300049F51AC0002309F400E4C22EDD24EE243B
:10664000FF2480E090E0BF01202F0BE819C0002359
:1066500009F400E1C22EDD24EE24FF2480E090E066
:10666000BF01202F0CE80CC0002309F400E1C22E6A
:10667000DD24EE24FF2480E090E0BF01202F0DE810
:106680000E94213181E00F91FF90EF90DF90CF9039
:106690000895CF92DF92EF92FF920F93FC01613049
:1066A000A1F0613028F06230E9F06A3099F527C036
:1066B000002309F400E4C22EDD24EE24FF2480E050
:1066C00090E0BF01202F08E823C0002309F400E177
:1066D000C22EDD24EE24FF2480E090E0BF01202FB5
:1066E00009E816C0002309F400E1C22EDD24EE24DF
:1066F000FF2480E090E0BF01202F0AE809C0C22EED
:10670000DD24EE24FF2480E090E0BF01202F05EC83
:106710000E94213181E00F91FF90EF90DF90CF90A8
:106720000895CF92DF92EF92FF920F939C01809198
:106730006803813011F080E00EC0C62EDD24EE2407
:10674000FF248CE098E0B90140E050E021E004E84B
:106750000E94213181E00F91FF90EF90DF90CF9068
:106760000895CF92DF92EF92FF920F939C01809158
:106770006803813011F080E00EC0C62EDD24EE24C7
:10678000FF248CE098E0B90140E050E021E003E80C
:106790000E94213181E00F91FF90EF90DF90CF9028
:1067A0000895CF92DF92EF92FF920F939C01809118
:1067B0006803813011F080E00EC0C62EDD24EE2487
:1067C000FF248CE098E0B90140E050E021E007E8C8
:1067D0000E94213181E00F91FF90EF90DF90CF90E8
:1067E0000895CF92DF92EF92FF920F939C018091D8
:1067F0006803813011F080E00EC0C62EDD24EE2447
:10680000FF248CE098E0B90140E050E021E006E888
:106810000E94213181E00F91FF90EF90DF90CF90A7
:106820000895CF92DF92EF92FF920F939C01809197
:106830006803813011F080E015C06770862F806E8C
:10684000442311F0862F886EC82EDD24EE24FF2409
:106850008CE098E0B90140E050E021E005E80E94BA
:10686000213181E00F91FF90EF90DF90CF9008955C
:10687000CF92DF92EF92FF920F939C018091680379
:10688000813011F080E015C06770862F806F44233F
:1068900011F0862F886FC82EDD24EE24FF248CE0B3
:1068A00098E0B90140E050E021E005E80E94213184
:1068B00081E00F91FF90EF90DF90CF900895CF92FD
:1068C000DF92EF92FF920F93282F80E090E060E03C
:1068D00070E040E050E002E8CC24DD2476010E9424
:1068E000213181E00F91FF90EF90DF90CF900895DC
:1068F000CF92DF92EF92FF920F93FC01242F662339
:1069000011F400E801C001E880E090E0BF0140E040
:1069100050E0CC24DD2476010E94213181E00F91EA
:10692000FF90EF90DF90CF900895CF92DF92EF929B
:10693000FF920F939C01C62EDD24EE24FF2480E0FD
:1069400090E0B90140E050E021E001E90E942131EE
:1069500081E00F91FF90EF90DF90CF9008952F92FC
:106960003F924F925F926F927F928F929F92AF92DF
:10697000BF92CF92DF92EF92FF920F931F93DF931C
:10698000CF93CDB7DEB72A970FB6F894DEBF0FBE10
:10699000CDBF1C012A013B0148015901009709F4B0
:1069A00093C1DC0119968C9190E0837090708130D6
:1069B000910571F08230910524F4892B09F41CC1F2
:1069C00083C18230910591F1039709F07DC198C090
:1069D00084269526A626B726C40181709070892B3F
:1069E00069F0F1016081718180E090E040E050E069
:1069F00024E004E0730162010E9421318EE190E005
:106A0000A0E0B0E088229922AA22BB22811491043E
:106A1000A104B10409F458C1D1016D917C9180E0C9
:106A200090E040E050E024E005E4E1C0D901C80175
:106A300084279527A627B7278D839E83AF83B887A2
:106A40008D819E8181709070892B69F0D1016D914B
:106A50007C9180E090E040E050E024E004E07301AD
:106A600062010E942131BD81B1FF0DC0F101608141
:106A7000718180E090E040E050E024E001E47301A7
:106A800062010E942131FD81F2FF0DC0D1016D91A3
:106A90007C9180E090E040E050E024E002E473016B
:106AA00062010E94213188E090E0A0E0B0E08822FD
:106AB0009922AA22BB22D301C20184709070A070D7
:106AC000B07088169906AA06BB0669F0D1016D91CF
:106AD0007C9180E090E040E050E024E003E473012A
:106AE00062010E942131BD81B4FFEEC0F1016081DD
:106AF000718180E090E040E050E024E004E477C061
:106B000084269526A626B726D501C4018F719070DC
:106B1000A070B0700097A105B10569F0D1016D9129
:106B20007C9180E090E040E050E024E004E07301DC
:106B300062010E942131D501C401807E9170A07054
:106B4000B0700097A105B10569F0F1016081718114
:106B500080E090E040E050E024E005E07301620155
:106B60000E942131D501C40180709E71A070B07067
:106B70000097A105B10569F0D1016D917C9180E08C
:106B800090E040E050E024E006E0730162010E94E2
:106B90002131D501C4018070907EAF71B070009733
:106BA000A105B10569F0F1016081718180E090E09B
:106BB00040E050E024E002E9730162010E942131CB
:106BC00080E090E0A0EEBFE188229922AA22BB22B9
:106BD00081149104A104B10409F476C0D1016D912E
:106BE0007C9180E090E040E050E024E003E9730114
:106BF00062010E94213168C0D901C801842795270C
:106C0000A627B72789839A83AB83BC83892BA9F0F6
:106C1000D1016D917C911FEFC12E1FEFD12EE12C80
:106C2000F12CC420D520E620F72080E090E040E061
:106C300050E023E004E00E94213189819A81AB81F8
:106C4000BC81807090700097A105B105E9F1812C9D
:106C5000912CB1E0AB2EB12CE0E1F0E0FA87E987AE
:106C600089819A81AB81BC8188219921AA21BB218C
:106C70000097A105B105E9F0D1016D917C91CC247B
:106C8000DD247601D501C40184219521A621B721F7
:106C90000097A105B10529F0A1E0CA2ED12CE12C65
:106CA000F12C80E090E049855A8523E004EC0E94B5
:106CB0002131880C991CAA1CBB1CE985FA85EF318F
:106CC000F10511F03196CACF81E02A960FB6F894FB
:106CD000DEBF0FBECDBFCF91DF911F910F91FF900F
:106CE000EF90DF90CF90BF90AF909F908F907F906C
:106CF0006F905F904F903F902F900895CF92DF92CA
:106D0000EF92FF920F937C010E94B838FC0100972C
:106D100039F18185282F30E0237030702130310522
:106D2000FCF02330310584F023303105C9F40E9492
:106D3000253E0E97A9F480E090E060E070E040E02E
:106D400050E021E002E807C080E090E0B70140E0B9
:106D500050E027E002E0CC24DD2476010E942131BE
:106D600081E00F91FF90EF90DF90CF900895CF9248
:106D7000DF92EF92FF920F93CF93DF93EC010E948B
:106D8000B838FC01009761F1818583708150C0841F
:106D9000823090F4DD24EE24FF2480E890E0A0E02F
:106DA000B0E0C822D922EA22FB2280E090E0BE01B6
:106DB00040E050E02BE011C0DD24EE24FF2480E809
:106DC00090E0A0E0B0E0C822D922EA22FB2280E0D5
:106DD00090E0BE0140E050E024E003E00E94213159
:106DE00081E0DF91CF910F91FF90EF90DF90CF90F6
:106DF0000895CF92DF92EF92FF920F93CF93DF939C
:106E0000EC01C62E0E94B838892B61F0DD24EE24F7
:106E1000FF248CE098E0BE0140E050E026E000E472
:106E20000E94213181E0DF91CF910F91FF90EF908F
:106E3000DF90CF900895CF92DF92EF92FF920F9361
:106E40001F93CF93DF938C01C62E0E94B838EC01BC
:106E50000097C1F1898590E083709070833091052F
:106E600034F48130910534F4892B79F02BC00397E9
:106E700049F50BC0DD24EE24FF248CE098E0B80136
:106E800040E050E024E001E01BC0DD24EE24FF24BC
:106E90008CE098E0B80140E050E022E001E00E9480
:106EA000213189858F70833069F480E090E060E063
:106EB00070E040E050E021E002E8CC24DD247601DF
:106EC0000E94213181E0DF91CF911F910F91FF90BE
:106ED000EF90DF90CF90089583E080936C0910923B
:106EE00071091092720910927309109274098091BD
:106EF000710990917209A0917309B09174098093FE
:106F00006D0990936E09A0936F09B09370098091F9
:106F1000DA079091DB07A091DC07B091DD0788517B
:106F20009C4FAF4FBF4F80930E0890930F08A093D4
:106F30001008B09311088093BC089093BD08A093EB
:106F4000BE08B093BF088091DA079091DB07A0914B
:106F5000DC07B091DD078854944FAF4FBF4F80934B
:106F6000120890931308A0931408B0931508809307
:106F7000C0089093C108A093C208B093C3081092B0
:106F800016081092170810921808109219081092FB
:106F9000C4081092C5081092C6081092C70885EA66
:106FA00090E0909366038093650380E00E9419321D
:106FB0000E94836C809369031092670381E00E94B2
:106FC0007D3181E00E94CF31E2E6F0E08081846093
:106FD00080830895CF92DF92EF92FF920F937C010E
:106FE000062F0E94E03883708150823060F48CE07C
:106FF00098E0B70140E050E0202F02E0CC24DD24EF
:1070000076010E94213181E00F91FF90EF90DF9097
:10701000CF900895CF92DF92EF92FF920F931F933C
:10702000CF93DF93EC018B01C42E0E94E038837074
:10703000833011F080E00CC0DD24EE24FF2480E0DA
:1070400090E0BE01A80124E004E90E94213181E022
:10705000DF91CF911F910F91FF90EF90DF90CF9034
:10706000089520E030E08F708950823010F421E0E4
:1070700030E0C901089520E030E08F708550823003
:1070800010F421E030E0C9010895EF92FF920F93D0
:107090001F93CF93DF937C0105E719E0C0E0D0E0B8
:1070A0000BC02196E114F10429F0C801F7010995FC
:1070B000882329F0055F1F4FC034D10591F7CE0119
:1070C000DF91CF911F910F91FF90EF9008958091E4
:1070D000830308959091350C992319F420E030E052
:1070E00011C0809182038F5F80938203891710F013
:1070F00010928203909182038BE0989F900111245B
:107100002B58364FC9010895CF92DF92EF920F931B
:107110001F93CF93DF93EC01162F6901442361F095
:107120000E94836C8823E1F0CE01612FA601202FFD
:107130000E2D0E940D3305C0A901202F0E2D0E9497
:107140004933EE2069F484E00E945F3460E011115D
:1071500061E0CE0141E00E9478348AE00E945F3411
:10716000DF91CF911F910F91EF90DF90CF90089515
:10717000CF93DF93EC010E946A12873019F424E860
:1071800033E01AC02097B1F03091350CE5E7F9E013
:1071900020E00EC0808191813B968C179D0739F4C9
:1071A0008BE0289F900111242B58364F05C02F5F8C
:1071B000231780F320E030E0C901DF91CF910895DB
:1071C0000E94B838FC01009711F480E00895818591
:1071D0008F7008958F929F92AF92BF92CF92DF925D
:1071E000EF92FF920F931F93DF93CF9300D000D0C5
:1071F00000D0CDB7DEB74C01062F0E946A1287304F
:1072000009F447C0C4010E94B8385C01009709F432
:1072100040C07E010894E11CF11CC701B4010E942A
:10722000E16FF50124813581468157810023B9F052
:10723000C701BA01A9010E94ED6F8FEF6DE0A701B0
:107240000E94BE70F50124813581468157819A01E3
:1072500044275527C401B9010E94EE3E1AC0C70158
:10726000F501608500E00E9406708FEF6AE0A701DB
:107270000E94BE70F501C480D580E680F78087014A
:10728000222733270170C4016085A601202F0E94A8
:10729000163F26960FB6F894DEBF0FBECDBFCF9136
:1072A000DF911F910F91FF90EF90DF90CF90BF90F3
:1072B000AF909F908F9008951F93CF93DF93C5E772
:1072C000D9E010E01BC08A85989FC0011124803549
:1072D000910534F0888590E08F779070892B61F06C
:1072E000888580788887888199810E94B7368881CF
:1072F000998160E00E94EA381F5F2B969091350CCF
:10730000191708F3DF91CF911F9108958F929F92E3
:10731000AF92BF92CF92DF92EF92FF920F931F93A3
:10732000DF93CF930F92CDB7DEB74C017A018B017B
:10733000922F81149104E1F1F401A480B580C680FC
:10734000D780A416B506C606D70691F1243061F49D
:1073500029830E946A129981873031F5F401E48211
:10736000F5820683178324C0F4011286992329F03D
:10737000818580628187913031F0F401818580645C
:107380008187943021F0F401818580618187F40147
:10739000E482F58206831783C401B801A701960130
:1073A00085010E94AF3404C0F401818584FFDCCFE5
:1073B0000F90CF91DF911F910F91FF90EF90DF9091
:1073C000CF90BF90AF909F908F900895EF92FF92D3
:1073D0000F931F93CF93DF93EC01162F042F009789
:1073E00009F492C0443051F40E946A12873009F0C7
:1073F00087C0188789C08F7E898786C089850E944B
:10740000253E482F5985812F90E08F779070242F4B
:1074100030E02817390714F41078142B68856117A9
:1074200009F472C01A86002329F089858062898751
:10743000013029F0898580648987043019F08985B5
:1074400080618987E62EFF24812F862787FF34C03D
:1074500097012F7730702115310509F01078852FAD
:107460008370833011F08823D1F4232B29F0888195
:1074700099810E94B73610C089858C70883061F47C
:10748000812F90E08F779070892B31F4612F6160AC
:10749000888199810E941B37888199810BC08881DE
:1074A0009981232B39F00E941B37888199810E9492
:1074B000B73602C00E947E361887212F30E0C901FE
:1074C0008F779070892BB1F089858F7085508230CD
:1074D00088F410FD03C0612F6F5F08C00894E108B5
:1074E000F1082E153F0531F4612F61508881998193
:1074F0000E94F93688819981612F0E941B3704C050
:10750000898584FF7BCF77CFDF91CF911F910F913A
:10751000FF90EF9008950F931F93CF93DF930E94F6
:107520006A12873041F4809183038F5F80938303D5
:10753000C4E8D3E01DC09091350C992319F4C0E044
:10754000D0E04EC0809181038F5F809381038917C3
:1075500038F0809183038F5F8093830310928103BF
:10756000909181038BE0989FE0011124CB58D64F76
:107570008091830390E087709070892BA1F46885D7
:10758000262F30E0C9018F779070892B61F08985B3
:107590008F708550823038F460FD05C06F5F888140
:1075A00099810E94F936809183038770843099F421
:1075B00089858370813079F44C815D816E817F8112
:1075C0000EE110E020E030E00427152726273727BA
:1075D000CE010E94AF348A858F3F11F08F5F8A877A
:1075E000CE01DF91CF911F910F91089580EC92E031
:1075F000E5E7F9E0DF019C011D9221503040E1F701
:1076000010928203109281031092350C08959F927C
:10761000AF92BF92CF92DF92EF92FF920F931F93A0
:10762000DF93CF9300D00F92CDB7DEB76C01962ECB
:10763000009719F400E010E028C020E2E22EF12CBF
:1076400000E010E05E010894A11CB11CA895C501E2
:10765000B70143E050E00E94E9AC69817A81CB0137
:1076600001978F5F9F4340F4892D4B8120E030E0EC
:10767000F60109950F5F1F4F84E090E0E80EF91EB8
:107680009CEDE9169FE0F90609F7C8010F900F90ED
:107690000F90CF91DF911F910F91FF90EF90DF90AE
:1076A000CF90BF90AF909F900895AF92BF92CF922E
:1076B000DF92EF92FF920F931F93DF93CF93CDB79B
:1076C000DEB727970FB6F894DEBF0FBECDBF8FEFA2
:1076D0009FEFAFEFBFEF8C839D83AE83BF8300E24C
:1076E00010E05E010894A11CB11C34E0C32ED12C23
:1076F000CC0EDD1EF02EE12EC501B80143E050E0B6
:107700000E94E9AC89819A818F5F9F4F19F48B8128
:107710008F3F39F0C6016F2D7E2D44E050E00E946E
:1077200001AD0E9471120C5F1F4F8FE00C3D1807D6
:1077300009F727960FB6F894DEBF0FBECDBFCF91E5
:10774000DF911F910F91FF90EF90DF90CF90BF904E
:10775000AF900895CF92DF92EF92FF920F931F9315
:10776000DF93CF9300D00F92CDB7DEB78C01009797
:1077700009F441C0FC018081918101978F5F9F4393
:1077800010F540E2E42EF12C6E010894C11CD11CCE
:10779000A895C601B70143E050E00E94E9AC2981F9
:1077A0003A81F801808191812817390719F48B817A
:1077B0008F7020C084E090E0E80EF91E9CEDE91681
:1077C0009FE0F90629F7F80180819181F8E2803085
:1077D0009F0718F0F80111860EC08F3F910509F040
:1077E00028F488E00E94896C882311F087E001C0AA
:1077F00082E0F80181870F900F900F90CF91DF9179
:107800001F910F91FF90EF90DF90CF900895FF921E
:107810000F931F93CF93DF938C01F62E0E946A1271
:107820008730E9F480918403909185038017910754
:1078300009F455C0109385030093840384E893E012
:107840000E94AA3B80918D0390E083709070019715
:10785000029708F444C082E080938D0340C0C801C1
:1078600001978F5F9F4318F0C0E0D0E03CC0C80193
:107870000E94B838AC010097A9F52091350C20344E
:1078800050F48BE0289FE0011124CB58D64F2F5F96
:107890002093350C10C0E5E7F9E0EF0192858A8569
:1078A000891708F4EF013B968CE0E533F807B1F750
:1078B0008A858823B9F019830883CE010E94AA3BE8
:1078C00080E888871C821D821E821F821B821A828A
:1078D0001A86FF2041F0C8010E94D28704C0C4E884
:1078E000D3E001C0EA01CE01DF91CF911F910F914A
:1078F000FF900895CF92DF92EF92FF921F93CF9364
:10790000DF936B015FEFE52E5FE7F52EE822F922AA
:10791000C70160E00E94073CEC010097E1F0188588
:107920001078D7FC10588FEF9FE7C822D922C601E4
:1079300060E00E94073CFC01009769F080858F772A
:10794000182B1087DB82CA821A86F382E2821286A3
:10795000C7010E942287DF91CF911F91FF90EF9086
:10796000DF90CF90089561E00E94073C0895CF9387
:10797000DF93EC010E9404870BC0CE010E94B33C50
:10798000FC01009739F0C281D381138212821286E2
:10799000209799F7DF91CF910895CF93DF93C5E7B3
:1079A000D9E08A819B81892B21F0888199810E946D
:1079B000B73C8CE0CA32D80711F02B96F2CFDF919A
:1079C000CF910895DF92EF92FF920F931F937A0168
:1079D0008B01D22E0E94B33C009729F0B801A70179
:1079E0002D2D0E9486391F910F91FF90EF90DF900F
:1079F00008951F93CF93DF93EB01142F0E94B33CA4
:107A0000FC010097A1F0AE0160E070E0BA015527DB
:107A1000442784819581A681B781A070B070482BDE
:107A2000592B6A2B7B2BCF01212F0E948639DF91A6
:107A3000CF911F9108951F93CF93DF93EB01142FE4
:107A40000E94B33CFC01009789F0AE0160E070E059
:107A500084819581A681B78180709070482B592BC5
:107A60006A2B7B2BCF01212F0E948639DF91CF918A
:107A70001F9108950E94B33CFC01009729F420E077
:107A800030E040E050E004C02481358146815781D8
:107A9000B901CA0108950E94B33CFC01009711F49A
:107AA00080E0089580850895FF920F931F93CF93F0
:107AB000DF93EC01062FF42E0E946A12833041F00E
:107AC0000E946A12873021F084E0F81609F40078E9
:107AD000CE010E94B33CEC010097C1F01885602FE5
:107AE0004F2D0E94E6398A819B81009779F060E0F2
:107AF0000E94073CFC01009749F08085182717FD7C
:107B00000058CF01602F4F2D0E94E639DF91CF91B1
:107B10001F910F91FF9008958F929F92BF92CF92E5
:107B2000DF92EF92FF920F931F93DF93CF9300D0DA
:107B30000F92CDB7DEB76C01B62E2FE0B22251F412
:107B400082E00E94896C882329F482E00E940E6FF3
:107B50000E94E86E00E210E0EE24EA94FE2C4E0152
:107B60000894811C911CA895C401B80143E050E021
:107B70000E94E9AC89819A818C159D0511F47801E8
:107B80000FC02FEFE2162FEFF20621F48050904441
:107B900008F078010C5F1F4F8FE00C3D180719F7B4
:107BA00029813A812C153D0541F08FEFE8168FEFC2
:107BB000F80619F42FEF3FEF17C08B818B1519F4DE
:107BC0002C153D0579F0BB82DA82C982A895CE01D9
:107BD0000196B70144E050E00E9401ADC6016B2D53
:107BE0000E94E68520E030E0C9010F900F900F90D1
:107BF000CF91DF911F910F91FF90EF90DF90CF9089
:107C0000BF909F908F9008951F93CF93DF93EC01C7
:107C1000162F0E94B33CFC01009799F0412F4F7042
:107C20006185862F90E08F709070242F30E082174E
:107C3000930739F0607F642B61871286CE010E9422
:107C40008C3DDF91CF911F910895E82FF0E0EF7008
:107C5000F070E85EFB4FE4918E2F90E0089590E085
:107C600083709070009731F0039711F48CE10895C0
:107C700084E008958FE1089584E993E00895809168
:107C8000B00382FF05C080919603909197030895F9
:107C9000809194039091950308958091B00381FDA4
:107CA0000CC08260877F8093B0031092B40380E0A1
:107CB00090E060E070E00E94871E08958823E9F05C
:107CC00082E06EE671E00E94292083E066E771E0C1
:107CD0000E94292084E06EE771E00E94292085E05F
:107CE00066E871E00E94292086E06EE871E00E945B
:107CF000292087E066E971E01CC082E06EE271E055
:107D00000E94292083E06EE371E00E94292084E034
:107D10006EE471E00E94292085E066E571E00E9432
:107D2000292086E06EE571E00E94292087E066E662
:107D300071E00E942920089580919303833014F00C
:107D400010929303809193038F5F809393038150EC
:107D5000813041F0823061F0882379F481E066E37C
:107D600072E003C081E06EE272E00E942920089573
:107D700081E066E272E00E9429200895882321F0C4
:107D800082E066EB71E003C082E06EEA71E00E947F
:107D900029200895882321F081E066EA71E003C07C
:107DA00081E06EE971E00E94292008958093C40368
:107DB0000E946D1208952091B00321FD0EC02B7F0B
:107DC00021602093B0039093970380939603709360
:107DD0009F0360939E030E946D120895E0919403A7
:107DE000F09195038E179F0711F0EF2BF1F49B0193
:107DF00040E050E0A9013327222780919A03909117
:107E00009B03A0919C03B0919D03A070B070282BA0
:107E1000392B4A2B5B2B20939A0330939B0340937F
:107E20009C0350939D030E946D120895FC01809164
:107E3000940390919503E817F90711F51092B30395
:107E40006093B20360E070E080919A0390919B038D
:107E5000A0919C03B0919D0380709070482B592B8A
:107E60006A2B7B2B222311F0616001C06E7F40934F
:107E70009A0350939B0360939C0370939D030FC0E0
:107E80008091960390919703E817F90751F41092A7
:107E9000B3036093B20350939F0340939E030E94E9
:107EA0006D1208951F93182F80E06CE00E94481F08
:107EB000112309F100D000D00F92EDB7FEB7319633
:107EC00082E0ADB7BEB711968C938BEB93E09283B3
:107ED00081838091B40390E08F7790709483838343
:107EE0000E94C2200F900F900F900F900F9080E093
:107EF0000E94FF1E05C082E066EB73E00E941C2119
:107F00001F910895EF92FF920F931F93182F80FFF8
:107F100002C083E001C085EA0E94FF1EE12E11FF2E
:107F200002C084E001C085EA0E94FF1EE2FE02C09A
:107F300085E001C085EA0E94FF1EE3FE02C086E0E4
:107F400001C085EA0E94FF1EE4FE02C087E001C076
:107F500085EA0E94FF1E1F910F91FF90EF900895F8
:107F60006091A0037091A1038091A2039091A3035B
:107F7000611571058105910561F00E942F19882313
:107F800041F01092A0031092A1031092A20310924C
:107F9000A3036091A4037091A5038091A60390911F
:107FA000A703611571058105910571F00E942F19D4
:107FB000882351F01092A4031092A5031092A603F7
:107FC0001092A7030E946D126091A8037091A903FB
:107FD0008091AA039091AB0361157105810591050C
:107FE00061F00E942F19882341F01092A80310928B
:107FF000A9031092AA031092AB038091B303181641
:108000006CF42091B20330E02F7730708091B5038B
:1080100090E02817390714F01092B3038091B3034E
:1080200087FF09C08091B20390E08F779070892B11
:1080300011F41092B3038091B30320918F03309118
:1080400090034091910350919203882381F421156C
:1080500031054105510511F00E946D1210928F03F8
:10806000109290031092910310929203089521159B
:1080700031054105510539F0CA01B9010E942F1996
:10808000882309F46CC08091B303181644F40E944D
:108090006A12833049F48091B2038F5F03C08091EC
:1080A000B20381508093B2038091B303813059F0C1
:1080B0008F3F49F0823061F08E3F51F028E833E184
:1080C00040E050E009C020E335E740E050E004C064
:1080D00020EE3EE240E050E08091B5038E3781F41F
:1080E0008091DA079091DB07A091DC07B091DD0762
:1080F000E7E05695479537952795EA95D1F721C042
:108100008E3081F48091DA079091DB07A091DC0733
:10811000B091DD0774E056954795379527957A9588
:10812000D1F70FC08091DA079091DB07A091DC07AF
:10813000B091DD0765E056954795379527956A9587
:10814000D1F7280F391F4A1F5B1F20938F033093ED
:10815000900340939103509392030E946D120895EF
:108160008091B00380FD25C06091A0037091A103B0
:108170008091A2039091A30361157105810591057A
:1081800021F00E942F198823A1F0109297031092DA
:1081900096031092B7031092B603109295031092B3
:1081A00094031092B0031092B8030E946D1281E004
:1081B000089580E00895DF92EF92FF920F931F934E
:1081C0001091C403112399F081E060E00E94481FE0
:1081D000812F81500E94316CBC0182E00E941C21E1
:1081E0001092C40388EE93E00E94F51902C0882320
:1081F00019F00E943C1F04C080E060E00E94481F0C
:108200008091940390919503892BF9F00E947C6CE6
:10821000FC014091940350919503828193818417CE
:10822000950749F4218532858091B6039091B70373
:108230002817390751F0538342838091B6039091F8
:10824000B703928781870E94E86E20919403309152
:10825000950321153105C9F410929A0310929B03DE
:1082600010929C0310929D031092B30310929F03EF
:1082700010929E031092B2031092B4038091B00347
:108280008F7E8093B0031092B1038091B00382FD82
:108290000DC08091AC039091AD03A091AE03B0915D
:1082A000AF030097A105B10531F430C082E065E16C
:1082B00074E00E941C218DB79EB707970FB6F89403
:1082C0009EBF0FBE8DBFEDB7FEB7319682E0ADB752
:1082D000BEB711968C9382E094E092838183809163
:1082E000AC039091AD03A091AE03B091AF03838333
:1082F0009483A583B6830E94C220EDB7FEB737965C
:108300000FB6F894FEBF0FBEEDBF51C02115310569
:1083100031F482E06BEF73E00E941C2121C000D099
:1083200000D00F92EDB7FEB7319682E0ADB7BEB781
:1083300011968C9386EF93E0928381833483238319
:108340000E94C2208091B0030F900F900F900F9069
:108350000F9080FF02C081E001C080E20E94FF1EFA
:108360001091B1030E946A12682F863008F06150A4
:10837000633091F48091940390919503892B61F07F
:10838000612F70E06370707013E0660F771F1A95AD
:10839000E1F76A5A7C4F08C070E0B3E0660F771FC0
:1083A000BA95E1F76A587C4F82E00E941C2180E078
:1083B0006CE00E94481F8091B00383FF12C000D080
:1083C00000D00F92EDB7FEB7319682E0ADB7BEB7E1
:1083D00011968C9382EF93E0928381838091B40312
:1083E00011C000D000D00F92EDB7FEB7319682E0F9
:1083F000ADB7BEB711968C938EEE93E092838183D6
:108400008091B20390E08F779070948383830E9471
:10841000C2200F900F900F900F900F9080919403B7
:1084200090919503892B89F08091B10383708130FD
:1084300081F487E10E94401D882339F080E00E948A
:10844000FF1E80E06EEE71E05BC080E20E94FF1EC6
:1084500059C080E00E94FF1E0E947C6CFC0180815C
:1084600085FF43C08091B20387FF04C080E062EFC4
:1084700070E003C080E066EF70E040E024E00E941E
:10848000F21F8091B3038823E1F018163CF08E3F71
:1084900081F08F3F94F48D3FA9F507C08230C9F079
:1084A00082309CF0833071F518C080E062E171E0A9
:1084B00017C080E06EE071E013C080E06AE071E018
:1084C0000FC080E06AEF70E00BC080E06EEF70E0FC
:1084D00007C080E062E071E003C080E066E071E028
:1084E00044E024E00E94F21F0DC08091B20387FF98
:1084F00004C080E062EE70E003C080E06AEE70E0ED
:108500000E9429200E946A12813049F489E00E9469
:108510004D6CAC0181E060E00E94A21F03C280911B
:10852000B00383FD06C080E060E040E050E00E94C0
:10853000511F8091B00387FD03C000E010E014C01C
:108540008091960390919703892B19F001E010E038
:108550000BC08091B1030E942F3E20E030E08530B7
:1085600010F021E030E08901F02E81E060E00E940F
:10857000481F8091AC039091AD03A091AE03B091E0
:10858000AF030097A105B10509F429C18DE00E9450
:10859000401D882329F48EE00E94401D882381F12C
:1085A00000D00F9282E0EDB7FEB7818382EE93E0B8
:1085B000938382830E94C2200F900F900F908DE0D2
:1085C0000E94401D882369F081E066EA71E00E9404
:1085D000292082E06EEA71E00E9429208AEC9EE365
:1085E0000CC081E06EE971E00E94292082E066EB18
:1085F00071E00E9429208EEB9EE36CE271E0ECC0FA
:1086000087E00E944D6CBC0182E00E941C2187E043
:108610000E944D6C0E9410AA182F04C080E20E9494
:10862000FF1E1F5F1031D0F31091B103812F0E9404
:108630002F3E90E0A0E0B0E02091AC033091AD037C
:108640004091AE035091AF0382179307A407B5077B
:108650000CF44DC081E06BE00E94481F6091AC03B8
:108660007091AD0381E090E0A0E0B0E0062E04C080
:10867000880F991FAA1FBB1F0A94D2F720919A0353
:1086800030919B0340919C0350919D03822393233F
:10869000A423B5230097A105B10519F425EA30E01C
:1086A00002C023E030E08DB79EB707970FB6F8946D
:1086B0009EBF0FBE8DBFEDB7FEB7319682E0ADB75E
:1086C000BEB711968C9389ED93E092838183CB01A1
:1086D00063839483368325830E94C220EDB7FEB75F
:1086E00037960FB6F894FEBF0FBEEDBFC0C0137033
:1086F000133009F0BCC08FE00E94401D882351F464
:1087000080E10E94401D882329F48CE00E94401DD6
:10871000882369F180E10E94401D882321F081E0D7
:1087200066E272E003C081E06EE172E00E942920FF
:1087300081E06FE00E94481F00D000D00F92EDB79B
:10874000FEB7319682E0ADB7BEB711968C9386ED39
:1087500093E09283818381E090E0948383830E94FD
:10876000C2200F900F900F900F900F90DBC081E010
:1087700066E272E00E94292081E06BE00E94481FBF
:10878000EDB7FEB739970FB6F894FEBF0FBEEDBF39
:10879000319682E0ADB7BEB711968C938DEC93E025
:1087A0009283818386E090E09483838387E090E0E6
:1087B0009683858381E090E0908787830E94C22022
:1087C000EDB7FEB739960FB6F894FEBF0FBEEDBFFA
:1087D0008CE99EE368EC70E00E94871EA3C02091A4
:1087E0009603309197032115310539F100D000D05F
:1087F0000F92EDB7FEB7319682E0ADB7BEB71196D6
:108800008C9388EC93E092838183348323830E944A
:10881000C2200F900F900F900F900F9080919E03A9
:108820008F710E94823F002321F08CE30E94FF1E83
:108830002DC080E20E94FF1E1CC000D000D00F920D
:10884000EDB7FEB7319682E0ADB7BEB711968C9307
:108850008FEB93E09283818388EB93E0948383830F
:108860000E94C2200F900F900F900F900F90FF204A
:1088700069F48091A4039091A503A091A603B091FF
:10888000A7030097A105B10509F444C080919603A0
:1088900090919703892BF1F58091B1030E942F3EAF
:1088A0008530C0F181E060E00E94481F86E40E94AC
:1088B000FF1EA2E0EA2EF12C012D112DDD24D39410
:1088C00080919A0390919B03A0919C03B0919D038A
:1088D0008E219F21A023B1230097A105B10549F066
:1088E000B9E0BD1518F08D2D805D04C08D2D885028
:1088F00001C085EA0E94FF1ED394E0E1DE1629F054
:10890000EE0CFF1C001F111FDBCF80E20E94FF1E38
:1089100081E006C080919A038F710E94823F80E0BF
:108920000E945E3E1F910F91FF90EF90DF9008959F
:10893000CF93DF93EB018093B103E82FF0E0EF706A
:10894000F070E85EFB4FE491E093B50361157105AB
:1089500059F0CB0160E070E048EB53E00E941A86CA
:10896000D093B703C093B6030E946D12DF91CF91ED
:1089700008951F93FC01009769F41092B0031092C0
:10898000A0031092A1031092A2031092A3030E94CD
:10899000B04064C07091B00371FD60C06093B203D9
:1089A000CA01A0E0B0E020919A0330919B0340916E
:1089B0009C0350919D0320703070822B932BA42B2D
:1089C000B52B80939A0390939B03A0939C03B09341
:1089D0009D038091DA079091DB07A091DC07B091AD
:1089E000DD0788519C4FAF4FBF4F81608093A0033C
:1089F0009093A103A093A203B093A30372FF25C099
:108A000071607B7F7093B003F0939703E0939603BC
:108A1000CF010E94B838FC01009761F08091B20349
:108A20009085892787FF06C0609196037091970310
:108A3000706804C0609196037091970380919403CD
:108A4000909195030E947A3C07C07E7F7093B0039B
:108A5000F0939503E09394030E946D121F91089583
:108A6000AC018091B0038C7F8093B0031092B70368
:108A70001092B603662309F045C01092B803209106
:108A80009403309195032115310521F0309399031A
:108A90002093980310929A0310929B0310929C03C8
:108AA00010929D0310929F0310929E0310929703C1
:108AB0001092960310929503109294031092B303B0
:108AC0001092B1031092360C4115510551F18FEF00
:108AD000BA010E94CA6E8091B00381FD22C010923B
:108AE0009A0310929B0310929C0310929D03109284
:108AF000970310929603109295031092940310928C
:108B0000B1030DC01092360C6091940370919503DF
:108B10008FEF0E94486E8091B00381FD02C090E00B
:108B200001C091E08091B0038B7F82608093B0039D
:108B3000892F0895CF93DF93EC01288D398D4A8DCD
:108B40005B8D203088E2380780E0480780E05807D6
:108B50001CF08C8D86FF5DC0203080E4380780E0FB
:108B6000480780E058070CF054C06A817B812115CA
:108B700031054105510509F443C061157105E1F066
:108B800088819981A0E0B0E082179307A407B50718
:108B900041F0CB01A0E0B0E082179307A407B5072E
:108BA00059F48C8D8E7F8C8F888199810E94B73C7F
:108BB0001B821A821982188288819981A0E0B0E014
:108BC000288D398D4A8D5B8D82179307A407B507D1
:108BD00029F48C8D91E089278B7F16C081E060E0BD
:108BE0000E94481F80E00E944D6CBC0182E00E9400
:108BF0001C216C8D6470888D998D0E94304505C054
:108C0000672B19F48C8D84608C8F188E198E1A8EB8
:108C10001B8EDF91CF910895DF92EF92FF920F9319
:108C20001F939C018531910509F465C38631910537
:108C300024F58C30910509F480C18D309105A4F4A0
:108C40008A30910544F4813091050CF0AAC3009755
:108C500009F45BC3F0C38A30910509F4D4C38B30A7
:108C6000910509F0E8C3C6C3813191050CF054C2E7
:108C70008F3091050CF0BFC206C28A38910509F405
:108C8000BEC38B389105C4F48B31910564F48931EE
:108C900091053CF58631910509F4E1C287319105D2
:108CA00009F0C9C30FC18132910509F4D0C28332E2
:108CB000910509F0C0C3B6C38F3891054CF48D38C7
:108CC00091050CF0E0C18C38910509F0B4C3B5C131
:108CD000813991050CF4ADC28739910509F0ABC318
:108CE000A8C38091B00383FF03C01091B40302C0F6
:108CF0001091B20300E02931310509F401E0E09060
:108D0000B5030E947C6CFC01F7800E947C6CFC0126
:108D1000808184FF35C017FD05C080E0002309F481
:108D200081E0082F002311F001E02CC0812F90E09A
:108D30008F779070892B79F48091A8039091A90383
:108D4000A091AA03B091AB030097A105B10519F456
:108D5000212F2058ADC08091DA079091DB07A091B8
:108D6000DC07B091DD07845D9E4FAF4FBF4F80930E
:108D7000A8039093A903A093AA03B093AB0324C0C4
:108D8000002311F10E947C6CFC01808185FF07C0EB
:108D90008091B30383300CF08AC08F5F21C00E94A2
:108DA0006A12833009F083C0812F90E08F77907032
:108DB0002E2D30E0821793070CF079C0FEE7EF16F6
:108DC000E1F5FF20E1F439C00E947C6CFC01808158
:108DD00085FF09C08091B3038E3F0CF468C08150B9
:108DE0008093B30364C0812F90E08F779070892BBC
:108DF00009F45DC04EE7E41641F5FF2031F181E052
:108E0000F81619F460E820E00EC0E2E0FE1619F44E
:108E10006EE324E108C0F3E0FF1619F466E12AE0EE
:108E200002C060E820E8812F90E030E0002341F0AC
:108E30008F779070821793075CF4212F2F5F38C0D3
:108E40008F779070281739071CF0212F215030C0E0
:108E5000462F50E0812F90E08F7790704817590788
:108E60001CF0212F2E7F04C0212F261B2C7F260FC4
:108E7000211719F0002319F41BC0002361F0822F81
:108E800090E08F7790708417950714F482E001C00A
:108E900084E0280F0DC0822F90E08F7790704817E4
:108EA000590714F082E001C084E0281B01C0212F83
:108EB0008091B00383FF03C02093B40320782093F4
:108EC000B203B7C29091B00397FF21C088E0892711
:108ED0008093B00383FF0EC08091B2038093B403EC
:108EE00080788093B2031092B30382E59FE360E938
:108EF00071E00AC08091B4038093B2031092B4036E
:108F000080E090E060E070E00E94871E92C2809155
:108F1000B1038370813029F480E06EEE71E00E942D
:108F200029208091B203805880788093B2031092F8
:108F3000B3038091B003877F72C2809196039091B2
:108F40009703009709F049C0E090AC03F090AD039F
:108F50000091AE031091AF031E141F0410061106FA
:108F6000E4F5D090B1038D2D0E942F3E90E0A0E05B
:108F7000B0E08E159F05A007B1071CF181E090E0DD
:108F8000A0E0B0E004C0880F991FAA1FBB1FEA949D
:108F9000D2F720919A0330919B0340919C0350910A
:108FA0009D0382279327A427B52780939A03909344
:108FB0009B03A0939C03B0939D038091B0038068B2
:108FC0003BC143E0D422D41609F033C2809194030C
:108FD00090919503B70141E026C16091B00367FF0E
:108FE00010C0892B71F080919E0390919F0321E026
:108FF00030E08227932790939F0380939E036061C4
:1090000019C080919A0390919B03A0919C03B09109
:109010009D0321E030E040E050E082279327A42721
:10902000B52780939A0390939B03A0939C03B093DE
:109030009D036F7E6093B003FCC180919603909175
:109040009703892B29F48091B0038F778093B00325
:109050008091B00385FFEDC12091AC033091AD0349
:109060004091AE035091AF03121613061406150675
:109070000CF0DFC08091940390919503B90140E01A
:109080000E940A38D6C08091AC039091AD03A091A4
:10909000AE03B091AF030097A105B105D9F1893FA7
:1090A000E7E09E07E0E0AE07E0E0BE070CF0C1C1DC
:1090B000AC0141505040440F551FC9018F7790704B
:1090C0000E9709F4416027FF1FC0CA0160E044E029
:1090D0000E94D28F8091B00383FD05C080E090E0B4
:1090E00060E070E004C082E59FE360E971E00E9407
:1090F000871E81E066E271E00E94292082E06EE234
:1091000071E00E9429209AC0CA0161E044E00E94F7
:10911000D28F8FC127FD8DC1022F0D501091B0034A
:1091200017FF0AC08091960390919703892B21F431
:10913000213131050CF40C5F8091B1030E942F3E68
:10914000081708F076C10430A0F08091DA079091FA
:10915000DB07A091DC07B091DD078C509E4FAF4F2D
:10916000BF4F8093A4039093A503A093A603B0934D
:10917000A70317FF1DC08091960390919703892B39
:10918000B9F082E090E0A0E0B0E004C0880F991F41
:10919000AA1FBB1F0A95D2F720919E0330919F030F
:1091A0002827392730939F0320939E03106120C006
:1091B00082E090E0A0E0B0E004C0880F991FAA1FF1
:1091C000BB1F0A95D2F720919A0330919B034091DF
:1091D0009C0350919D0382279327A427B527809352
:1091E0009A0390939B03A0939C03B0939D031F7ECF
:1091F0001093B0031EC1E090AC03F090AD0300915A
:10920000AE031091AF03E114F1040105110509F457
:1092100083CF809194039091950340E02F303105E6
:1092200009F441E0B7010E940A388091B0038062DE
:10923000F6C08091B0038F7D8093B0031092AC0391
:109240001092AD031092AE031092AF03F2C0809162
:109250009403909195036CE30E94EA37EAC08091F1
:10926000AC039091AD03A091AE03B091AF03009712
:10927000A105B10571F18091B00382FD2AC00E9461
:109280006A12833019F58091B503282F30E040E051
:1092900050E08091AC039091AD03A091AE03B091EA
:1092A000AF03281739074A075B0744F42093AC0340
:1092B0003093AD034093AE035093AF038091B2035C
:1092C00080789091AC03892B8093B2031092B30302
:1092D000B5CFF89483E00E94851287E10E94401D7B
:1092E000882339F080919403909195036BE40E9458
:1092F000EA3778949EC08091B00387FF02C082E075
:1093000001C080E00E94851294C08091B00387FF65
:1093100012C08091980390919903009709F48BC033
:10932000A0E0B0E08093AC039093AD03A093AE03B4
:10933000B093AF031EC082FF21C08091AC03909117
:10934000AD03A091AE03B091AF030097A105B105A5
:10935000A9F489E00E948BA68091AC039091AD03A3
:10936000A091AE03B091AF030097A105B10509F438
:1093700062C084E993E00E949A455DC08091AC038D
:109380009091AD03A091AE03B091AF030097A105FA
:10939000B10539F48FEF0E948BA681E00E94DB407B
:1093A0004AC079010027F7FC0095102F6091AC03AB
:1093B0007091AD038091AE039091AF032AE030E04D
:1093C00040E050E00E9448A8E60EF71E081F191F53
:1093D000F0E0EF16F0E8FF06F0E00F07F0E01F07FF
:1093E00054F5E092AC03F092AD030093AE031093FA
:1093F000AF031FC084E993E00E949A451AC0809190
:10940000B0038F770CC01092AC031092AD03109292
:10941000AE031092AF038091B0038B7F806880937E
:10942000B00307C08091B20380788093B20310929A
:10943000B3030E946D121F910F91FF90EF90DF9088
:109440000895FC01EC5AFF4F2081E455F04022239F
:10945000C1F0E95AFF4F8081E755F040948180FDCB
:1094600008C0983511F0983761F4223020F481E07B
:109470000895892F01C085818095881F8827881FBE
:10948000089580E0089580E008950F931F93CF938F
:10949000DF93182FEB01622F9E0170E02EC0CA01EE
:1094A0008095909528233923DA01AC23BD231097AA
:1094B00011F0A1E0B0E06031B8F46117A8F4862F94
:1094C00090E0FC01E295F295F07FFE27E07FFE2719
:1094D000E81BF90BEA58FB4F8685882329F0808129
:1094E00091818230910508F0CD01892B11F0242B58
:1094F000352B7F5F440F551F6F5F701780F2C901D6
:10950000DF91CF911F910F910895E82F4423E9F047
:1095100088E5E89FF0011124EA53FC4F8091840410
:10952000882371F0809176049091770482309105C0
:1095300038F4892B29F0E95AFF4F8081816004C0FB
:10954000E95AFF4F80818E7F808381E008956530E6
:1095500069F1663070F4623001F1633028F46623FB
:10956000B1F06130B1F516C06330D1F0643089F5E7
:109570001AC0683021F1693028F46630D1F06730C4
:1095800041F51AC06930F1F0603119F51EC063ED84
:1095900077E01DC06DEC77E01AC069EC77E017C08A
:1095A00066EC77E014C060EC77E011C069EB77E01F
:1095B0000EC06EEA77E00BC067EA77E008C06FE99B
:1095C00077E005C060E977E002C068E877E00E94D4
:1095D0001C2181E0089560E979E00E941C2181E06E
:1095E000089569EC79E00E941C2181E0089566EEFF
:1095F00079E00E941C2181E008951F93182F69E5EE
:109600007AE00E941C21812F6AE37AE00E941C21EB
:10961000812F6DE17AE00E941C2181E01F91089565
:10962000CF93DF93EC01009719F16EE777E00E948A
:1096300007AA892B11F481E01CC0CE016AE777E00C
:109640000E9407AA892B11F482E013C0CE0166E7BD
:1096500077E00E9407AA892B11F483E00AC0CE01AB
:1096600063E777E00E9407AA892B11F480E001C02C
:109670008FEFDF91CF9108952F923F924F925F929B
:109680006F927F928F929F92AF92BF92CF92DF9212
:10969000EF92FF920F931F93DF93CF9300D0CDB73C
:1096A000DEB79A83898380EFE6E7F4E0DF011D925D
:1096B0008A95E9F749805A80F2019081992399F0BF
:1096C0009C3289F0943279F0953269F0892F805379
:1096D0008A3048F0892F992787FD90950E94F8A934
:1096E000892B09F4DFC096E7692E94E0792EAA242D
:1096F000A3941E010894211C311CADC00F5F1F4FA5
:109700001A83098309811A81D801BC908B2D99276E
:1097100087FD90950E94F8A9892B81F7BB2009F459
:10972000AAC0BCE2BB1609F48DC0E7E2BE1629F060
:10973000F2E2BF1611F0BB2404C00F5F1F4F1A8363
:10974000098382E0882E912C860C971CC980DA80D0
:10975000EE24FF2409C0D4011D934D010894C11CBF
:10976000D11C0894E11CF11CBBE0EB16F1049CF445
:10977000F6011081112379F0BB2019F01B1559F760
:109780000AC01C3241F0812F992787FD90950E94D5
:10979000F8A9892B01F3D4011C92E981FA81808117
:1097A000843241F4CF0101969A838983B10140E16B
:1097B00050E013C0853269F4CF0101969A83898302
:1097C000B10142E050E00E949AA8D3016D937C93CE
:1097D00009C0CF01B1014AE050E00E949AA8F3010C
:1097E00071836083E1E0D3011E96EC9304C00F5FA8
:1097F0001F4F1A83098309811A81D801FC90FF2029
:1098000081F08F2D992787FD90950E94F8A9892BCB
:1098100041F4BCE2FB1659F704C00F5F1F4F1A83D7
:10982000098309811A81F801F080FF2079F08F2DDA
:10983000992787FD90950E94F8A9892B71F7FCE282
:10984000FF1621F40F5F1F4F1A830983A3948FE043
:1098500090E0680E791EFA2CFA94E981FA818081F1
:10986000882321F091E1A91609F04CCF411451044D
:1098700011F0D2011C928F2D90E00F900F90CF919C
:10988000DF911F910F91FF90EF90DF90CF90BF90ED
:10989000AF909F908F907F906F905F904F903F9090
:1098A0002F9008950894411C511C5A82498202CF7E
:1098B0000F931F93082F162F603418F067ED75E093
:1098C00002C06FEC75E00E941C211A30A1F11B3020
:1098D00080F4163021F1173030F41130C1F012301D
:1098E00009F045C018C0183011F1193009F03FC017
:1098F0001AC01E3071F11F3028F41B3001F11D30E9
:10990000B1F521C0113449F1123489F52AC0802FF4
:109910006FEB75E01BC0802F6BEA75E017C0802FDE
:109920006EE975E013C0802F6BE875E00FC0802FE3
:1099300068E775E00BC0802F60E775E007C0802FF7
:109940006EE575E003C0802F65E575E00E941C217F
:1099500014C0802F6EE375E0F9CF802F63E375E0CC
:1099600003C0802F68E275E00E941C2102C0103401
:1099700020F0802F6DE00E94422081E01F910F9126
:109980000895782F6031C8F46417B8F4862F90E0FA
:10999000FC0144E0EE0FFF1F4A95E1F7E81BF90BCD
:1099A000EA58FB4F8685882341F040815181241776
:1099B000350718F04115510531F4872F62E00E94F8
:1099C000584C40E050E0CA0108950F931F93082FB0
:1099D000142F0E941C21802F60E20E94422011233C
:1099E00019F462E477E002C065E477E0802F0E941A
:1099F0001C21802F6DE00E9442201F910F9108953D
:109A0000DF92EF92FF920F931F93CF93DF93082F74
:109A10007B01EA01D22E10E012C0802F60E20E948A
:109A20004220CE018E219F21892B11F460E301C0D9
:109A300061E3802F0E9442201F5FCC0FDD1F1D15A8
:109A400060F3DF91CF911F910F91FF90EF90DF9026
:109A5000089560E00E9442208FEF08950F931F93B6
:109A6000182FFB010181002311F482E011C060E096
:109A70000E944220E02FF0E0E554F24F60816095B3
:109A8000812F0E944220812F60E00E9442208FEFB0
:109A90001F910F910895982F442309F440C080919D
:109AA00084048823E1F16091760470917704611554
:109AB0007105A9F120E46030720788F5272F33275C
:109AC0002F73307020543F4FAB015070ADB7BEB70D
:109AD0001F970FB6F894BEBF0FBEADBFEDB7FEB770
:109AE000319611969C9380EF97E0928381837483E3
:109AF0006383768365833087278332872187548702
:109B00004387568745870E94C22081E0EDB7FEB7A4
:109B10003F960FB6F894FEBF0FBEEDBF0895892F94
:109B200061E00E94A74A0895682F442371F0809154
:109B30008404882351F08091760490917704803CCE
:109B4000910518F0883E910510F080E090E0582FC4
:109B5000423060F080919304882341F02091850485
:109B6000309186042F3F310519F010F020E030E0ED
:109B7000852F805C883228F0862F61E00E94A74AFA
:109B8000089500D000D00F92EDB7FEB73196ADB773
:109B9000BEB711966C938BE298E092838183852FF8
:109BA00090E08F739070982F8827820F911D948377
:109BB00083830E94C22081E00F900F900F900F903E
:109BC0000F900895CF92DF92EF92FF920F931F9321
:109BD000DF93CF9300D000D000D0CDB7DEB7D82E22
:109BE0002DB73EB7275030400FB6F8943EBF0FBE9A
:109BF0002DBFEDB7FEB73196ADB7BEB711968C93BA
:109C000083EF95E0928381838DE090E0948383835A
:109C10008DEE95E0968385830E94C220EDB7FEB756
:109C200037960FB6F894FEBF0FBEEDBFDD2019F4D6
:109C300086E79FE402C081E79FE40E94D76F88E037
:109C4000E6E6F5E0DF011D928A95E9F700E010E015
:109C500031E0E32EF12C802F0E9433708823A9F08D
:109C6000F80123E0F595E7952A95E1F7EA59FA4FCF
:109C7000C80187709070970102C0220F331F8A9528
:109C8000E2F7C9012081282B20830F5F1F4F00348A
:109C9000110509F78E010F5F1F4F86E0D8011D9255
:109CA0008A95E9F78FEF6CE1A8010E94BE7094E1FC
:109CB000E92EF12CC02E012F23C0F901EA59FA4FE9
:109CC0008081882329F42F5F3F4F28303105A9F781
:109CD00028303105C0F48AE090E00E94F51908941C
:109CE000E108F108BAE0EB16F10439F48FEF6CE10A
:109CF0004C2D502F0E94BE7003C01E141F041CF474
:109D000020E030E0E2CF80E090E00E94D76F00E0FA
:109D100010E087EEE82E85E0F82EF801B3E0F59527
:109D2000E795BA95E1F7EA59FA4F808190E09801FA
:109D30002770307002C0959587952A95E2F780FFCD
:109D400015C000D000D00F92EDB7FEB73196ADB779
:109D5000BEB71196DC92F282E182148303830E94E3
:109D6000C2200F900F900F900F900F900F5F1F4F1A
:109D70000034110591F68D2D61EE75E00E941C21D5
:109D800081E026960FB6F894DEBF0FBECDBFCF910F
:109D9000DF911F910F91FF90EF90DF90CF9008958A
:109DA0001F93CF93DF93182FEB0198819F3F31F0E2
:109DB00089818C3119F48A81882321F4CE010E9493
:109DC0002E788BC09F77892F869586958695E82F6C
:109DD000F0E0EA59FA4F4081692F70E09B0127704B
:109DE0003070842F90E0022E02C0959587950A94DA
:109DF000E2F780FF72C081E090E002C0880F991FF7
:109E00002A95E2F78095842380838E81863211F42F
:109E10008FED8E838DB79EB70D970FB6F8949EBFCA
:109E20000FBE8DBFEDB7FEB73196ADB7BEB7119679
:109E30001C9382E096E092838183748363838A819A
:109E4000858316828B81878310868C818187128619
:109E50008D81838714860E94C2202E818DB79EB784
:109E60000D960FB6F8949EBF0FBE8DBF222389F1C9
:109E700000D000D00F92EDB7FEB73196ADB7BEB7A8
:109E800011961C938FEF95E0928381832383148234
:109E90000E94C2206F810F900F900F900F900F9033
:109EA0006623B9F000D000D00F92EDB7FEB731961F
:109EB000ADB7BEB711961C938CEF95E0928381836A
:109EC000638314820E94C2200F900F900F900F9016
:109ED0000F90812F6DE00E944220DF91CF911F9162
:109EE0000895BC0181E00E94D04E0895BC0180E03D
:109EF0000E94D04E08950E946B3284E06EEB71E0B8
:109F00000E94292085E066EC71E00E94292082E809
:109F10009EE968EC70E00E94871E80E060E00E948D
:109F2000481F0E94553B0E9488840E94436F0E94F4
:109F3000C36C81E008950F93042F82E00E94896C26
:109F4000882329F482E00E940E6F0E94E86E0023AD
:109F500009F46EC080918404882351F0A0917604A6
:109F6000B0917704109731F080E4A030B80710F07A
:109F7000A0E0B0E0023008F45DC080919304882333
:109F800041F0409185045091860484E040305807A8
:109F900010F04FEF5FEF023009F44EC08091A20441
:109FA000882339F0609194047091950460347105B0
:109FB00010F06FEF7FEF033009F440C08091B104DF
:109FC000882341F02091A3043091A4042F3F310550
:109FD00019F010F02FEF3FEF043061F08091C004D2
:109FE000882341F0E091B204F091B304EF3FF10512
:109FF00019F010F0E8E0F0E084E040305807A8F4F1
:10A000006034710590F42F3F310509F070F4F6E0EB
:10A01000440F551FFA95E1F7462B572BCD016AE007
:10A020000E2F0E94493381E001C080E00F91089516
:10A03000A0E0B0E04FEF5FEF6FEF7FEFE8E0F0E020
:10A040002FEF3FEFD9CF0F931F93082F142F82E0EC
:10A050000E94896C882329F482E00E940E6F0E947E
:10A06000E86E112379F080918404882359F060917F
:10A070007604709177046115710531F080E46030E9
:10A08000780710F060E070E08FEF0E94577E9B0130
:10A09000AC01611571058105910501F1ADB7BEB740
:10A0A00017970FB6F894BEBF0FBEADBFEDB7FEB7A2
:10A0B000319611960C9387E196E0928381832383F6
:10A0C0003483458356830E94C220EDB7FEB737968E
:10A0D0000FB6F894FEBF0FBEEDBF12C000D00F92B6
:10A0E000ADB7BEB711960C93119781E196E0139628
:10A0F0009C938E9312970E94C2200F900F900F9006
:10A1000081E01F910F91089566E879E00E941C217B
:10A1100082E00E94851280E0089583E00E9485120B
:10A1200080E0089580E00E94851280E0089560E05C
:10A130000E94422082E00E9485128FEF089580E005
:10A140000E9485120E94D6A681E008951F93182FC1
:10A150000E946A128430D1F0853038F4823071F078
:10A16000833080F4882331F01EC08730B8F0873008
:10A17000D1F410C0812F61ED78E013C0812F69EC1C
:10A1800078E00FC0812F62EC78E00BC0812F66EB86
:10A1900078E007C0812F6AEA78E003C0812F64EA83
:10A1A00078E00E941C2181E01F910895EF92FF92B8
:10A1B0000F931F93182F7B01042F83E00E948512B9
:10A1C000812FB701402F0E94A6501F910F91FF9041
:10A1D000EF900895EF92FF920F931F93182F7B013A
:10A1E000042F80E00E948512812FB701402F0E942A
:10A1F000A6501F910F91FF90EF9008951F93182F75
:10A200000E946A12833041F0873031F0823011F4BD
:10A2100068E103C060E001C068E0812F0E94422035
:10A220008FEF1F910895AF92BF92CF92DF92EF927E
:10A230000F931F93CF93DF93182F042F0E946A125E
:10A24000882319F4812F66E016C0002391F08091D5
:10A250008404882371F0A0907604B0907704A11450
:10A26000B10439F020E0A21628E2B20610F4023060
:10A2700028F4812F62E00E94584C58C080919304CA
:10A280008823B9F3C0908504D0908604C114D1040A
:10A2900081F331E0C31634E0D30658F7023061F0A1
:10A2A0008091A204882341F0C0919404D091950438
:10A2B000CF3FD10519F010F0C0E0D0E0C5010E94F9
:10A2C000E0388370833019F0812F6AE0D4CF960193
:10A2D00021503040C50160E041E000E0EC2E0E94DA
:10A2E00084388DB79EB709970FB6F8949EBF0FBEFE
:10A2F0008DBFEDB7FEB73196ADB7BEB711961C93C3
:10A300008DE196E092838183B482A382D682C58256
:10A31000D087C7830E94C22081E02DB73EB7275F58
:10A320003F4F0FB6F8943EBF0FBE2DBFDF91CF91C8
:10A330001F910F91EF90DF90CF90BF90AF90089555
:10A34000AF92BF92CF92DF92EF92FF920F931F9343
:10A35000CF93DF93B82E7B0180919304882309F477
:10A360007DC08091A204423008F478C00091850439
:10A37000109186040115110509F470C024E0013024
:10A38000120708F47AC06AC0423029F480E090E0F5
:10A3900020E030E019C020919404309195042F3FC3
:10A3A000310519F010F020E030E0443058F0809191
:10A3B000B104882339F08091A3049091A4048138DA
:10A3C000910510F080E090E0D22EC82EC7016DEE0E
:10A3D00077E00E9407AA892B39F0C7016AEE77E07F
:10A3E0000E9407AA892B01F5809184048823B1F18A
:10A3F000C0917604D091770481E0CF3FD80770F503
:10A40000C70167EE77E00E9407AA892B11F062E08E
:10A4100001C061E0219701501040CE01A3E0880FF8
:10A42000991FAA95E1F711C0809184048823B1F0A7
:10A430008091760490917704009781F020E4803039
:10A44000920760F40150104060E04A2D98010D2DF4
:10A45000EC2C0E9484388B2D60E002C08B2D61E0D3
:10A460000E94A74ADF91CF911F910F91FF90EF902B
:10A47000DF90CF90BF90AF900895AA24882309F071
:10A4800083CFAA24A394CC24DD24A0CFEF920F93F2
:10A49000FB01828190E087709070582F4427818162
:10A4A00090E0482B592B6381848197E0483F5907FE
:10A4B00000F590E087709070382F2227862F90E06B
:10A4C000282B392B2150304083E02F3F380788F468
:10A4D0008081893D29F4CA0162E040E0058104C021
:10A4E000CA0162E041E000E0EE240E94843880E08E
:10A4F00001C082E00F91EF9008951F93182F44231D
:10A5000059F080918404882339F0809176049091E9
:10A5100077048830910510F08FEF90E0883010F4C8
:10A520000E941A6F0E94836C00D000D00F92EDB78A
:10A53000FEB73196ADB7BEB711961C932AE236E04E
:10A5400032832183838314820E94C2200F900F9054
:10A550000F900F900F9081E01F9108951F93CF935C
:10A56000DF93142F80E00E94851288EE93E00E9412
:10A57000F519112371F080918404882351F0C09162
:10A580007604D0917704209721F0CF3FD10519F0C0
:10A5900010F0CEE4D0E0F89487E00E948512CE015E
:10A5A0000E94B33CCE0166E90E94EA37789481E0CC
:10A5B000DF91CF911F910895875E934091F56130AF
:10A5C00069F0613028F06230A9F0633051F51EC0A7
:10A5D0000E947C6CFC0180818F731DC00E947C6C8A
:10A5E000FC0180818F7780830E947C6CFC018081DC
:10A5F000806411C00E947C6CFC0180818068808333
:10A600000E947C6CFC0180818F7B05C00E947C6C69
:10A61000FC018081806C80830E94E86E20E030E045
:10A6200002C02FEF3FEFC9010895FB01928180E046
:10A63000218130E0822B932B63810E94DC52892F91
:10A64000881F8827881F880F08951F9381309105E0
:10A6500031F0875E9340A9F02FEF3FEF26C00E94B4
:10A660007C6CFC018181882311F484E608C084306D
:10A6700011F485E604C08150843008F08150282F01
:10A6800013C00E947C6CFC01808190E026E09695CE
:10A6900087952A95E1F7182F11700E947C6CFC01B8
:10A6A000808187FD1260212F30E0C9011F9108953C
:10A6B0001F93CF93DF93182F4423A9F18091840433
:10A6C000882341F0209176043091770483E0283E7E
:10A6D000380710F02FEF3FEF423039F580919304A7
:10A6E000882341F0C0918504D0918604CF3FD105E5
:10A6F00019F010F0C0E0D0E0C9016C2F0E94DC52CC
:10A7000097FD19C000D000D00F92EDB7FEB731967B
:10A71000ADB7BEB711961C938DE398E09283818309
:10A72000C38314821EC02FEF3FEFC9010E9425533F
:10A730009C0197FF05C0812F62E00E94584C19C010
:10A7400000D000D00F92EDB7FEB73196ADB7BEB7CF
:10A7500011961C938AE398E092838183307034834E
:10A7600023830E94C22081E00F900F900F900F90E2
:10A770000F90DF91CF911F9108951F93CF93DF9397
:10A78000182FFB01928180E0218130E0822B932BF6
:10A790000E942553EC0197FF02C082E009C0812F7F
:10A7A00060E00E944220812F6C2F0E9442208FEF98
:10A7B000DF91CF911F9108950F931F93CF93DF9354
:10A7C000082F142F0E947C6CDC0118968C91C82FE6
:10A7D000D0E0CC0FDD1F112361F080918404882329
:10A7E00041F080917604909177048134910508F4CA
:10A7F000EC010E947C6CFE01EF5F2E2F2695DC01A0
:10A8000018962C930E947C6C00D000D00F92EDB76C
:10A81000FEB73196ADB7BEB711960C932CE438E075
:10A8200032832183DC0118968C9190E0880F991F68
:10A83000948383830E94C2200F900F900F900F90FB
:10A840000F9081E0DF91CF911F910F9108950F93A9
:10A850001F93CF93DF93082F142F0E947C6CEC0181
:10A86000112351F14B8580918404882339F0209184
:10A870007604309177042531310518F0842F90E06B
:10A880009C012B878C85282F30E0220F331F12303C
:10A8900078F080919304882359F0809185049091F9
:10A8A00086048230910520F041E08F3F940708F044
:10A8B000C901969587958C870E94E86E8DB79EB7E3
:10A8C00007970FB6F8949EBF0FBE8DBFEDB7FEB7CA
:10A8D0003196ADB7BEB711960C938BE798E0928393
:10A8E00081838B85838314828C8590E0880F991FE8
:10A8F000968385830E94C2208DB79EB707960FB6B8
:10A90000F8949EBF0FBE8DBF81E0DF91CF911F9164
:10A910000F9108950F931F93FB010281818188237A
:10A9200019F08330C1F40CC00936A8F410E00F5FB1
:10A930001F4F159507950E947C6CFC01008709C08C
:10A940008091470D002311F0816001C08E7F8093BC
:10A95000470D80E001C082E01F910F9108950F9391
:10A960001F93082FFB018181882321F0833041F060
:10A9700082E012C00E947C6CFC011085110F03C0A4
:10A980001091470D1170802F60E00E944220802FAF
:10A99000612F0E9442208FEF1F910F910895EF9237
:10A9A000FF920F931F93CF93DF93082F142F0E94D2
:10A9B0007C6C7C0180918404882389F088E794E092
:10A9C00063E376E00E9407AAF7012081892B11F446
:10A9D0002B7F02C02460F70120830E94E930809120
:10A9E0009304882379F0123008F453C080918504D1
:10A9F00090918604893C910508F04BC097FD49C0B1
:10AA0000F70186838091A204882379F086E994E097
:10AA100060E376E00E9407AAF7012081892B11F4F8
:10AA2000277F02C02860F70120838091B10488232A
:10AA300059F08091A504F7012081893511F4216036
:10AA400002C02E7FF70120838091C004882369F023
:10AA50001530F8F08091B2049091B30485339105DC
:10AA6000C0F497FD16C0F70180878091CF0488233A
:10AA7000F1F0163070F0C091C104D091C204F4E03E
:10AA8000C03BDF0730F081EEC130D80710F410E092
:10AA900006C0802F62E00E94584C0CC01F5F812FBF
:10AAA0000E94D6148C179D07C8F3F70111830E94EA
:10AAB000E86E81E0DF91CF911F910F91FF90EF90B1
:10AAC00008950F931F93082F142F87E894E06DE3E8
:10AAD00076E00E9407AA892B19F063E070E002C0BB
:10AAE00061E070E090918404992341F48091930493
:10AAF000882321F0CB010E94D18D2DC0112361F05C
:10AB0000992351F020917604309177042F3F31053D
:10AB100009F010F437FF05C0802F62E00E94584C06
:10AB20001BC080919304F3E0220F331FFA95E1F7E5
:10AB3000882371F4C9010E94508D019719F066E3D2
:10AB400076E002C06AE376E0802F0E941C2103C0F9
:10AB5000C9010E94818D81E01F910F9108951F937B
:10AB6000182F67E978E00E941C21812F61E978E0C5
:10AB70000E941C210E94906C2DB73EB72750304098
:10AB80000FB6F8943EBF0FBE2DBFEDB7FEB731969E
:10AB9000ADB7BEB711961C9324E838E03283218309
:10ABA00063837483858396830E94C2202DB73EB74A
:10ABB000295F3F4F0FB6F8943EBF0FBE2DBF81E017
:10ABC0001F9108958F929F92AF92BF92CF92DF9282
:10ABD000EF92FF920F931F93DF93CF93CDB7DEB722
:10ABE00060970FB6F894DEBF0FBECDBFE82E82E0AF
:10ABF0000E9403829A8389834E010894811C911CD0
:10AC0000B3E0AB2EB12CAC0EBD1EA3E3CA2EA7E061
:10AC1000DA2E4BC080E1B4010E9479828501FF24C5
:10AC2000D8018D919C910097E1F19C013F77B0E4B0
:10AC300020303B07B0F5FF2019F480E091E002C01E
:10AC400081E091E0EDB7FEB737970FB6F894FEBFFD
:10AC50000FBEEDBF3196ADB7BEB71196EC92D28262
:10AC6000C18294838383368325830E94C220EDB7FB
:10AC7000FEB737960FB6F894FEBF0FBEEDBFFF20AC
:10AC800049F0D8018D919C9197FF04C08E2D61E20F
:10AC90000E944220F3940E5F1F4FB7E0FB1609F0AD
:10ACA000BFCF8E2D6DE00E94422089819A81892B31
:10ACB00009F0B0CF60960FB6F894DEBF0FBECDBFDF
:10ACC000CF91DF911F910F91FF90EF90DF90CF9088
:10ACD000BF90AF909F908F9008951F93182F0E9460
:10ACE000E255812F6DE677E00E941C2181E01F91E3
:10ACF00008954F925F926F927F928F929F92AF9240
:10AD0000BF92CF92DF92FF920F931F93DF93CF9367
:10AD1000CDB7DEB760970FB6F894DEBF0FBECDBFDC
:10AD2000F82E83E00E9403829A8389832E0108947F
:10AD3000411C511C9FE3692E97E0792E85E0882EF7
:10AD4000912C8C0E9D1E08E3A02E07E0B02E11E181
:10AD5000C12ED12CCC0EDD1E4BC080E1B2010E9471
:10AD6000798200D000D00F92EDB7FEB73196ADB723
:10AD7000BEB71196FC92728261828B819C81948312
:10AD800083830E94C22084010F900F900F900F9038
:10AD90000F90F8019181992311F12DB73EB72750FB
:10ADA00030400FB6F8943EBF0FBE2DBFEDB7FEB7D3
:10ADB0003196ADB7BEB71196FC92B282A182D8018E
:10ADC0008C9183831482958316820E94C220EDB7F2
:10ADD000FEB737960FB6F894FEBF0FBEEDBF0E5FFD
:10ADE0001F4F0C151D05A9F68F2D6DE00E94422006
:10ADF00089819A81892B09F0B0CF60960FB6F894BB
:10AE0000DEBF0FBECDBFCF91DF911F910F91FF909D
:10AE1000DF90CF90BF90AF909F908F907F906F907A
:10AE20005F904F9008951F93182F0E947956812F9D
:10AE300067E677E00E941C2181E01F910895EF9260
:10AE4000FF920F931F93CF93DF93F82E8B01E42E85
:10AE5000E901842F0E94253E2DB73EB72750304090
:10AE60000FB6F8943EBF0FBE2DBFEDB7FEB73196BB
:10AE7000ADB7BEB71196FC9220E637E0328321834E
:10AE800014830383968385830E94C2202E2D30E095
:10AE9000C9018370907001974DB75EB7495F5F4FEE
:10AEA0000FB6F8945EBF0FBE4DBF029778F4C9018C
:10AEB0008C7090708430910519F48F2D61E604C078
:10AEC000089721F48F2D62E60E9442208F2D6DE5B8
:10AED00077E00E941C214E2D50E0437050704130AD
:10AEE000510569F0423051051CF4452BA1F018C002
:10AEF0004230510541F04330510591F408C08F2D87
:10AF000069E577E00BC08F2D65E577E007C08F2DF1
:10AF100061E577E003C08F2D6EE477E00E941C218D
:10AF20002097D1F088818823B9F000D000D00F920B
:10AF3000EDB7FEB73196ADB7BEB71196FC9289E476
:10AF400097E092838183D483C3830E94C2200F90B1
:10AF50000F900F900F900F908F2D6DE00E94422068
:10AF6000DF91CF911F910F91FF90EF9008959F92E5
:10AF7000AF92BF92CF92DF92EF92FF920F931F9307
:10AF8000DF93CF93CDB7DEB72D970FB6F894DEBF22
:10AF90000FBECDBF982E80E090E00E949F857C017F
:10AFA0008C0122E0C22ED12CCC0EDD1E5E01089455
:10AFB000A11CB11C14C0C801B501A6010E941A86CB
:10AFC000BC01009779F0892D498196010E941F5795
:10AFD000C8010E949F858C018E159F0519F00115EF
:10AFE000110549F72D960FB6F894DEBF0FBECDBF01
:10AFF000CF91DF911F910F91FF90EF90DF90CF9055
:10B00000BF90AF909F900895AF92BF92CF92DF9282
:10B01000EF92FF920F931F93CF93DF93082F0E941D
:10B020007C6C6C01802F6BE277E00E941C21802FEA
:10B0300062E277E00E941C21802F6CE177E00E94A1
:10B040001C21802F6DE00E94422000D000D00F9282
:10B05000EDB7FEB73196ADB7BEB711960C938DE044
:10B0600097E0928381838DE090E0948383830E94B4
:10B07000C2200F900F900F900F900F90802F6EEFC7
:10B0800076E00E941C210E94906CEDB7FEB73797C6
:10B090000FB6F894FEBF0FBEEDBF3196ADB7BEB789
:10B0A00011960C9322EF36E03283218363837483FD
:10B0B000858396830E94C220EDB7FEB737960FB600
:10B0C000F894FEBF0FBEEDBF802F6AEE76E00E94BF
:10B0D0001C218FE197E5602F0E94073B802F0E9483
:10B0E000B757802F6DED76E00E941C21802F0E94C3
:10B0F000E255802F61ED76E00E941C21802F0E9496
:10B100007956802F67EC76E00E941C21C0E0D0E0E9
:10B11000EE24FF2432ECA32E36E0B32EC7010E94AA
:10B12000508D182F00D000D00F92EDB7FEB731969A
:10B13000ADB7BEB711960C93B282A182D483C383FC
:10B140000E94C2200F900F900F900F900F9011301F
:10B1500019F06BEB76E002C06FEB76E0802F0E9477
:10B160001C21802F6DE00E9442202196E8E0F0E053
:10B17000EE0EFF1ECF3FD10589F6802F61EB76E002
:10B180000E941C21D6014C914170802F67EA76E025
:10B190000E94E54CF60140814470802F69E976E019
:10B1A0000E94E54CD6014C914870802F6EE876E005
:10B1B0000E94E54C00D000D00F92EDB7FEB731965B
:10B1C000ADB7BEB711960C9380E896E09283818369
:10B1D000D60116968C91838314820E94C220EDB70B
:10B1E000FEB73196ADB7BEB711960C9381E796E0E6
:10B1F00092838183D60118968C91838314820E9456
:10B20000C220EDB7FEB73196ADB7BEB711960C931D
:10B2100082E696E092838183D6011B968C9122E38D
:10B22000829FC0011124948383830E94C220EDB7C2
:10B23000FEB73196ADB7BEB711960C9383E596E095
:10B2400092838183D6011C968C9124E6829FC00153
:10B250001124948383830E94C2200F900F900F903B
:10B260000F900F90F60181810E94D61400D000D07B
:10B270000F92EDB7FEB73196ADB7BEB711960C93EE
:10B2800026E436E032832183948383830E94C220A4
:10B290000F900F900F900F900F90802F60E476E04A
:10B2A0000E941C2181E0DF91CF911F910F91FF90AF
:10B2B000EF90DF90CF90BF90AF9008951F93182F1D
:10B2C0000E94B757812F62E877E00E941C2181E03D
:10B2D0001F9108951F93182F1F7701F11150862F8A
:10B2E0000E94253E8B3141F08C3171F08E30B1F4EB
:10B2F000812F90E008960DC083E0189FC0011124B3
:10B300000B966EE070E007C0812F90E0880F991FC8
:10B31000079669E070E00E9487A8162F812F1F9181
:10B3200008951F93182F1F7711F480E01DC0862FFA
:10B330000E94253E8B3151F08C3171F08E3091F4AA
:10B34000E12FF0E0E25CF64F84910EC0E12FF0E0D7
:10B35000E35BF64F849108C0E12FF0E0E759F64F28
:10B36000849102C0812F8F5F1F910895EF92FF9209
:10B370000F931F93CF93DF93182F882319F0E0E4E6
:10B38000FE2E02C070E2F72EC5E7D9E000E0EF2CF8
:10B39000E09430C069858F2D862351F188850E9405
:10B3A0009159682F812F0E9442202C813D814E812E
:10B3B0005F815695479537952795812F622F0E947B
:10B3C0004220812F68810E94422069816F738C81A5
:10B3D00080FD6064888587FD6068812F0E9442201F
:10B3E00068856F77812F0E94422089858E21898709
:10B3F0000F5F2B968091350C081760F280E8DF9183
:10B40000CF911F910F91FF90EF9008950E94CD3C36
:10B4100081E00895FF920F931F93CF93DF93042F42
:10B42000442309F441C0809184048823E9F1C09148
:10B430007604D09177042097B9F180E4C030D80722
:10B4400098F511E0BFE0FB2E2DC01031C0F4812F24
:10B4500090E0FC01A4E0EE0FFF1FAA95E1F7E81BC6
:10B46000F90BEA58FB4F8685882349F0608171818A
:10B470006115710531F080E46030780710F060E00C
:10B4800070E01F9DF0011124E858FB4F01C0319678
:10B490008081882319F08132D1F70DC0CE010E943E
:10B4A0007A3C1F5F101788F281E0DF91CF911F91E6
:10B4B0000F91FF9008957068F1CF0E94553B03C033
:10B4C00080E00E94858480E00E940382BC01009796
:10B4D000B9F703C083E00E94858483E00E94038261
:10B4E000BC010097B9F703C082E00E94858482E026
:10B4F0000E940382BC010097B9F781E008951F9371
:10B50000182F60E02FEF3FE30E94C14C009769F1D4
:10B510000E94B838FC01009721F4812F69E279E09C
:10B5200022C0818590E0837090708130910581F018
:10B53000823091051CF4892B39F017C082309105B7
:10B5400059F0039791F40CC0812F66E279E00BC0AB
:10B55000812F69E179E007C0812F6CE079E003C0B9
:10B56000812F68E079E00E941C2181E01F910895FD
:10B570000F931F93CF93DF93182FFB01042F92811A
:10B5800080E0218130E0282B392BC90101978F5FA2
:10B590009F4338F0812F62E00E944220C0E0D0E05B
:10B5A00015C0002321F0C9010E94B33C03C0C901AA
:10B5B0000E94B838EC01009749F4002319F0812F5C
:10B5C0006BE002C0812F6AE00E944220CE01DF9131
:10B5D000CF911F910F9108951F93CF93DF93182F51
:10B5E00041E00E94B85AEC01009711F1812F60E010
:10B5F0000E9442202C813D814E815F8191E15695D0
:10B600004795379527959A95D1F7812F622F0E94FC
:10B6100042202C813D814E815F8189E1569547957D
:10B62000379527958A95D1F7812F622F0E94422066
:10B630008FEFDF91CF911F9108951F93CF93DF93E9
:10B64000182F41E00E94B85AEC01009799F0812F21
:10B6500060E00E9442202C813D814E815F8169E043
:10B6600056954795379527956A95D1F7812F622F83
:10B670000E9442208FEFDF91CF911F9108951F9379
:10B68000CF93DF93182F41E00E94B85AEC01009746
:10B6900081F0812F60E00E9442202C813D814E810B
:10B6A0005F815695479537952795812F622F0E9488
:10B6B00042208FEFDF91CF911F9108951F93CF9379
:10B6C000DF93182F41E00E94B85AEC01009741F136
:10B6D000812F60E00E944220888569850E949159EF
:10B6E000682F812F0E9442208C819D81AE81BF8175
:10B6F0009C01AD015695479537952795622F6F7040
:10B7000081709070892B09F06061888587FD606287
:10B71000812F0E94422068856F77812F0E944220EE
:10B720008FEFDF91CF911F910895CF93DF93EB01BE
:10B7300041E00E94B85AFC01009711F48FEF2DC030
:10B740008B81813069F18130E0F0823019F08330F3
:10B7500019F50AC022E025C06B3111F4246015C030
:10B760006C31D1F4286011C06C816E3011F423E08B
:10B770000CC06C3111F427E008C06E3769F42BE07F
:10B7800004C08C818E3741F420E080819181622F4A
:10B790000E94043E80E001C082E0DF91CF910895D5
:10B7A00021E06C816E30C1F6F0CF1F93CF93DF9311
:10B7B000182FEB016115710559F18F3F51F113708D
:10B7C000CB010E94C9A98F3708F08EE7133018F417
:10B7D000113020F41BC01330E1F40DC08B3199F40B
:10B7E000CE0162E470E00E942EAA009711F018606A
:10B7F00010C014600EC08C3111F417E00AC08E37EF
:10B8000011F41BE006C08E3019F403C08E3709F026
:10B810001FEF812FDF91CF911F9108950F931F93F9
:10B82000CF93DF93082F442301F180918404882370
:10B83000E1F0C0917604D09177042097B1F080E4D4
:10B84000C030D807E8F111C08091A204882369F0C4
:10B8500086E994E00E94104B8F3F39F067E874E06E
:10B860000E94D55B182F8F3F29F4802F62E00E9441
:10B87000584C21C0CE010E94B838892B21F0CE014E
:10B88000612F0E94043ECE01612F0E948C3DCE01AB
:10B890000E94AE85BC018091B104882341F0CB01A8
:10B8A000BE01412F25EA34E00E94718603C080E08A
:10B8B0000E94858481E0DF91CF911F910F910895BF
:10B8C00080919304882309F0BFCFCFCF1F93CF93EC
:10B8D000DF93182F442361F180918404882341F180
:10B8E000C0917604D0917704209711F180E4C030A4
:10B8F000D80748F11DC0812F6BE00E94584C1FC033
:10B90000618580919304882339F087E894E00E9450
:10B91000104B682F8F3F61F08091A204882359F06B
:10B92000862F66E974E00E94D55B682F8F3F19F47B
:10B93000812F62E0E2CFCE010E94043E81E0DF91E0
:10B94000CF911F910895CE010E94B33CFC01009756
:10B95000B9F6D1CFEF92FF921F93CF93DF93182FB9
:10B96000442351F180918404882331F1C0917604FD
:10B97000D0917704C038D105F8F080E4C030D80702
:10B98000D8F47E016F2D606C80E190E00E94B37D61
:10B9900099233CF081E190E06C2F0E94B37D97FFEA
:10B9A00003C0812F67E00DC08CE190E065E041E0CD
:10B9B0000E94C97D97FF03C0812F61E002C0812FE3
:10B9C00060E00E94A74ADF91CF911F91FF90EF9016
:10B9D00008950F931F93CF93DF93182F80E190E08A
:10B9E0000E94A97D97FD10C0082F805C883228F046
:10B9F000812F61E00E94A74A32C081E190E00E945D
:10BA0000A97DEC0197FF03C0812F67E0F3CF8CE1A4
:10BA100090E065E041E00E94C97D97FDE9CF00D04C
:10BA200000D00F92EDB7FEB73196ADB7BEB7119605
:10BA30001C9386ED97E092838183802F90E08F7333
:10BA40009070982F88278C0F911D948383830E9478
:10BA5000C22081E00F900F900F900F900F90DF9118
:10BA6000CF911F910F9108951F93182FFB01809183
:10BA70009304882309F461C0442309F45EC08091D3
:10BA80008404882309F459C0209176043091770406
:10BA90002115310509F451C084E02130380708F43C
:10BAA0005AC04BC060918504709186046F3F710548
:10BAB00019F010F060E070E083818434B1F08534D7
:10BAC0001CF48234D1F516C0803551F08235A9F5C9
:10BAD0002930310590F5822F81500E94927D30C02F
:10BAE000C90101970E947C7D2BC0C90101970E946A
:10BAF000B37D26C0423038F0609185047091860491
:10BB00006830710510F06FEF70E06F3FB1F04330B7
:10BB100058F08091A204882339F040919404509108
:10BB200095044230510510F04FEF50E04F3F29F09F
:10BB3000C90101970E94C97D03C0812F61E007C040
:10BB4000892B19F0812F67E002C0812F60E00E94ED
:10BB5000A74A1F910895423008F0A4CFABCFFF92BF
:10BB60000F931F93CF93DF93082FFB01442311F111
:10BB7000809184048823F1F0809176049091770479
:10BB80000097C1F024E08130920708F459C012C038
:10BB90008930910578F481500E94877D07C0019714
:10BBA0000E94727D03C001970E94A97DEC0197FF5E
:10BBB00009C003C0802F61E002C0802F67E00E94AF
:10BBC000A74A38C08DB79EB707970FB6F8949EBFA7
:10BBD0000FBE8DBFEDB7FEB73196ADB7BEB71196AC
:10BBE0000C9389ED97E092838183D483C383D683BA
:10BBF000C5830E94C220FC2E8DB79EB707960FB654
:10BC0000F8949EBF0FBE8DBF802F65E20E94422038
:10BC100010E8C0E0D0E0812F8F2111F460E301C073
:10BC200061E3802F0E94422016952196C830D105ED
:10BC300091F781E0DF91CF911F910F91FF900895CF
:10BC40006381643409F4AFCF653424F4623409F0BD
:10BC5000B1CFA9CF603509F4A2CF623509F0AACFE0
:10BC600097CF1F93182F442319F5813031F481E0C9
:10BC700066E478E00E941C211DC00E94041500D0DB
:10BC800000D00F92EDB7FEB73196ADB7BEB71196A3
:10BC90001C9323E438E032832183948383830E94BE
:10BCA000C22081E00F900F900F900F900F900FC067
:10BCB000813011F481E00BC060E478E00E941C2127
:10BCC00080917604909177040E94981480E01F91EF
:10BCD0000895EF92FF920F931F93CF93DF93082F56
:10BCE000442371F080918404882351F020917604DC
:10BCF000309177042115310529F02533310510F0F5
:10BD000020E030E0122F2223D9F100D000D00F9292
:10BD1000EDB7FEB73196ADB7BEB711960C9382E57D
:10BD200098E092838183238314820E94C2200F9023
:10BD30000F900F900F900F90812F8150602F0E94D5
:10BD4000AB807C01C0E0D1E010E00BC0183019F0EE
:10BD5000CC0FDD1F06C0802F60E20E944220C1E0B0
:10BD6000D0E0CE018E219F21892B19F0802F61E335
:10BD700002C0802F60E30E9442201F5F103131F724
:10BD800081E0DF91CF911F910F91FF90EF90089587
:10BD9000FF920F931F93F82EFB0181818150843312
:10BDA00010F082E011C06F2D0E94AB808C018F2DAE
:10BDB00060E00E9442208F2D612F0E9442208F2D33
:10BDC000602F0E9442208FEF1F910F91FF900895E6
:10BDD0001F93182F4423A9F08091470D282F30E09E
:10BDE0002170307080918404882341F08091760422
:10BDF000909177048230910508F49C01822F0E9473
:10BE0000B68000D000D00F92EDB7FEB73196ADB737
:10BE1000BEB711961C9385E798E092838183809149
:10BE2000470D90E081709070948383830E94C220BC
:10BE30000F900F900F900F900F9081E01F91089539
:10BE4000CF92DF92EF92FF920F931F93CF93DF93E6
:10BE5000D82E8B0121E0281708F45AC0FB018281FB
:10BE600090E087709070D82FCC27818190E0C82B0C
:10BE7000D92B2197F7E0C83FDF0710F082E049C0D7
:10BE80000E946A12982F8250823020F0973011F071
:10BE900086E03FC07E01EE0CFF1CF801628167FD69
:10BEA00004C081E090E0E82AF92A88E5D89EE00104
:10BEB0001124CA53DC4F862F90E016E096958795A3
:10BEC0001A95E1F7CC24C394C8228E010B5A1F4F58
:10BED000F80180819181FFEF8F3F9F0749F060E07B
:10BEE0004D2D0E94D28F8FEF9FEFF80191838083B9
:10BEF000C7016C2D4D2D0E94D28F882311F489E04B
:10BF000008C0CC2029F0FE01EB5AFF4FF182E082FD
:10BF100080E0DF91CF911F910F91FF90EF90DF9024
:10BF2000CF9008950F931F93CF93DF93082FFB01BA
:10BF3000828190E087709070D82FCC27818190E02B
:10BF4000C82BD92B219787E0C83FD80710F082E093
:10BF50001BC0CE010E94228D873621F0873411F05C
:10BF600010E001C014E0CE01880F991F0E94508D8F
:10BF7000039709F41160802F60E00E944220802F17
:10BF8000612F0E9442208FEFDF91CF911F910F917F
:10BF90000895AF92BF92DF92EF92FF920F931F939B
:10BFA000CF93DF93D82E142F0E946A12882319F49E
:10BFB0008D2D66E061C08D2D60E0412F28EF37E0C8
:10BFC0000E94C14C5C01009709F49CC021E02D1532
:10BFD00008F498C0123008F459C088E5D89E700162
:10BFE000112486EC93E0E80EF91EE701CB5ADF4FEF
:10BFF00088819981AFEF8F3F9A0741F060E04D2D26
:10C000000E94D28F8FEF9FEF99838883809187045E
:10C01000873411F490E012C0823511F491E00EC023
:10C0200080919304882339F080918504909186044F
:10C030008230910510F082E090E0982F123059F094
:10C040008091A204882339F0009194041091950402
:10C050000230110510F000E010E0E5012197CC0F4F
:10C06000DD1FC90FD11DCE01602F4D2D0E94D28F33
:10C07000882329F48D2D69E00E94584C44C0002388
:10C0800029F0F701EB5AFF4FD183C083C501019717
:10C090000E94228D082F112707FD1095C8010E94CC
:10C0A000FFA97C01C8010E94E7A92DB73EB729501E
:10C0B00030400FB6F8943EBF0FBE2DBFEDB7FEB7B0
:10C0C0003196ADB7BEB71196DC9229ED38E03283D8
:10C0D0002183B482A382F682E58220E030E0892BBE
:10C0E00011F021E030E0308727830E94C22081E0F8
:10C0F0002DB73EB7275F3F4F0FB6F8943EBF0FBE38
:10C100002DBF01C081E0DF91CF911F910F91FF9072
:10C11000EF90DF90BF90AF9008956F927F928F92D3
:10C120009F92AF92BF92CF92DF92EF92FF920F93C6
:10C130001F93DF93CF93CDB7DEB760970FB6F89418
:10C14000DEBF0FBECDBFC82ED42E60E02FEF3FE381
:10C150000E94C14C7C01009709F4DFC021E0D21697
:10C1600009F063C00E942F889A83898300D000D091
:10C170000F92EDB7FEB73196ADB7BEB71196CC9220
:10C1800087EF98E092838183F482E3820E94C22049
:10C190000F900F900F900F900F903E010894611C2C
:10C1A000711C05E0802E912C8C0E9D1E10EFA12E8F
:10C1B00018E0B12EB1E1EB2EF12CEC0EFD1E30C0DB
:10C1C00080E1B3010E9479828401F8019181992371
:10C1D00011F12DB73EB7275030400FB6F8943EBF4F
:10C1E0000FBE2DBFEDB7FEB73196ADB7BEB71196F6
:10C1F000CC92B282A182D8018C91838314829583E0
:10C2000016820E94C220EDB7FEB737960FB6F8949B
:10C21000FEBF0FBEEDBF0E5F1F4F0E151F05A9F627
:10C2200089819A81892B61F678C0F2E0DF1619F0D6
:10C2300001E012E070C080919304882341F00091E6
:10C240008504109186040F3F110519F010F000E0ED
:10C2500010E0C701602F0E94C2882DB73EB7295059
:10C2600030400FB6F8943EBF0FBE2DBFEDB7FEB7FE
:10C270003196ADB7BEB71196CC9224EE38E032833A
:10C280002183F482E38205831682878310860E94CD
:10C29000C220EDB7FEB739960FB6F894FEBF0FBEB9
:10C2A000EDBF3BC00031A8F4802F90E0FC01A4E07A
:10C2B000EE0FFF1FAA95E1F7E81BF90BEA58FB4FB9
:10C2C0008685882331F0608171816F3F710519F097
:10C2D00010F060E070E01031B8F41D15A8F4812F63
:10C2E00090E0FC0174E0EE0FFF1F7A95E1F7E81B88
:10C2F000F90BEA58FB4F8685882331F04081518144
:10C300004F3F510519F010F040E050E0C7010E9486
:10C3100052890E5F1E5F0D1528F281E060960FB600
:10C32000F894DEBF0FBECDBFCF91DF911F910F916B
:10C33000FF90EF90DF90CF90BF90AF909F908F9045
:10C340007F906F900895EF92FF920F931F93CF937A
:10C35000DF93182F042F60E02FEF3FE30E94C14CC2
:10C36000EC01009709F45BC00E94B8387C0100978B
:10C3700071F4023018F4812F6AE011C0CE010E94DE
:10C38000B33C7C01009729F4812F6BE008C0023098
:10C39000F0F00E943322882329F0812F68E00E9468
:10C3A000584C3EC0D70114966D917C911597802F03
:10C3B00040E052E021E008E00E94454ABC01CE0185
:10C3C000412F0E941B3DCE0160E00E94EA380E948E
:10C3D0006A12882321F4812F62E40E94584C00D015
:10C3E00000D00F92EDB7FEB73196ADB7BEB711963C
:10C3F0001C938DEF98E092838183D483C3830E9442
:10C40000C2200F900F900F900F900F90F701648152
:10C410007581812F40E052E028E00E94004D81E0CC
:10C42000DF91CF911F910F91FF90EF900895EF92C0
:10C43000FF920F931F93CF93DF93182F042F60E089
:10C440002FEF3FE30E94C14CEC01009709F45BC061
:10C450000E94B8387C01009771F4023018F4812FE3
:10C460006AE011C0CE010E94B33C7C01009729F420
:10C47000812F6BE008C00230F0F00E943322882345
:10C4800029F0812F68E00E94584C3EC0D7011496D5
:10C490006D917C911597802F42E050E021E008E0FB
:10C4A0000E94454ABC01CE01412F0E941B3DCE0196
:10C4B00060E00E94EA380E946A12882321F4812FEA
:10C4C00062E40E94584C00D000D00F92EDB7FEB746
:10C4D0003196ADB7BEB711961C9383E099E0928375
:10C4E0008183D483C3830E94C2200F900F900F904A
:10C4F0000F900F90F70164817581812F42E050E029
:10C5000028E00E94004D81E0DF91CF911F910F91B3
:10C51000FF90EF900895DF92EF92FF920F931F9399
:10C52000CF93DF93D82E142F60E02FEF3FE30E94CC
:10C53000C14C7C01009709F4E8C00E94B838EC01B6
:10C54000009771F4123018F48D2D6AE012C0C70103
:10C550000E94B33CEC01009731F48D2D6BE009C0D3
:10C56000123008F481C00E943322882329F08D2DD7
:10C5700068E00E94584CCAC08C819D81AE81BF8109
:10C58000BC016E7FAC0141705070123059F0809147
:10C59000A204882339F0209194043091950422302C
:10C5A000310508F09A01232B09F06160812F42E0E8
:10C5B00050E024E004E00E94454ABC01C7014D2D33
:10C5C0000E941B3D888569850E949159482F809162
:10C5D0009304882339F02091850430918604203813
:10C5E000310508F0242F8091A504863411F411E060
:10C5F0001AC0823511F410E016C040E050E0888582
:10C6000087FF02C041E050E0143058F08091B1043F
:10C61000882339F08091A3049091A404823091057D
:10C6200008F0CA01182F213029F4C7010E94B7363B
:10C6300000E005C0822F69850E946A59082F1111F8
:10C6400000686885802F862787FF05C06078C7014E
:10C650004D2D0E94543DC701602F4D2D0E94543D29
:10C66000C70160E00E94EA380E946A12823019F421
:10C670008D2D61E406C00E946A12833021F08D2D59
:10C6800062E40E94584C888569850E949159682F00
:10C690008C8180FD03C040E350E002C041E350E0E4
:10C6A000888587FD03C022E730E002C026E630E03F
:10C6B0008DB79EB70B970FB6F8949EBF0FBE8DBF78
:10C6C000EDB7FEB73196ADB7BEB71196DC9280E3F9
:10C6D00099E092838183F482E38265831682508796
:10C6E0004783328721870E94C2208DB79EB70B9661
:10C6F0000FB6F8949EBF0FBE8DBF6C817D818D2DCE
:10C7000042E050E024E00E94004D81E0DF91CF91B3
:10C710001F910F91FF90EF90DF900895AF92BF921D
:10C72000CF92DF92EF92FF920F931F93CF93DF93FD
:10C73000C82E882349F047E7A42E4CE0B42E3EE4EF
:10C74000E32E3DE0F32E08C02FEDA22E2CE0B22EFA
:10C7500098E4E92E9DE0F92EDD2433C0F8940D2DE8
:10C7600010E0C701B8010E948392882341F1F801CB
:10C77000EE0FFF1FD501AE0FBF1FEC5AF24FCD9148
:10C78000DC91119780819181C82BD92B1D921C922D
:10C7900080819181C817D90721F4C701B8010E948F
:10C7A0006D9278946D2D6F5F8C2D0E9442208C2DA0
:10C7B0006D2F0E9442208C2D6C2F0E944220789475
:10C7C000D3940E947C6CFC018085D81638F28C2DA5
:10C7D00060E00E9442208FEFDF91CF911F910F9177
:10C7E000FF90EF90DF90CF90BF90AF900895CF92E1
:10C7F000DF92EF92FF920F931F93DF93CF93CDB70A
:10C80000DEB7C254D0400FB6F894DEBF0FBECDBF26
:10C81000C82EDD247E010894E11CF11C8C2D0E94A1
:10C820003B918C018FEF0F3F180719F1C8010E944F
:10C83000228D282FC8010196F7018083892F8770E8
:10C840008183273411F0273629F48068F70181832A
:10C85000273411F0223521F4F7018181806481832E
:10C86000D394F0E2DF1629F082E090E0E80EF91EA2
:10C87000D5CF8C2D6D2D0E944220ED2CFF24EE0C87
:10C88000FF1C8E010F5F1F4FD02E06C0F801619173
:10C890008F018C2D0E944220802F8D1990E08E15E3
:10C8A0009F05A4F38FEFCE5BDF4F0FB6F894DEBF8A
:10C8B0000FBECDBFCF91DF911F910F91FF90EF90F1
:10C8C000DF90CF9008951F93CF93DF93182F0E948E
:10C8D000E391692F629566956695617095FD646038
:10C8E00080FD686097FD6062EC01CE7FDF7120976C
:10C8F00009F06068812F0E9442202097A1F0CE01AC
:10C9000096958795682F6170C2FD6064C97F2097F6
:10C9100009F06068812F0E944220CD2B21F0812FE9
:10C9200060E00E9442208FEFDF91CF911F91089528
:10C93000CF92DF92FF920F931F93DF93CF93CDB7E8
:10C94000DEB760970FB6F894DEBF0FBECDBFF82EEE
:10C9500063E00E9442208F2D62E00E9442208F2DD2
:10C9600062E00E9442208F2D63E00E9442208F2DC2
:10C9700064E00E9442200E94906C2DB73EB7285080
:10C9800030400FB6F8943EBF0FBE2DBFEDB7FEB7D7
:10C9900031968E010F5F1F4FADB7BEB712961C9335
:10C9A0000E93119723E73AE03383228364837583E0
:10C9B000868397830E9460AAEDB7FEB738960FB6BC
:10C9C000F894FEBF0FBEEDBF79E0C72ED12CCC0E80
:10C9D000DD1ED8016C916295607F11968C91805319
:10C9E000682B0E5F1F4F8F2D0E9442200C151D05D6
:10C9F00081F780E060960FB6F894DEBF0FBECDBF22
:10CA0000CF91DF911F910F91FF90DF90CF9008950C
:10CA10000E94C08080E008950F931F93CF93DF930F
:10CA20008B01823030F5FB01828190E0877090703D
:10CA3000D82FCC27818190E0C82BD92B2197F7E004
:10CA4000C83FDF0710F082E015C00E946A12982FDD
:10CA50008250823020F0973011F086E00BC0F80150
:10CA60006281669566956695CE01880F991F0E9432
:10CA7000953480E0DF91CF911F910F910895CF936E
:10CA8000DF93EB0140E00E94B85AFC01009711F4DB
:10CA90008FEF1CC081858370833011F082E016C057
:10CAA0004B816C8170E07695762F66277795679538
:10CAB000842F90E08F779070682B792B441F442748
:10CAC000441F808191810E940A3880E0DF91CF91DC
:10CAD0000895DF92EF92FF920F931F93CF93DF930E
:10CAE000D82EEB0141E00E94B85A7C01009711F466
:10CAF0008FEF5DC0FC0181850E942F3EF70104810C
:10CB00001581268137814B819C818D3100F1217007
:10CB1000307050E060E070E0F1E1440F551F661F97
:10CB2000771FFA95D1F7892F90E0A0E0B0E0E9E116
:10CB3000880F991FAA1FBB1FEA95D1F7482B592BC5
:10CB40006A2B7B2B402B512B622B732B23C0217024
:10CB5000307E50E060E070E081E1440F551F661FB9
:10CB6000771F8A95D1F7402B512B622B732B892F7E
:10CB700090E0A0E0B0E08F709070A070B07019E10C
:10CB8000880F991FAA1FBB1F1A95D1F7482B592B45
:10CB90006A2B7B2BF701808191812D2D0E94E23C35
:10CBA000F7018081918161E00E94EA3880E0DF91A5
:10CBB000CF911F910F91FF90EF90DF900895FF921A
:10CBC0000F931F93CF93DF93F82E8B0141E00E94C8
:10CBD000B85AEC01009711F48FEF21C08C819D8130
:10CBE000AE81BF819170AE7FF801438150E060E07B
:10CBF00070E019E0440F551F661F771F1A95D1F793
:10CC0000482B592B6A2B7B2B888199812F2D0E94D1
:10CC1000E23C8881998160E00E94EA3880E0DF91FF
:10CC2000CF911F910F91FF900895FF920F931F9343
:10CC3000CF93DF93F82E8B0141E00E94B85AEC01AC
:10CC4000009711F48FEF1EC08C819D81AE81BF8152
:10CC500081709E7FF801438150E060E070E0440FF6
:10CC6000551F661F771F482B592B6A2B7B2B8881FA
:10CC700099812F2D0E94E23C8881998160E00E9479
:10CC8000EA3880E0DF91CF911F910F91FF900895D6
:10CC9000CF92DF92EF92FF920F931F93CF93DF9388
:10CCA000C82E8B01F42E41E00E94B85AEC01009787
:10CCB00011F48FEF78C00E943322882311F088E0AE
:10CCC00072C0D8011396DC90FF2071F0B1E0DB1642
:10CCD00031F4888199810E94B736DD2405C08D2DFD
:10CCE00069850E946A59D82EF8016481262F30E0A8
:10CCF00065FF02C0F0E8DF2AEC80FD800E811F8115
:10CD00008EEF9FEFAFEFBFEFE822F9220A231B233C
:10CD100024FF08C081E090E0A0E0B0E0E82AF92A12
:10CD20000A2B1B2B67FF15C081EE9FEFAFEFBFEF04
:10CD3000E822F9220A231B232F703070220F331FA1
:10CD4000C901AA2797FDA095BA2FE82AF92A0A2B2C
:10CD50001B2B68858D2D862787FF06C0607888810C
:10CD600099814C2D0E94543D888199816D2D4C2DC7
:10CD70000E94543D88819981B801A7012C2D0E9401
:10CD8000E23C8881998160E00E94EA380E946A1240
:10CD9000833041F0873031F0823011F082E403C0FB
:10CDA00081E401C080E0DF91CF911F910F91FF904E
:10CDB000EF90DF90CF90089540E00E94486608957C
:10CDC00041E00E94486608951F93CF93DF93182F88
:10CDD000EB010E946A12833011F082E43EC0812F81
:10CDE000BE0141E00E94B85AFC01009711F48FEF98
:10CDF00034C0118613821282148215821682178221
:10CE000010866C8170E080E090E0982F872F762F5D
:10CE100066272D8130E040E050E0A901332722272A
:10CE2000622B732B842B952B2B8130E040E050E05C
:10CE3000622B732B842B952B2E8130E040E050E049
:10CE4000522F442733272227622B732B842B952BB9
:10CE5000408151810E94D03280E0DF91CF911F91BB
:10CE600008951F93CF93DF93182F41E00E94B85A83
:10CE7000EC01009701F1812F60E00E94422069855A
:10CE80006370812F0E94422089850E943138892B4E
:10CE900019F0812F6CE105C089850E94253E682F1D
:10CEA000812F0E944220812F6FEF0E944220812F0C
:10CEB0006FEF0E9442208FEFDF91CF911F91089575
:10CEC000CF92DF92EF92FF920F931F93CF93DF9356
:10CED000D82EEB01C42E21E0281708F4F9C02881D0
:10CEE0003FE1F32EF222422F50E0CA01807E907083
:10CEF0008034910509F49AC08134910534F4009787
:10CF000089F0809709F0E4C050C08038910509F499
:10CF1000B5C0803C910509F4C7C08036910509F081
:10CF2000D7C0A4C081E08C1508F0D4C00981802F3F
:10CF300090E00E94B33CFC01009709F4C9C06481F1
:10CF40007581F4FE03C0EB01C16002C0EB01CE7F2E
:10CF50001F2D1F70F0841F3021F46F2D60956078B5
:10CF600017C08185112389F00E94253E8C3139F04C
:10CF70008E3739F08B3149F4110F115006C0110F63
:10CF800004C089E0189F102D11246F2D6078612B4B
:10CF9000802F90E04D2D0E94543D802F90E0BE01E7
:10CFA0004D2D0E941B3D802F5CC088E5D89E7001EE
:10CFB0001124E6ECF3E0EE0EFF1E237F28838701A9
:10CFC0000B5A1F4FF80180819181FFEF8F3F9F0720
:10CFD00049F060E04D2D0E94D28F8FEF9FEFF80156
:10CFE000918380832881203209F472C0233209F4AE
:10CFF0006FC0F1E0FC1508F06DC06981213231F499
:10D00000C62FD0E02197CC0FDD1F05C0C62FD0E082
:10D01000CC0FDD1F2197CE0161E04D2D0E94D28FF4
:10D02000F701EB5AFF4FD183C08352C021E02C158A
:10D0300008F050C01981812F90E00E943A3D9B0179
:10D04000AC01217E8F2D90E08F709070880F991F1A
:10D05000282B392B812F90E0B9014D2D0E941B3DCB
:10D06000812F90E060E00E94EA3832C020FF02C0C9
:10D0700080E001C083E00E9485122AC0FF2011F4E5
:10D0800080E015C000E0802F6D2D0E949280182F47
:10D090008D2D692F0E9442208D2D612F0E944220EC
:10D0A0000F5F0F1580F314C0FF2021F481E00E9470
:10D0B000B6800EC08F2D81506D2D0E949280182F4A
:10D0C0008D2D692F0E9442208D2D612F0E944220BC
:10D0D00081E001C080E0DF91CF911F910F91FF901F
:10D0E000EF90DF90CF900895BF92CF92DF92EF92B2
:10D0F000FF920F931F93CF93DF93B82E81E08B1590
:10D1000008F441C388E5B89E60011124E6ECF3E021
:10D11000CE0EDF1EE601C95ADF4F888187FD33C37B
:10D120008B2D0E942E208C01FFEF8F3F9F0709F46B
:10D130002AC388818068888344E5E42EF12CEC0CB6
:10D14000FD1CF70180818823F1F0F6016081718177
:10D150008281938168537F4F8F4F9F4F0E942F1979
:10D16000882389F0F7018081882349F0888180FD38
:10D170000AC0F6018481883531F0883721F0F60144
:10D18000EC5AFF4F10828091DA079091DB07A09153
:10D19000DC07B091DD07F60180839183A283B3831E
:10D1A000EC5AFF4F8081803508F01082C6010E9442
:10D1B000214A8823B1F00830110551F4F601EC5AE8
:10D1C000FF4F8081882309F4D0C281508083CDC273
:10D1D0000115110509F4C9C20D30110511F400E063
:10D1E00010E0F601EC5AFF4F8081D601A80FB11D67
:10D1F00014960C93F82EF394F082FF2091F0F60130
:10D20000E95AFF4F808190E0EC01C170D07080FD41
:10D21000B3C2F6018481883509F4AEC2883709F4B7
:10D22000ABC2B6016C5F7F4F8B2D4F2D0E946067A4
:10D23000882309F096C299C2012B09F096C2F60123
:10D24000EC5AFF4F108286010C5F1F4FF601E95A1E
:10D25000FF4F808180FD03C086010B5F1F4FF801E7
:10D260008081882309F44DC2C80164E275E043E07F
:10D2700050E00E9419AA892B59F4C5E8DAE4C801E4
:10D2800003960E944EAAC8010E943C4BF82E32C25F
:10D29000C8010E944EAAC8010E943C4BF82EC8014A
:10D2A00062E275E00E9407AA892B39F0C80160E2AA
:10D2B00075E00E9407AA892B19F4CDEFDAE41AC2AF
:10D2C000C8016DE175E00E9407AA892B19F4C7EF28
:10D2D000DAE410C2C8016AE175E00E9407AA892B4E
:10D2E00019F4C1EFDAE406C2C80167E175E00E94F3
:10D2F00007AA892B19F4CBEEDAE4FCC1C80165E179
:10D3000075E00E9407AA892B39F0C80160E175E039
:10D310000E9407AA892B19F4CAEED0E5EBC1C80117
:10D320006EE075E00E9407AA892B39F0C8016BE016
:10D3300075E00E9407AA892B19F4C6EDD0E5DAC181
:10D34000C80166E075E00E9407AA892B19F4C4E8B9
:10D35000D0E5D0C1C80164E075E00E9407AA892B1E
:10D3600019F4CBE8D2E6C6C1C80161E075E00E94BD
:10D3700007AA892B19F4CFE7DAE5BCC1C8016FEF22
:10D3800074E00E9407AA892B19F4C7E1D2E6B2C162
:10D39000C8016CEF74E00E9407AA892B19F4C3EA54
:10D3A000D1E6A8C1C80169EF74E00E9407AA892BE1
:10D3B00019F4CDE8D0E69EC1C80167EF74E00E9481
:10D3C00007AA892B19F4C9ECDFE594C1C80165EF00
:10D3D00074E00E9407AA892B19F4C6EAD0E58AC135
:10D3E000C80163EF74E00E9407AA892B19F4CFEA01
:10D3F000D5E580C1C80160EF74E00E9407AA892BBF
:10D4000019F4C7E2D4E576C1C8016DEE74E00E945C
:10D4100007AA892B19F4C8EEDEE56CC1C8016AEED3
:10D4200074E00E9407AA892B19F4C9E6DEE562C1FF
:10D43000C80167EE74E00E9407AA892B19F4CCEDAD
:10D44000D3E558C1C80164EE74E00E9407AA892B95
:10D4500019F4C3ECDCE64EC1C80162EE74E00E9430
:10D4600007AA892B19F4C1E3DEE544C1C8016FEDB9
:10D4700074E00E9407AA892B19F4C8E5D3E53AC1E4
:10D48000C8016CED74E00E9407AA892B19F4C4E965
:10D49000DDE430C1C80169ED74E00E9407AA892B60
:10D4A00019F4CBE4DDE426C1C80166ED74E00E9406
:10D4B00007AA892B39F0C80163ED74E00E9407AA1E
:10D4C000892B19F4C0EAD1E515C1C8016EEC74E0EE
:10D4D0000E9407AA892B51F1C80169EC74E00E94EF
:10D4E00007AA892B69F1C80164EC74E00E9407AABD
:10D4F000892BE1F0C8016FEB74E00E9407AA892B29
:10D50000F9F0C8016AEB74E00E9407AA892B71F058
:10D51000C80165EB74E00E9407AA892B89F0C80155
:10D5200060EB74E00E9407AA892B19F4CFEADDE5CD
:10D53000E1C0C8016BEA74E00E9407AA892B19F4C4
:10D54000C4E3DDE5D7C0C80166EA74E00E9407AA1B
:10D55000892B19F4C9EEDCE5CDC0C80161EA74E09D
:10D560000E9407AA892B19F4CAEADCE5C3C0C801E6
:10D570006EE974E00E9407AA892B19F4C6E6DCE57F
:10D58000B9C0C80166E974E00E9407AA892B19F4A2
:10D59000CEE5D9E5AFC0C8016FE874E00E9407AAE4
:10D5A000892B19F4CEE0DCE5A5C0C80166E874E07B
:10D5B0000E9407AA892B19F4CDE5DAE59BC0C801C2
:10D5C0006EE774E00E9407AA892B19F4CDE6D6E530
:10D5D00091C0C80167E774E00E9407AA892B19F47B
:10D5E000CAE0DAE587C0C8016EE674E00E9407AAC7
:10D5F000892B19F4C6E0DAE57DC0C80166E674E05F
:10D600000E9407AA892B19F4C3E1D7E573C0C801AA
:10D610006EE574E00E9407AA892B19F4C4E0D8E5EE
:10D6200069C0C80167E574E00E9407AA892B19F454
:10D63000C1E6D5E55FC0C80160E574E00E9407AAB5
:10D64000892B19F4CFECD4E555C0C8016CE474E023
:10D650000E9407AA892B19F4CEEAD2E54BC0C80173
:10D6600069E474E00E9407AA892B19F4CDE7D2E59A
:10D6700041C0C80165E474E00E9407AA892B19F42F
:10D68000C3E1D1E537C0C8016CE374E00E9407AA8A
:10D69000892B19F4CFE9D0E52DC0C80168E374E007
:10D6A0000E9407AA892B19F4C3E2D0E523C0C80160
:10D6B00065E374E00E9407AA892B19F4CBE9DFE443
:10D6C00019C0C80160E374E00E9407AA892B19F40D
:10D6D000CBE7DFE40FC0C8016BE274E00E9407AA49
:10D6E000892B19F4C2EEDDE405C08B2D61E00E94A8
:10D6F000584C05C08B2DB8014F2DFE01099588238C
:10D70000A1F18B2D68E274E00E941C212EC0CD2B6C
:10D7100031F0B6016C5F7F4FF601948106C0B6010F
:10D720006B5F7F4FFA94F6019581E4E0F1E012C05F
:10D73000891779F48181F816C0F00280F381E02D19
:10D74000309779F08B2D0995682F8F3F51F08B2DF5
:10D7500006C034968081882359F78B2D61E00E94A2
:10D760004220F601EC5AFF4F1082F601E95AFF4FB2
:10D7700080818F77808307C0C6010E94214A882359
:10D7800009F05ACDC4CFDF91CF911F910F91FF9037
:10D79000EF90DF90CF90BF9008956F5F7F4F42E092
:10D7A0000E9460678FEF08956F5F7F4F41E00E9496
:10D7B00060678FEF08958230C0F4282F30E088E54D
:10D7C00090E0289FF001299FF00D389FF00D112463
:10D7D000EA53FC4FEC5AFF4F1082339610828FEFC2
:10D7E0009FEF929382930E94919108951F93182F17
:10D7F000823118F029EF3EE031C00E947C6CFC01C0
:10D800002581223079F02330B9F0812F90E021304A
:10D81000E9F49C0154E0220F331F5A95E1F7275891
:10D82000354F1CC0212F30E044E0220F331F4A95B2
:10D83000E1F72756344F12C0212F30E094E0220F39
:10D84000331F9A95E1F72754334F08C09C0184E0B9
:10D85000220F331F8A95E1F72752324FC9011F91DA
:10D860000895882319F02EE43FE015C00E947C6CD7
:10D87000FC018581823039F0833041F0813049F4F8
:10D880002AE03FE008C02BE13FE005C02CE23FE08A
:10D8900002C02DE33FE0C90108951F93182F833282
:10D8A00018F02AEA38E125C00E947C6CFC018581D1
:10D8B000823059F0833081F08130A9F481E1189FE2
:10D8C00090011124225A304F14C081E1189F900119
:10D8D00011242F543E4E0DC081E1189F9001112458
:10D8E0002C5F3B4E06C081E1189F90011124295AFC
:10D8F000394EC9011F9108958EE695E008958091F3
:10D900006F0590E0089580917D05089580916E05E2
:10D91000089590916E05982309F091E0892F08955C
:10D920002CEF3FEF41E050E04BBFF90127913791D9
:10D93000479156915070B901CA0108958FEF9FEF3A
:10D94000A1E0B0E0ABBFFC018791823029F40799D8
:10D9500002C080E8089582E00895EEE8F5E0808155
:10D960009181892B29F08381882311F411821082FF
:10D970008381882311F081508383349685E0EE39CA
:10D98000F80769F708950E946B32F89488E181BD29
:10D990008BE081BDFFCF0E94B838DC010097C1F059
:10D9A000EEE8F5E0208131818D919C911197281747
:10D9B000390739F012968D919C91139728173907E2
:10D9C00011F411821082349685E0EE39F80751F790
:10D9D00008957F928F929F92AF92BF92CF92DF92E3
:10D9E000EF92FF920F931F93DF93CF9300D000D05D
:10D9F00000D0CDB7DEB7782E5B01042FFE01319643
:10DA000086E0DF011D928A95E9F7CF010E94E16F60
:10DA1000EEE8F5E014E088249924143029F480819C
:10DA20009181892B09F4182D808191818A159B059C
:10DA300009F0E5C0F401EE0FFF1FEE0FFF1FE257E4
:10DA4000FA4F88E08383F401EE0FFF1FEE0FFF1FF4
:10DA5000E057FA4F80818F5F8083833008F403C1E1
:10DA6000C5010E94B33C6C01009709F4FCC0BFEFF4
:10DA70007B16B1F5FC0144815581002319F0C501E5
:10DA8000BA0129C0C501D60118966C910E94B9440B
:10DA9000F6011185C5010E94AE85BC01812F0E944F
:10DAA0009844D60114962D913D914D915C91179714
:10DAB0009A0144275527C501B9010E94EE3EF6019F
:10DAC00082819381009749F00E94B33CFC016481FC
:10DAD0007581808191810E94DB3E0E944D3E82C013
:10DAE000DC0114962D913D914D915C911797002387
:10DAF00069F07E010894E11CF11CC70160E000E0C0
:10DB00000E940670872D68E0A7016AC000E0FC0152
:10DB100082819381892B09F001E07E010894E11C48
:10DB2000F11CC701D60118966C910E940670872DD2
:10DB300067E0A7010E94BE70F60181858F778B8315
:10DB400082819381892B41F4C5010E94AE85BC017D
:10DB5000CE0104960E94E16F0E94AC788823E1F325
:10DB6000872D69E08E010F5F1F4FA8010E94BE70D4
:10DB7000D60114964D915D916D917C911797C801D6
:10DB80000E94ED6F0E94AC788823E1F3872D6DE051
:10DB90005E010894A11CB11CA5010E94BE70F60193
:10DBA000828193810E94B8388C010097D9F0DC0102
:10DBB0006D917C91C5010E94E16FF801248135814E
:10DBC00046815781C50160E000E00E9406700E9416
:10DBD000AC788823E1F3872D68E0AE014F5F5F4F9B
:10DBE0000E94BE70880C991C880C991C8EE895E0E8
:10DBF000880E991ED4011D921C9281E035C00894B4
:10DC0000811C911C3496B4E08B16910409F005CF69
:10DC1000143041F48FEF66E0AE014F5F5F4F0E941A
:10DC2000BE7021C00E943F3E8A159B0519F40E94D8
:10DC3000B04007C08FEF65E0AE014F5F5F4F0E94BD
:10DC4000BE70E12FF0E0EE0FFF1FEE0FFF1FDF01B0
:10DC5000A257BA4F1196BC92AE92E057FA4F10827B
:10DC600088E013968C9380E026960FB6F894DEBF7A
:10DC70000FBECDBFCF91DF911F910F91FF90EF901D
:10DC8000DF90CF90BF90AF909F908F907F9008953E
:10DC90007F928F929F92AF92BF92CF92DF92EF923C
:10DCA000FF920F931F93DF93CF9300D000D000D04B
:10DCB000CDB7DEB7782E4B017A01CB010E94B33C81
:10DCC0005C01009709F452C0C7010E94B33C6C018B
:10DCD000009709F44BC0D50119968C910E94253EFE
:10DCE0008C01F60181850E94253E9801281B390B85
:10DCF000C90137FF03C0909581959F4F0297B4F0FB
:10DD00003FEF731621F481E00E94D63E2FC0FE0142
:10DD1000319686E0DF011D928A95E9F781E08983DB
:10DD2000872D61E2AF010E94BE7020C000E0872D08
:10DD3000B70141E00E94E96C882389F0F6018085F3
:10DD4000D50118969C91892787FF04C0E0E0F0E890
:10DD5000EE2AFF2AC401B7010E947A3C07C00E9444
:10DD6000AC788823E1F30F5F043109F726960FB6EC
:10DD7000F894DEBF0FBECDBFCF91DF911F910F9101
:10DD8000FF90EF90DF90CF90BF90AF909F908F90DB
:10DD90007F9008951F93CF93DF93EB016115710579
:10DDA00099F08F3F71F410E08FEFBE0140E00E94C8
:10DDB000E96C0E94AC788823E1F31F5F1A30A1F769
:10DDC00003C040E00E94E96CDF91CF911F9108955C
:10DDD000CF93DF93C0E0D0E0CE010E94F9ACFE010A
:10DDE000E259FA4F6081861719F0CE010E940BADFF
:10DDF000A8952196C032D10579F7DF91CF9108958A
:10DE0000982F909520916E05922390936E0582FF36
:10DE100002C00E94E9300E94E86E089590916E055C
:10DE2000982B90936E0582FF02C00E94E9300E94F9
:10DE3000E86E08951F93182F82FD136011FD116085
:10DE400010937D050E94E86E812F0E947B231F9115
:10DE500008951F93182F883008F017E080916F0500
:10DE6000181751F010936F050E94E86E812F68E03B
:10DE70004EE421E00E9401141F91089580937305E0
:10DE80000E94E86E089590917305973008F091E034
:10DE900080E1EEE6F5E0DF011D928A95E9F788E181
:10DEA000809372059093730597E090936F0584E1DA
:10DEB0008093740582E08093790582E380937A05EC
:10DEC0008CE080936E0590937D0583E090E00E9446
:10DED000D18D0E94E86E08950E946B3284E06EEB53
:10DEE00071E00E94292085E066EC71E00E94292003
:10DEF00082E89EE968EC70E00E94871E80E060E0A6
:10DF00000E94481F83E00E944D6CBC0182E00E9489
:10DF10001C210E94553B0E9488840E94436F0E94EE
:10DF2000C36C08958EE695E060E070E040E250E05A
:10DF30000E94E9AC80917005909171058F5F9F4FB1
:10DF400011F40E94436F80916F05883018F087E0CC
:10DF500080936F0580917B0590917C05885F974049
:10DF600020F010927C0510927B058091730587301C
:10DF700010F0109273058AEF9FEFA1E0B0E0ABBF05
:10DF8000FC019791892F81508E3F10F490936F0080
:10DF90000895682780E097E067FF03C0660F692750
:10DFA00001C0660F8F5F8830B9F7862F08952091E2
:10DFB000FD053091FE059093FE058093FD05C90196
:10DFC0000895FC01862F8F778083660F672F661F69
:10DFD000770B71956F7761830895FC01CB01AA27B8
:10DFE000BB278F77828327E176956795579547956D
:10DFF0002A95D1F7842F8F77838397E0769567955D
:10E00000579547959A95D1F7448308950F93FC014E
:10E01000862F8F778283DA01C9017AE0B695A795BA
:10E02000979587957A95D1F78F7366956074862B4F
:10E030008383DA01C90163E0B695A7959795879523
:10E040006A95D1F78F778483822F82958077858335
:10E0500040FF02C088608583002319F085818160BC
:10E0600085830F910895982FE82FF0E0E95CF34F36
:10E070008081882311F081E008958091F705981739
:10E08000B9F49923A9F09150992371F0292F2150C7
:10E09000E92FF0E0E95CF34F8081882311F4922F9F
:10E0A000F3CF9093F70502C01092F70580E0089532
:10E0B00080E00895CF92DF92EF92FF921F93CF936B
:10E0C000DF93782F162F7A01A8952091F205809181
:10E0D000F30530E090E001972817390709F445C0AF
:10E0E0008091F205873021F48091F3058823E9F1CE
:10E0F0009091F20589E0989FE0011124C655DA4F0E
:10E10000672F6068688380E00E94C96F1983612F60
:10E110000E94C96F982FE2E0CE2ED12CCC0EDD1ECE
:10E12000E60110E0E114F10431F0F70181917F0183
:10E130008F77888301C01882892F69910E94C96FE7
:10E14000982F1F5F163071F787FD9095F601968323
:10E150008091F2058F5F8093F2058091F2058830FF
:10E1600010F01092F20581E001C080E0DF91CF91C4
:10E170001F91FF90EF90DF90CF9008950F931F9322
:10E18000CF93DF93082F162FEA0102C00E9471126D
:10E19000802F612FAE010E945A708823B9F3DF915E
:10E1A000CF911F910F910895DF93CF9300D000D0AE
:10E1B00000D0CDB7DEB7FE01319696E0DF011D92AB
:10E1C0009A95E9F74983AF010E94BE7026960FB673
:10E1D000F894DEBF0FBECDBFCF91DF9108952F928F
:10E1E0003F924F925F926F927F928F929F92AF92E7
:10E1F000BF92CF92DF92EF92FF920F931F93DF9324
:10E20000CF93CDB7DEB7E4970FB6F894DEBF0FBE5D
:10E21000CDBF5C01DC018C9187FF07C70FE7602E43
:10E220006822BFE3B61518F48F3F09F0FEC680914F
:10E23000A905853008F0F9C68F5F8093A90512E023
:10E24000E12EF12CEA0CFB1CB3E08B2E912C8A0CF6
:10E250009B1CF5018381C82EDD24D694DC2CCC24B4
:10E26000D794C7947280872D90E0C82AD92A8E014E
:10E270000E5F1F4F86E0D801E82F1D92EA95E9F75F
:10E28000D50111969C91963170F5943108F064C0D7
:10E290009930B0F4973008F0B9C0933009F469C0F0
:10E2A000943038F4913009F4D4C1923009F0AFC6FB
:10E2B00064C3953009F472C3963008F090C0D2C19F
:10E2C000903109F4E4C1913150F49D3009F498C1C2
:10E2D0009E3009F4C3C09B3009F099C640C1933108
:10E2E00008F463C275C29E3109F4D1C29F31C0F4F3
:10E2F000993109F471C29A3130F49731C1F19831F2
:10E3000008F003C22BC09B3109F44CC39B3108F4C5
:10E3100075C29C3109F4AEC29D3109F078C6BDC208
:10E32000903409F452C6913450F4903209F487C104
:10E33000903208F4C8C2943209F069C65CC39234C2
:10E3400009F418C6923408F42FC6933409F4EFC5C3
:10E35000903709F05CC604C0FF24DCC180E0D7C15F
:10E36000850176E0E72EF12CEA0CFB1C48C680E024
:10E37000CDC1C114D10409F44AC6F50114818581C7
:10E38000282F30E086FD1068322F2227330F330FFD
:10E39000D50116966C91169770E06F77707053E008
:10E3A000660F771F5A95E1F717968C9190E080776A
:10E3B000907044E0959587954A95E1F7682B792B05
:10E3C000622B732BC60144E00E941B3DC601612FE6
:10E3D00044E00E94543DC6010E94CB6C18C6F50172
:10E3E0008481382F3295330F330F307C20E0A60123
:10E3F000422B532B8581882319F0CA0161E002C0AA
:10E40000CA0160E044E00E94D28F01C6D501159692
:10E410008C911597E82FF0E017966C916F7740E09C
:10E42000983009F441E09F01277030703695322F03
:10E43000222737952795D50114968C91149790E053
:10E44000282B392BE074F070EE0FFF1F16960C91FD
:10E450000E2BC601EE240E948438D9C5C6010E9445
:10E46000B8385C01009781F48E01025F1F4F8BE08A
:10E47000F80111928A95E9F7DF86CE8680E88E8BC7
:10E48000C8010E94AA3B5801D50112962D913C91DA
:10E4900013972115310511F1822F8F778A83220F6F
:10E4A000232F221F330B3195822F8F778B83129668
:10E4B0008D919C9113970E943A3D9B01AC01F2E033
:10E4C000EF2EF12CEC0EFD1EC70160E000E00E9473
:10E4D0000670862D6FE0A7010E94BE708C2D8F778D
:10E4E0008A83CC0CCD2CCC1CDD08D1948C2D8F775D
:10E4F0008B83F50181858C8372E0E72EF12CEC0E85
:10E50000FD1E862D69E0A7010E94BE70D5011496FC
:10E510002D913D914D915C91179700E012968D9150
:10E520009C911397892B09F001E0C701F5016085E3
:10E530000E9406708E010E5F1F4F862D6EE0A801AF
:10E540000E94BE70D50114964D915D916D917C91A4
:10E550001797C8010E94ED6F862D6DE094C0F501FC
:10E56000248130E040E050E0E781D50115968C91A0
:10E57000159790E09695982F8827979587957C0119
:10E580000027F7FC0095102F16966C91962F929508
:10E59000990F990F907C80E0AA2797FDA095BA2F3C
:10E5A000E82AF92A0A2B1B2BE22AF32A042B152B23
:10E5B0008E2F90E0A0E0B0E087709070A070B070F7
:10E5C00055E1880F991FAA1FBB1F5A95D1F7E82A5A
:10E5D000F92A0A2B1B2BD801C7010197A109B10900
:10E5E0008F5F9F4FAF4FB04008F011C5E695E6959D
:10E5F000E695C801B701A6012E2F0E945E8A07C5C5
:10E60000D50114962C91149730E015966C911597BE
:10E6100070E07695762F66277795679516964C91DC
:10E62000942F9295990F990F907C80E0682B792B0D
:10E63000622B732BC60144E00E94F93CE8C40E949F
:10E640006A12843009F4E3C4F50182810E948512C4
:10E65000DEC4C114D10409F4DAC4862DB6010E94C7
:10E66000CA6ED5C4C601D50114966C910E94043EB1
:10E67000F50182818A8383818B83C6010E94E03801
:10E680008C83862D69E0A8010E94BE70C0C4B801C9
:10E690006E5F7F4FC601AE01475E5F4F0E941A86D4
:10E6A000282F2F772A83880F892F881F990B919500
:10E6B0008F778B83898D8D838A8D8E831F82862DA4
:10E6C00061E1A8010E94BE70FE017B96D8019E0107
:10E6D000205E3F4F81918D93E217F307D9F7862D86
:10E6E00062E1AE014E5F5F4F0E94BE70FE01B096C8
:10E6F0009E012C5D3F4F8191D8018D938D01E217D2
:10E70000F307C9F7862D63E14CC083E08D5F23E0FA
:10E71000F22EF80E943189F4F5018581682F70E0AE
:10E720007695762F662777956795848190E0682B9C
:10E73000792B86818983198E21C08E01075E1F4F38
:10E74000C601BE016F5F7F4FA8010E941A86BC01FF
:10E75000D50194E00CC0F801EF0DF11D14968C91D9
:10E76000149780839F5FF3941196973019F0FAE025
:10E77000FF1588F7FE01EF0DF11D118EC6014981CD
:10E780009E01275E3F4F0E947186282F2F772A8394
:10E79000880F892F881F990B91958F778B83862DF2
:10E7A00060E1AE014E5F5F4F6FCF913121F4C60142
:10E7B0000E949F8503C0C6010E9490859C018F77AF
:10E7C0008A83220F232F221F330B3195822FE5CF0F
:10E7D000C6010E946C861BC48C2D8F778A83C6016C
:10E7E000880F892F881F990B91958F778B83C6018E
:10E7F0000E94228D8C83862D69E145CFD501159627
:10E800008C911597082F10E01695102F002717955B
:10E81000079516962C911697922F9295990F990F0E
:10E82000907C80E0082B192B14968C9190E0082B9B
:10E83000192B7601E4E0EE0CFF1CEA95E1F771E09C
:10E84000C72ED12C60E1A62EB12CAE0CBF1C60E00F
:10E85000C60180239123892B09F061E0C7010E9442
:10E86000188ECC0CDD1C0894E11CF11CEA14FB048E
:10E8700071F7CDC3772009F0CAC38DE08A8382E0A7
:10E880008B838C8383E08D83862D6CE18ACFC601D8
:10E89000F501648145810E945289D50114966C91DD
:10E8A0008C2D8F778A83C601880F892F881F990B3B
:10E8B00091958F778B836C83C6010E94C2888D836C
:10E8C000862D6EE16ECF8C2D8F778A83C601880FDF
:10E8D000892F881F990B91958F778B83C6010E9492
:10E8E0002F889EA38DA3FF2425E2222E312C2C0EEF
:10E8F0003D1E99E2492E512C4C0E5D1EC801902EF2
:10E90000E92E85E3A82EB12CAC0EBD1E26C080E1F9
:10E91000B1010E9479828FA198A58C159D0509F5FA
:10E920008201F8018181882399F08081F0FC04C084
:10E930008C8381818D830BC08E83D80111968C913D
:10E940008F83862D6FE1492D5E2D0E94BE70F3945A
:10E950000E5F1F4F0A151B0521F78DA19EA1892B64
:10E96000B1F6F0FC05C0FC821F821E821D8202C02F
:10E97000FE821F82862D6FE114CFF501458150E0A4
:10E980005695542F442757954795848190E0482BFE
:10E99000592B862DB6010E94486E39C3C6010E94CC
:10E9A000B73C35C3D50116964C91169750E0159695
:10E9B0006C91159770E06F7770707695762F66275B
:10E9C00077956795CA018170907090E4899F902D2A
:10E9D00088271124682B792B14968C9190E0682B52
:10E9E000792BE6E056954795EA95E1F74170C60127
:10E9F0000E940A380CC3FE013896DF011D928A95E9
:10EA0000E9F70E947C6C8C01B6E07B1609F4AEC07D
:10EA1000B715A8F0E2E07E1609F44BC0E71538F010
:10EA2000772041F1F1E07F1609F0F1C22CC024E01B
:10EA3000721609F473C0271508F47EC052C08BE02B
:10EA4000781609F432C1871560F098E0791609F458
:10EA5000CEC0791608F491C0A9E07A1609F0D7C2A1
:10EA6000D1C0B4E1B71508F02FC1E6E17E1609F078
:10EA7000CEC221C218860E94866C8F7089870E9440
:10EA8000836C877049C0D50113968C918F700E945A
:10EA90000E6F0E94836CF4019181982B892F8770EF
:10EAA0000E941A6FD50113968C9186FFE3CF81E007
:10EAB00015C0F50183818F700E94006F0E94836CE6
:10EAC000D40111969C9190959823892F87700E946C
:10EAD0001A6FF501838186FFCDCF80E00E94B6805A
:10EAE000C9CFD50113968C91882361F0F4018281FE
:10EAF0008795882787959181892BD80116968C93C5
:10EB00000E94E86E83E08887F80186818F77898785
:10EB10008681881F8827881F8A8703C2D50113969C
:10EB20008C91853310F4F801808784E08887D801C0
:10EB300018968C918987F5C1F501838164E00E9464
:10EB400092809C0185E08887822F8F778987C90111
:10EB5000880F892F881F990B91958F778A87832F2C
:10EB600082958695869583708B87DBC1D501139638
:10EB70008C9164E00E94AB80E4CFF4018181082F86
:10EB800010E01695102F002717950795D5011396BD
:10EB90008C9190E0082B192BBFE0003F1B0728F059
:10EBA000EFE30F3F1E0709F032C2D40112966C91B9
:10EBB000633011F0613069F4BFE30F3F1B0729F4A4
:10EBC000862F90E00E94D18D04C0C80170E00E94A1
:10EBD000818D87E08887F50183818987D40111962B
:10EBE0008C918A87C8010E94508D8F77BDCFF50127
:10EBF0008381882319F00E94478C02C00E94B48A46
:10EC000088E08EC181E0888738E0C32ED12CCC0EFD
:10EC1000DD1E862D65E2A6010E94BE70D40111960C
:10EC20006C9170E07695762F662777956795F5015C
:10EC3000838190E0682B792B862D0E94577E7B0183
:10EC40008C011886862D65E2A6010E94BE7078862A
:10EC50008E2D8F77898797E016950795F794E7941F
:10EC60009A95D1F78E2D8F778A8787E0169507952D
:10EC7000F794E7948A95D1F78E2D8F778B87B7E03D
:10EC800016950795F794E794BA95D1F78E2D8F775F
:10EC90008C87A7E016950795F794E794AA95D1F786
:10ECA000ED86862D64E2A601EFCC7886862D64E29F
:10ECB000AE01485F5F4F0E94BE7082E390E00E9409
:10ECC000F5190E946C6FA3C180E00E94851281E05B
:10ECD0008887862D65E2AE01485F5F4F0E94BE7057
:10ECE000F0E17F1609F47EC0F71588F02DE072166A
:10ECF00089F1271520F08CE07816C1F41AC09EE047
:10ED0000791609F442C0AFE07A1681F453C0B2E13B
:10ED10007B1609F47EC07B1608F46BC0E3E17E1617
:10ED200009F488C0F4E17F1609F49BC0EE24FF24A7
:10ED3000A4C0D40111968C9190E09695982F8827C5
:10ED400097958795F501238130E0822B932B0E94C4
:10ED5000A97D92C0D40111968C91119790E096955F
:10ED6000982F882797958795F501238130E0139692
:10ED70006C91139767956627679512964C91642B53
:10ED8000822B932B0E94B37D77C0D40111968C9176
:10ED9000119790E09695982F882797958795F5017C
:10EDA000238130E012966C916770822B932B0E9426
:10EDB000BE7D62C0D40111968C91119790E096951A
:10EDC000982F882797958795F501238130E0129633
:10EDD0006C9112976770822B932B13964C910E9423
:10EDE000C97D4AC0D50113968C918F700E94877D92
:10EDF00043C0F5018381D40112966C9112976795F7
:10EE00006627679511969C91692B8F700E94927D61
:10EE100033C0F401818190E09695982F88279795CB
:10EE20008795D50113962C9130E0822B932B0E946D
:10EE3000727D22C0F401818190E09695982F8827F9
:10EE400097958795D50113962C9130E0638167954E
:10EE5000662767954281642B822B932B0E947C7DD1
:10EE60000BC0F4018181879588278795D50113967A
:10EE70009C91892B0E949E7D7C0118868E01085FE3
:10EE80001F4F862D65E2A8010E94BE7085E188872C
:10EE90008E2D8F778987C701880F892F881F990B3F
:10EEA0008F778A878F2D82958695869583708B873D
:10EEB000862D64E2E8CBF4016381A62FB0E0818166
:10EEC00090E09695982F882797958795F501E38090
:10EED000FF2462956370AD0106E0569547950A954B
:10EEE000E1F741709D01277030703695322F22274F
:10EEF00037952795F4015281E52FF0E02E2B3F2B1B
:10EF0000A870B070F4E0AA0FBB1FFA95E1F7F40106
:10EF100004810A2B8E299F29EE240E94843885E1E2
:10EF20008887862D64E2AE01485F5F4FADCB6624D3
:10EF3000862D0E9433708823A9F4862D64E0A701F2
:10EF40000E94BE708091F705861510F46092F70557
:10EF5000FFE3F61558F0E62DF0E0E95CF34F8EE1A3
:10EF6000808304C0639420E4621611F784E08093E8
:10EF7000F8054DC08091F805833008F048C083E063
:10EF80008093F805D50112968C9112978093F9051C
:10EF900013968C9113978093FA0514968C91809315
:10EFA000FB051092FC0533C08091F805823078F59E
:10EFB00082E08093F805F50182818093F9058381D1
:10EFC0008093FA051092FB0522C08091F8058823F2
:10EFD000F1F481E08093F805D50112968C9180932D
:10EFE000F9051092FA0513C08A3019F48DE00E94D9
:10EFF0003A16F80182810E943A160F5F1F4FD8011E
:10F0000012968C91882319F00E151F0569F7BFE33E
:10F01000B61530F0E62DF0E0E95CF34F8EE1808329
:10F020008091A90581508093A905E4960FB6F894C4
:10F03000DEBF0FBECDBFCF91DF911F910F91FF902B
:10F04000EF90DF90CF90BF90AF909F908F907F9088
:10F050006F905F904F903F902F9008950E94EF70B7
:10F0600008950F931F93CF93DF93EC01162F009712
:10F0700009F46CC086E0DE011D928A95E9F70E94D2
:10F080007C6C2091F5053091F60554E0220F331F7A
:10F090005A95E1F7FC01858596858217930720F440
:10F0A0001092F6051092F5051F77DE011D93E09191
:10F0B000F505F091F6058E2F8F7789839D012F5FDF
:10F0C0003F4FCF01880F892F881F990B91958F771C
:10F0D00011968C93A9014F5F5F4FEE0FFF1FDF0169
:10F0E000A454B24F8C918F77E9018983EA0121966C
:10F0F000E354F24F8081880F8E779C91991F992756
:10F10000991F892BDA0111968C938E010F5F1F4F87
:10F1100080818295869586958370898382E00E949E
:10F12000896C882329F089818460898381E001C00A
:10F1300080E00E94EA92E80121968091F505909185
:10F14000F60501969093F6058093F505CE01DF91C3
:10F15000CF911F910F910895AF92BF92DF92EF92DE
:10F16000FF920F931F93DF93CF93CDB7DEB729970D
:10F170000FB6F894DEBF0FBECDBFFFEEEF2EF0E767
:10F18000FF2EBB24B394DD24DA943DC087FF07C073
:10F19000B0929F058093A005D092A10534C0209124
:10F1A0009F05222381F1293040F4E22FF0E0E05660
:10F1B000FA4F80832F5F20939F0580919F058930B0
:10F1C00010F100EA15E090E0F80161918F01892FBC
:10F1D0000E94C96F982FF5E0083A1F07A9F787FD2D
:10F1E00090958091A805981761F467C1F092FE058B
:10F1F000E092FD05E091FD05F091FE0580EA95E0C5
:10F20000099510929F050E9478182FEF8F3F920763
:10F2100009F0BCCF0E940A180A970CF43AC19091E9
:10F22000F2058091F305981719F19091F30589E0A3
:10F23000989F700111248AEA95E0E80EF91E00E01B
:10F2400010E0F70181917F010E941B180F5F1F4F93
:10F2500009301105B1F78091F3058F5F8093F305B5
:10F260008091F305883008F414C11092F30511C1A0
:10F2700080919E05882311F0DD240EC181E08093EA
:10F280009E054091F405403429F08091F8058823CB
:10F2900009F473C08FEF89838091F8058130B1F054
:10F2A000813030F0823021F1833009F056C036C011
:10F2B00080E48A838091F905982F97709B838F5FF4
:10F2C0008093F905E4E0EE2EF12C4CC081E48A83B2
:10F2D0008091F90587708B838091FA05982F9F772D
:10F2E0009C838F5F8093FA059E012B5F3F4F2FC059
:10F2F00082E48A838091F90587708B838091FA0577
:10F300008F778C838091FB05982F9F779D838F5FEC
:10F310008093FB059E012A5F3F4F19C083E48A83D7
:10F320008091F90587708B838091FA058F778C83A4
:10F330008091FB058F778D838091FC05982F9F77B7
:10F340009E838F5F8093FC059E01295F3F4F87FF5F
:10F3500002C01092F805790107C01092F80572E01A
:10F36000E72EF12CEC0EFD1E8091F805882309F0A4
:10F3700064C04F5F4093F40560C04134E9F58FEFFE
:10F38000898383E08A830E946A12682FCE010396E4
:10F390000E9431787C018091F4058F5F8093F405A1
:10F3A0000E943C3E8C01FC01848D81FF22C0F8014B
:10F3B00080819181668D44E00E94543DF801468130
:10F3C0005781608571858081918124E00E94E23CB3
:10F3D000F80182819381009729F06285738544E06A
:10F3E0000E941B3DF801808191810E94CB6C0E949C
:10F3F000AD6CDD24D3942BC0403410F01092F40592
:10F400009091F405892F8068898382E08A83903403
:10F4100048F4E92FF0E0E95CF34F8081882311F094
:10F42000815080839F5F9093F4058091F7059E0142
:10F430002D5F3F4F891718F07901DD2408C080E463
:10F440008093F405F9CFF70111927F0102C0CE013C
:10F450000996E816F906B8F38E010F5F1F4FFF24D7
:10F4600069E0A62EB12CAC0EBD1E8F2DF801608177
:10F470000E94C96FF82EF80181918F010E941B181C
:10F480000A151B0590F3F7FCF0948F2D0E941B18B2
:10F4900001C0DD2410929E058D2D29960FB6F8949B
:10F4A000DEBF0FBECDBFCF91DF911F910F91FF90B7
:10F4B000EF90DF90BF90AF9008958091FD059091FF
:10F4C000FE05892B09F096CE91CE0F931F93DF9303
:10F4D000CF9300D000D000D0CDB7DEB7682F8E011B
:10F4E0000F5F1F4FC8010E9431788FEF63E0A801C2
:10F4F0000E94BE7026960FB6F894DEBF0FBECDBF39
:10F50000CF91DF911F910F910895EF92FF920F938A
:10F510001F93CF93DF93182F80E00E94851282E320
:10F5200090E00E94F51984E00E948512112319F0E1
:10F530000E94623202C00E949E3284EF91E00E94DB
:10F54000F5190E947B260E94822384E690E00E94A7
:10F55000F5191123D9F00E949D238C0180E090E0E1
:10F5600060E040E00E94113480E090E060E041E023
:10F570000E94113483E090E00E94BD7B84E690E01D
:10F580000E94F5190E949D23EC015FC04AE0E42E21
:10F59000F12C0E9482230E947B2660E070E080E0D4
:10F5A00090E040E20E94EE3204C084E190E00E94CC
:10F5B000F5190E94BC308823C1F30E949D238C0161
:10F5C0000E94822360E070E080E090E841E00E94C9
:10F5D000EE3260E070E080E090E041E00E94EE32C8
:10F5E00004C084E190E00E94F5190E94BC30882399
:10F5F000C1F384E690E00E94F5190E949D23EC017E
:10F600000531110534F0C801880F991FC817D907B3
:10F61000C4F48E2D8A50823060F0C7010E947E3281
:10F6200004C084E190E00E94F5190E94BC30882358
:10F63000C1F30894E11CF11C20E1E216F10409F089
:10F64000A8CF80E090E00E947E320E947B26C80115
:10F650004497855A9B40B0F081E060E00E94481FCB
:10F660000431110514F48DE101C08EE10E944D6C4E
:10F67000BC0182E00E941C2180E00E94851288EE7D
:10F6800093E002C086E990E00E94F519C801880F56
:10F69000991F8C179D0754F481E0C53FD80734F0BB
:10F6A00098012C0F3D1F359527950AC024E0C13BDA
:10F6B000D2071CF428EE33E003C09E01285C3040E2
:10F6C000C901DF91CF911F910F91FF90EF900895A5
:10F6D000DF93CF9300D000D000D0CDB7DEB716B8FF
:10F6E00086B187B90E947C6CDC0114968C910E94D3
:10F6F000BF1EFE01319686E0DF011D928A95E9F773
:10F7000081E089838FEF62E2AF010E94BE70E2E682
:10F71000F0E080818D7F808326960FB6F894DEBF5F
:10F720000FBECDBFCF91DF910895DF93CF9300D06F
:10F7300000D000D0CDB7DEB7E2E6F0E08081826095
:10F74000808380E00E94BF1EFE01319686E0DF01CB
:10F750001D928A95E9F78FEF62E2AF010E94BE70B9
:10F7600083EC87B98FEE86B926960FB6F894DEBF84
:10F770000FBECDBFCF91DF9108950F931F93CF930D
:10F78000DF93EC0101C0A8950E94BC308823D9F317
:10F7900011C0A89504C081E090E00E94F5190E9474
:10F7A000BC308823C1F380E090E060E041E00E943B
:10F7B000783421970E947E23882311F4209749F7FB
:10F7C0000E947E23082F15E00FC080E090E060E0EB
:10F7D00043E00E9478340E94822301C0A8950E94D1
:10F7E000BC308823D9F311500E947E23882319F05E
:10F7F000112359F707C0112329F0802F002319F096
:10F8000081E001C080E0DF91CF911F910F910895B9
:10F81000EF92FF920F931F93CF93DF937C01C0E091
:10F82000D0E0C7016C2F0E94D13380E090E00E94AD
:10F83000BD7B882319F40FEF1FEF02C00C2F10E0DF
:10F84000CF3FD10551F4E80183E090E00E94BD7BF9
:10F85000882349F00FEF10E00AC021968FEF0F3F89
:10F860001807F9F204C08FEF0F3F1807C1F0102FEF
:10F87000C701612F0E94D13383E090E00E94BD7BDD
:10F88000882319F4CFEFDFEF02C0C12FD0E011239E
:10F8900031F08FEFCF3FD80711F41150E9CFCE01EF
:10F8A000DF91CF911F910F91FF90EF9008952F92CC
:10F8B0003F924F925F926F927F928F929F92AF9200
:10F8C000BF92CF92DF92EF92FF920F931F93CF934D
:10F8D000DF93D82E7B01C42EA22E302E0E94957B62
:10F8E000C7019695879596958795482E4394CFEFB7
:10F8F000DFEFBB2437E0632E712C6E207F2023E0E6
:10F90000822E912C8E209F205A2C222481E00E944E
:10F91000857A0E948C230E9482230E946A1284307E
:10F9200009F0C7C083E0D81609F446C08D1530F041
:10F9300081E0D81631F18D15F8F00EC085E0D816AB
:10F9400040F086E08D1508F057C088E08D1508F06E
:10F9500072C0CFEFDFEF9FC0C7016C2D4A2D0E9410
:10F9600038348FE090E00E94BD7B882309F493C077
:10F97000852D922DEC0189C0C7016C2D0E94B133F9
:10F980004BC0C7016C2D40E00E94113483E090E031
:10F990000E94BD7B882309F0A2C0C7016C2D41E005
:10F9A0000E94113483E090E00E94BD7B882309F41B
:10F9B00072C0C1E0D0E069C010E000E00695C70168
:10F9C000612F40E00E94113483E090E00E94BD7BF3
:10F9D000882309F400681F5F183081F7C701602F82
:10F9E0000E94913383E090E00E94BD7B882309F45C
:10F9F00052C0C02FD0E049C085E090E061E00E9495
:10FA0000F1338FE090E00E94BD7B85E0D81661F471
:10FA1000C3016C2D0E94F1338FE090E00E94BD7B0A
:10FA2000882309F05CC037C0C3010E94087CEC0148
:10FA300093E0B92E28C085E090E0642D0E94F13358
:10FA40008FE090E00E94BD7B87E0D81669F4C40186
:10FA50006C2D0E94F1338FE090E00E94BD7B8823E3
:10FA600049F0C0E0D0E006C0C4010E94087CEC016F
:10FA700083E0B82E85E090E061E00E94F1338FE0F2
:10FA800090E00E94BD7BD7FD06C0332021F08CE2C0
:10FA900091E00E94F51980E00E948512D7FF09C00D
:10FAA0008CE291E00E94F519B39482E08B1508F086
:10FAB0002DCF0E94687BCE01DF91CF911F910F91D6
:10FAC000FF90EF90DF90CF90BF90AF909F908F907E
:10FAD0007F906F905F904F903F902F900895C0E07F
:10FAE000D0E0D3CF0F93BC0188E040E020E000E0FD
:10FAF0000E94577C0F9108950F939C01462F87E039
:10FB0000B90120E001E00E94577C0F9108950F9306
:10FB1000682F86E070E040E020E000E00E94577C23
:10FB20000F9108950F93982F462F85E0692F70E06D
:10FB300020E001E00E94577C0F9108950F93482F19
:10FB400085E060E070E020E001E00E94577C0F91CA
:10FB500008950F93BC0183E040E020E000E00E94A4
:10FB6000577C0F9108950F939C01462F82E0B901B5
:10FB700020E001E00E94577C0F9108950F939C01B3
:10FB8000462F81E0B90120E000E00E94577C0F91F0
:10FB900008950F93FC01962F242F80E0BF01492F79
:10FBA00001E00E94577C0F910895DF92EF92FF923F
:10FBB0000F931F932091DA073091DB074091DC0708
:10FBC0005091DD077C0100E010E0E20EF31E041FFF
:10FBD000151F10C081E090E00E94F5190E94822359
:10FBE000C801B7010E942F19882391F40E947E2337
:10FBF000882311F0DD2401C0D3940E94BC308823F7
:10FC000049F30E947E23882329F789E08D1510F798
:10FC10000E94BC30882319F480E090E008C00E9464
:10FC20007E2390E0811191E081E09827892F1F9138
:10FC30000F91FF90EF90DF900895EF92FF920F9356
:10FC40001F932091DA073091DB074091DC07509138
:10FC5000DD077C0100E010E0E20EF31E041F151F1B
:10FC600001C0A8950E94BC308823D9F301C0A89593
:10FC70000E947E23882331F4C801B7010E942F1906
:10FC80008823A9F30E94BC30882319F480E090E017
:10FC900009C00E947E2390E0882309F491E081E06E
:10FCA0009827892F1F910F91FF90EF9008952F9221
:10FCB0003F924F925F926F927F928F929F92AF92FC
:10FCC000BF92CF92DF92EF92FF920F931F93DF9339
:10FCD000CF93CDB7DEB767970FB6F894DEBF0FBEF0
:10FCE000CDBF8B8B7D8B6C8B0E94957B80E00E94BF
:10FCF000857A8E8B9F8B8C899D890E94B33C9A8BD1
:10FD0000898B009771F0DC0119961C92E989FA89B8
:10FD100014821582168217828C899D8960E00E9468
:10FD20008C3D0E946A12843021F0CC24DD247601BF
:10FD3000D9C118861F8288EE93E00E94D57D01E02C
:10FD4000CC24DD247601812C912CA12C60E8B62EE8
:10FD500009870E947E1D0A9709F4B5C1FB89FF3F00
:10FD600051F581E060E00E94481F2DB73EB7295051
:10FD700030400FB6F8943EBF0FBE2DBFEDB7FEB7B3
:10FD8000319622E0ADB7BEB711962C9345ED58E100
:10FD90005283418303831482C582D682E782F08630
:10FDA0000E94C2208DB79EB709960FB6F8949EBFE9
:10FDB0000FBE8DBF37C09AE099838C2D8F778A83D1
:10FDC000D701C60157E0B695A795979587955A959F
:10FDD000D1F78F778B83D701C6014EE0B695A795F3
:10FDE000979587954A95D1F78F778C83D701C60170
:10FDF00035E1B695A795979587953A95D1F78F7781
:10FE00008D83D701C6012CE1B695A7959795879567
:10FE10002A95D1F78E838B8964E2AE014F5F5F4FE5
:10FE20000E94BE70023028F420E030E040E050E84C
:10FE30000EC0802F90E0019720E030E040E050E8D5
:10FE400004C056954795379527958A95D2F72D8703
:10FE50003E874F87588B8E899F899C011901260107
:10FE6000370135E03C87C1010E948C2384E690E095
:10FE70000E94D57DC301B201402F0E94EE328AE07C
:10FE800090E00E941D7E811181E0182F0E949D2329
:10FE90009B878A878D859E85AF85B8894826592698
:10FEA0006A267B2684E690E00E94D57DC301B201DC
:10FEB000402F0E94EE328AE090E00E941D7E811168
:10FEC00012600E949D23AA85BB858A1B9B0B97FF0E
:10FED00003C0909581959F4F8059914014F484E020
:10FEE00005C0112311F01330CCF0812FEC85E150C7
:10FEF000EC87EE2391F0882329F428E33FEF220ECC
:10FF0000331E06C0833021F448EC50E0240E351E29
:10FF100084E690E00E94F519A6CF182F812F81501A
:10FF200031F0813051F4C828D928EA28FB28B6944A
:10FF3000A794979487940F5F15C0023028F0880C1F
:10FF4000991CAA1CBB1C0150D501C4018095909539
:10FF5000A095B095C822D922EA22FB2284E690E03F
:10FF60000E94F51959855F5F5987503621F001329B
:10FF700008F4EFCE03C0013208F499C0C114D104D3
:10FF8000E104F10409F493C08FEFC8168FEFD8068F
:10FF90008FEFE8068FEFF80609F495C09B899F3F25
:10FFA00041F581E060E00E94481FADB7BEB71997E8
:10FFB0000FB6F894BEBF0FBEADBFEDB7FEB731961A
:10FFC00022E011962C9349EC58E1528341838F81B2
:10FFD000988594838383C582D682E782F0860E94C7
:10FFE000C220ADB7BEB719960FB6F894BEBF0FBE0C
:10FFF000ADBFE989FA89EF2B09F468C02C893D89E6
:020000021000EC
:100000002115310509F462C0C701B601A9010E949A
:10001000D03288EE93E00E94F519BB2489899A8931
:1000200041E050E060E070E000E010E020E030E00F
:100030000E94AF340E94BC308823E1F384E690E054
:100040000E949219B39435E0B31641F784E690E02C
:100050000E94D57DC701B6014C895D890E94B232EC
:100060008AE090E00E941D7E882381F54B894F3FF6
:10007000F1F481E060E00E94481F00D000D00F92B0
:10008000EDB7FEB7319622E0ADB7BEB711962C930F
:1000900047EB58E1528341838F8198859483838312
:1000A0000E94C2200F900F900F900F900F9088EE3B
:1000B00093E00E94F519AF81B8851196B887AF8398
:1000C000159709F038CECC24DD24760180E00E941B
:1000D0008512C114D104E104F10421F488EE93E007
:1000E0000E94F5190E94687B80E00E948512B6018B
:1000F000C70167960FB6F894DEBF0FBECDBFCF9194
:10010000DF911F910F91FF90EF90DF90CF90BF9004
:10011000AF909F908F907F906F905F904F903F90A7
:100120002F900895662319F027E73CE002C02FEDD9
:100130003CE0F894E82FF0E0EE0FFF1FE20FF31F12
:10014000208191818091470D80FF02C01182108231
:100150007894822F0895E82FF8947894F0E0EE0FC9
:10016000FF1FEC5AF24F8081918108959091470DC5
:10017000882311F0916001C09E7F9093470D0895F0
:10018000BF92CF92DF92EF92FF920F931F93CF9384
:10019000DF93882339F03EE4C32E3DE0D32EC7E73A
:1001A000DCE006C028E4C22E2DE0D22ECFEDDCE04C
:1001B0000E947C6CFC01B08404E51DE07E01C0E07F
:1001C000D0E018C0F894F80180819181F701918303
:1001D0008083F80180819181892B21F0C601BE01C5
:1001E0000E945892789421960E5F1F4F82E090E013
:1001F000E80EF91ECB1530F3DF91CF911F910F91CF
:10020000FF90EF90DF90CF90BF90089584E08093AF
:1002100074001092710083E08093700008951F9223
:100220000F920FB60F920BB60F9211248F939F93DC
:10023000EF93FF938091710090E0887F90708032FF
:10024000910509F485C0813291055CF480319105F6
:10025000D1F08831910509F442C0089709F07AC0BD
:1002600016C080349105A9F18134910524F4889752
:1002700009F070C03EC080359105D9F088359105F0
:1002800009F068C00AC08091FF0587FF02C080EABC
:1002900001C081EA8093730059C0E0910506F09196
:1002A0000606809173008193F0930606E09305069D
:1002B00046C0E0910506F091060680917300819397
:1002C000F0930606E0930506809100068150809326
:1002D0000006809100068230CCF185EC3FC0809111
:1002E000030690910406909373008FEF8093FF05AF
:1002F0002DC08091FF0587FF09C080910306909172
:100300000406809373001092FF0520C080910106BF
:100310008823F1F080910006882389F0E09105069A
:10032000F0910606819180937300F0930606E093A6
:1003300005068091000681508093000607C084E97D
:100340008093740081E0809302060AC085E806C0AD
:1003500085EA04C08FEF8093020684E980937400DD
:10036000FF91EF919F918F910F900BBE0F900FBE59
:100370000F901F9018958091740020E090E0877096
:100380009070892B09F021E0822F08956093000678
:10039000909304068093030620930106509306066B
:1003A000409305068EEF8093FF051092020685EAC2
:1003B00080937400089520910206332727FD30951D
:1003C000C901089560930006909304068093030684
:1003D0002093010650930606409305068EEF809306
:1003E000FF051092020685EA8093740001C0A8956B
:1003F000809102068823D9F320910206332727FD36
:100400003095C90108958130B1F0813070F08230AB
:1004100019F0833021F406C0EBE0F6E008C020E0DC
:1004200030E007C0EDE0F6E002C0E7E0F6E0208152
:100430003181C9010895E9E0F6E0F9CF8130D1F0CA
:10044000813058F0823019F08330B9F403C0EBE00A
:10045000F6E005C0EDE0F6E002C0E7E0F6E08081FE
:1004600091818617970749F07183608381E08093BB
:100470000F060895E9E0F6E0F2CF089524E0880F32
:10048000991F2A95E1F721E00E94E281089534E066
:10049000880F991F3A95E1F720E00E94E2810895C4
:1004A000DF93CF9300D0CDB7DEB794E0603079070B
:1004B00018F020E030E017C06115710571F0CB0134
:1004C00044E0880F991F4A95E1F762E0AE014F5F63
:1004D0005F4F20E00E94E28104C00E9403829A8361
:1004E000898329813A81C9010F900F90CF91DF91C3
:1004F00008950F931F93282FFB0100811181C801DC
:1005000054E0880F991F5A95E1F7622FAF0120E060
:100510000E94E281C8011F910F910895CF92DF924E
:10052000EF92FF920F931F93DF93CF9300D0CDB73D
:10053000DEB77B0194E06030790710F50E940382FA
:100540009A83898320E030E06E010894C11CD11C9D
:100550000CC0C80164E0880F991F6A95E1F762E05A
:10056000A60120E00E94E281980109811A8101150B
:10057000110521F00E151F0561F704C0EF2811F0D9
:100580002FEF3FEFC9010F900F90CF91DF911F9197
:100590000F91FF90EF90DF90CF900895CF93DF936E
:1005A000EC0180E0BE010E948E829C0184E020303C
:1005B0003807B8F082E0BE010E948E829C0184E080
:1005C0002030380770F083E0BE010E948E829C01CB
:1005D00084E02030380728F081E0BE010E948E823E
:1005E0009C01C901DF91CF91089580910F06882366
:1005F00051F080E090E068E047E056E021E00E94A2
:10060000E28110920F0608950F931F93DF93CF930B
:1006100000D0CDB7DEB70091090610910A0601158A
:100620001105A1F0C80174E0880F991F7A95E1F7D0
:1006300062E0AE014F5F5F4F20E00E94E28169817E
:100640007A8181E00E941E820E94F582C8010F908B
:100650000F90CF91DF911F910F910895DF92EF924C
:10066000FF920F931F93DF93CF9300D0CDB7DEB7E8
:10067000D82E8B01CB0101978F5F934058F5CB01AA
:10068000F4E0880F991FFA95E1F762E07E01089483
:10069000E11CF11CA70120E00E94E2818D2DB80130
:1006A0000E948E82009731F469817A818D2D0E949B
:1006B0001E820EC024E08030920750F4E4E0880FE0
:1006C000991FEA95E1F762E0A70121E00E94E2812B
:1006D0000E94F5820F900F90CF91DF911F910F91A3
:1006E000FF90EF90DF9008955F926F927F928F92CC
:1006F0009F92AF92BF92CF92DF92EF92FF920F93B1
:100700001F93DF93CF93CDB7DEB762970FB6F89400
:10071000DEBF0FBECDBF982E7A8B698B542E852EEF
:10072000390184E06030780708F067C06115710511
:1007300021F0892D0E942E8307C00E940483009718
:1007400009F45BC09A8B898B892D0E9403829A835E
:100750008983E52CF82CCC24DD245E010894A11CAF
:10076000B11C17C0C80124E0880F991F2A95E1F732
:1007700060E1A50120E00E94E281852D982DB50160
:10078000F30109951816190614F4C80107C0680189
:10079000C80109811A810115110521F7C816D9066A
:1007A00011F480E090E0F7019183808389899A8930
:1007B000B4E0880F991FBA95E1F762E0A70121E044
:1007C0000E94E281C114D10431F469897A89892DAA
:1007D0000E941E820DC0C601A4E0880F991FAA9531
:1007E000E1F762E0AE014F5E5F4F21E00E94E281DF
:1007F0000E94F58229893A8902C020E030E0C901CF
:1008000062960FB6F894DEBF0FBECDBFCF91DF91D9
:100810001F910F91FF90EF90DF90CF90BF90AF901E
:100820009F908F907F906F905F900895EF92FF92CE
:100830000F931F93DF93CF93CDB7DEB762970FB6B9
:10084000F894DEBF0FBECDBF482F7A8B698BCB01EA
:1008500001978F5F934008F04BC0842F0E942E8336
:100860008091090690910A069A8389837E010894F3
:10087000E11CF11C0CC0C80154E0880F991F5A9567
:10088000E1F762E0A70120E00E94E281C80109814E
:100890001A810115110579F7009731F469897A8970
:1008A00081E00E941E820CC044E0880F991F4A9587
:1008B000E1F762E0AE014F5E5F4F21E00E94E2810E
:1008C000CE0103966FEF70E04EE050E00E9427AA41
:1008D00089899A8934E0880F991F3A95E1F760E198
:1008E000AE014F5F5F4F21E00E94E2810E94F582DE
:1008F00062960FB6F894DEBF0FBECDBFCF91DF91E9
:100900001F910F91FF90EF9008950E941684089513
:10091000CF92DF92EF92FF920F931F93DF93CF93CB
:10092000CDB7DEB760970FB6F894DEBF0FBECDBF70
:1009300088E0E7E0F6E0DF011D928A95E9F781E0C3
:1009400090E090930A068093090681E080930F0659
:10095000A8950E94F582CE0103966FEF70E04EE0FD
:1009600050E00E9427AA01E010E060E1E62EF12CA1
:100970006E010894C11CD11CB3E00F3F1B0739F076
:100980000F5F1F4F1A8309830150104002C01A8263
:1009900019820E947112C70160E1A60121E00E9444
:1009A000E2810F5F1F4F80E190E0E80EF91E94E0B6
:1009B0000030190709F760960FB6F894DEBF0FBE36
:1009C000CDBFCF91DF911F910F91FF90EF90DF90FE
:1009D000CF900895CF92DF92EF92FF920F931F93E3
:1009E000DF93CF93CDB7DEB760970FB6F894DEBF35
:1009F0000FBECDBF80E090E068E047E056E020E029
:100A00000E94E28110920F0689E00E94401D882317
:100A100029F08EE00E94401D882371F48091090620
:100A200090910A068F5F9F4F31F580910706909154
:100A300008068F5F9F4FF9F484E06EEB71E00E942F
:100A4000292085E066EC71E00E94292082E89EE979
:100A500068EC70E00E94871E80E060E00E94481F02
:100A600083E00E944D6CBC0182E00E941C210E9428
:100A700088840E94C36C00910706109108066E01DD
:100A80000894C11CD11C1EC0C80174E0880F991FB6
:100A90007A95E1F760E1A60120E00E94E281F98009
:100AA000EA808B819C8101978F5F9F4320F080E0DB
:100AB000B8010E941684A8950E94681D8F2D9E2D56
:100AC0009C018901C80101978F5F9340E8F28091F2
:100AD0000B0690910C068050944028F082E060E074
:100AE00070E00E941E8280910D0690910E0680504B
:100AF000944028F083E060E070E00E941E820E9433
:100B0000F58260960FB6F894DEBF0FBECDBFCF91D1
:100B1000DF911F910F91FF90EF90DF90CF9008959C
:100B2000BC0180E00E948E829C01009731F480E03D
:100B300060E070E00E948E829C01C9010895BC01B2
:100B400080E00E9450829C01009731F480E060E0D8
:100B500070E00E9450829C01C9010895EF92FF92BB
:100B60000F931F93DF93CF93CDB7DEB760970FB688
:100B7000F894DEBF0FBECDBF8C01009719F420E0C2
:100B800030E016C080E00E9403829A8389837E0150
:100B90000894E11CF11C05C08B819C818017910792
:100BA00039F084E0B7010E9479829C010097A1F797
:100BB000C90160960FB6F894DEBF0FBECDBFCF91CE
:100BC000DF911F910F91FF90EF900895DF92EF92C8
:100BD000FF920F931F93DF93CF93CDB7DEB760974C
:100BE0000FB6F894DEBF0FBECDBFD62E0E94AE85E5
:100BF0008C01009789F060E17E010894E11CF11CF2
:100C0000A7010E9447828D818D1531F0DD82C801D8
:100C100060E1A7010E943E8260960FB6F894DEBFA5
:100C20000FBECDBFCF91DF911F910F91FF90EF903D
:100C3000DF900895EF92FF920F931F93DF93CF936E
:100C4000CDB7DEB760970FB6F894DEBF0FBECDBF4D
:100C50008B017A0124E08030920770F5009781F4CF
:100C600080E00E940382009759F40115110511F0EC
:100C7000F8011082E114F104F9F0F70110821CC0B0
:100C800060E1AE014F5F5F4F0E9447820115110581
:100C900019F08D81F8018083E114F10451F0D7013E
:100CA000FE0136968BE001900D928150E1F7F7013D
:100CB00013862B813C8102C020E030E0C9016096A0
:100CC0000FB6F894DEBF0FBECDBFCF91DF911F915D
:100CD0000F91FF90EF900895BC0180E00E94858401
:100CE0000895EF92FF920F931F93DF93CF93CDB7A9
:100CF000DEB760970FB6F894DEBF0FBECDBF7C01A4
:100D0000D9012115310569F16115710551F180E0B5
:100D1000E81684E0F80628F57C836B834D83FE019A
:100D200036969E012F5E3F4F02C0819311968C91A3
:100D3000882321F0E217F307C1F704C0E217F30795
:100D400008F4108280E0B7018E010F5F1F4FA801E9
:100D500029EC36E80E9474837C0160E1A8010E94BE
:100D60003E82C70160960FB6F894DEBF0FBECDBFBE
:100D7000CF91DF911F910F91FF90EF900895FC01AB
:100D8000A62F9A0180E090E0BF014A2F0E94718651
:100D900008959B01BC01009769F0C9012115310537
:100DA00049F06B5F7F4F05964BE050E00E9440AAF0
:100DB0009C0102C020E030E0C90108950F931F9309
:100DC000CF93DF938C01EB0182E00E940382998331
:100DD00088830AC0828193819F778017910771F081
:100DE0004F5F32964730B1F780E1BE010E947982B1
:100DF0009C01009719F0FE0140E0ECCFC901DF91A2
:100E0000CF911F910F910895DF93CF93CDB7DEB7A8
:100E100060970FB6F894DEBF0FBECDBFBE016F5F07
:100E20007F4F0E94DE86BC01009719F082E00E948D
:100E3000858460960FB6F894DEBF0FBECDBFCF910C
:100E4000DF9108956F927F928F929F92AF92BF929F
:100E5000CF92DF92EF92FF920F931F93DF93CF9386
:100E6000CDB7DEB760970FB6F894DEBF0FBECDBF2B
:100E70004C0180911006882309F07CC0C4010E94B7
:100E8000B8388C01009709F475C0DC0112968D9179
:100E90009C911397892B09F46DC01896BC90C401DE
:100EA000BE016F5F7F4F0E94DE867C010097A1F438
:100EB0000E9404837C01009709F45EC082E00E94D6
:100EC00003829A8389838050944010F01A82198299
:100ED00082E0B7010E941E828EE0FE013396DF01A0
:100EE0001D928A95E9F79C828B8225E0C22ED12C37
:100EF000CC0EDD1E91E1692E712C6C0E7D1EAB2C8B
:100F0000BB24A7FCB094AA24BB0CAA1CBB241DC004
:100F10000E94B8388C01009719F1FC0120813181C1
:100F2000D6012D933C9340E050E0808587FF02C0BE
:100F300041E050E04A155B0521F03068F60131834D
:100F4000208382E090E0C80ED91ED80112968D91C0
:100F50009C9113978815990519F0C614D704C1F60A
:100F6000C70160E1AE014F5F5F4F0E943E820E9469
:100F7000F58202C0EE24FF24C70160960FB6F894F4
:100F8000DEBF0FBECDBFCF91DF911F910F91FF90BC
:100F9000EF90DF90CF90BF90AF909F908F907F9019
:100FA0006F900895CF92DF92EF92FF920F931F936D
:100FB000DF93CF93CDB7DEB760970FB6F894DEBF5F
:100FC0000FBECDBF9C01809110068823C1F5C901D9
:100FD000BE016F5F7F4F0E94DE86892B81F181E029
:100FE00080931006EB80FC80C7010E94B33C892BE4
:100FF00011F18E010B5F1F4F3FE0C32ED12CCC0EA1
:10100000DD1EF801208131813F77C90101978E5F94
:101010009F4358F4C9010E94B33C892B61F0F80149
:1010200060817181C7010E947A3C0C151D0519F081
:101030000E5F1F4FE6CF1092100681E001C080E0E6
:1010400060960FB6F894DEBF0FBECDBFCF91DF9193
:101050001F910F91FF90EF90DF90CF900895CF9266
:10106000DF92EF92FF920F931F93DF93CF93CDB751
:10107000DEB760970FB6F894DEBF0FBECDBF7C0120
:1010800083E00E9403828C016E010894C11CD11C74
:101090000CC0C80164E0A6010E9447828B819C813C
:1010A0008E159F0528F409811A810115110589F70C
:1010B000C80160960FB6F894DEBF0FBECDBFCF91CA
:1010C000DF911F910F91FF90EF90DF90CF900895E7
:1010D0009F92AF92BF92CF92DF92EF92FF920F93C7
:1010E0001F93DF93CF93CDB7DEB760970FB6F89419
:1010F000DEBF0FBECDBF6C01962E5A0189012115AE
:10110000310519F48E010F5F1F4FC6010E942F8811
:101110007C0120C0C70160E1A8010E944782F8015C
:10112000828193818C159D05C1F420E030E084819B
:10113000891539F4A114B10491F0F501F182E0822E
:101140000EC02F5F3F4F32962630310581F7F801F0
:10115000E080F180E114F104E9F62FEF3FEFC901DF
:1011600060960FB6F894DEBF0FBECDBFCF91DF9172
:101170001F910F91FF90EF90DF90CF90BF90AF90B5
:101180009F9008950F931F93DF93CF93CDB7DEB752
:1011900062970FB6F894DEBF0FBECDBF9C010197DA
:1011A0008F5F9F43B8F48FEF9FEF9A838983C901C4
:1011B0008E010F5F1F4FA8019E012D5F3F4F0E94C0
:1011C000688897FD07C0880F991F080F191FF8013D
:1011D000878101C080E062960FB6F894DEBF0FBE33
:1011E000CDBFCF91DF911F910F910895EF92FF92A4
:1011F0000F931F93DF93CF93CDB7DEB762970FB6F0
:10120000F894DEBF0FBECDBF9C0101978F5F9F4357
:10121000E0F58FEF9FEF9A83898353E0E52EF12C61
:10122000EC0EFD1EC9018E010F5F1F4FA801970133
:101230000E9468888630910540F5FC013296EE0FD9
:10124000FF1FE00FF11F1282880F991F080F191F4F
:10125000F8011782FE013896A0E0B0E0A701BE01B8
:101260006C5E7F4F8081811111963296E617F707E9
:10127000C9F769817A81AB2B21F483E00E948584D0
:1012800004C0CB0160E10E943E8262960FB6F894E2
:10129000DEBF0FBECDBFCF91DF911F910F91FF90A9
:1012A000EF9008958F929F92AF92BF92CF92DF926C
:1012B000EF92FF920F931F93DF93CF93CDB7DEB7DB
:1012C00062970FB6F894DEBF0FBECDBF8C01A62E7D
:1012D000B42E01978F5F9F4308F09DC08FEF9FEF63
:1012E0009A838983442321F4C8010E94F68893C01D
:1012F000B3E0CB2ED12CCC0EDD1EC8017E010894AC
:10130000E11CF11CA70196010E94688886309105B6
:1013100078F4FC01EE0FFF1FEE0DFF1D87818B158A
:1013200009F479C0B78289819A8160E1A60171C010
:10133000C8010E942F887C019A8389834601E8E0D6
:10134000CE2ED12CCC0EDD1E29C060E1A4010E945E
:1013500047828D819E818017910721F5F60120E05B
:1013600030E08081882381F4F9013296EE0FFF1F6F
:10137000DE011196EA0FFB1FA282220F331FA20F7C
:10138000B31F1796BC923FC02F5F3F4F3296263057
:10139000310539F78B819C819A83898389819A8170
:1013A000009799F60E9404830097A9F19A83898394
:1013B00080E1FE013396DF011D928A95E9F7FC82F8
:1013C000EB821E830D83AF82B88683E0B7010E9453
:1013D0008E82BFEF8F3F9B0731F469817A8183E072
:1013E0000E94858418C0009741F469817A8183E066
:1013F0000E941E820E94F58206C062E0AE014F5F2D
:101400005F4F0E943E8289819A8160E1AE014D5F0B
:101410005F4F0E943E8262960FB6F894DEBF0FBE09
:10142000CDBFCF91DF911F910F91FF90EF90DF9093
:10143000CF90BF90AF909F908F900895CF92DF9202
:10144000EF92FF920F931F93DF93CF93CDB7DEB749
:1014500060970FB6F894DEBF0FBECDBF7C01019739
:101460008F5F9F43E0F4C7010E942F888C016E01BB
:101470000894C11CD11C10C0C80164E0A6010E94E0
:1014800047828B819C818E159F0549F483E0B801CA
:101490000E94858409811A810115110569F76096FA
:1014A0000FB6F894DEBF0FBECDBFCF91DF911F9175
:1014B0000F91FF90EF90DF90CF900895EF92FF9201
:1014C0000F931F93DF93CF93CDB7DEB728970FB657
:1014D000F894DEBF0FBECDBF7B018C018091110659
:1014E00090911206892B99F1E982FA820B831C8371
:1014F00018861F82122F20FF0AC058874F83CA0107
:1015000060E070E040E050E00E941A86AC0111FFFC
:1015100005C08F819885906898878F834115510504
:10152000B1F080911106909112065E834D8368E0C0
:10153000AE014F5F5F4F21E00E94E2818091110672
:1015400090911206089690931206809311062896A1
:101550000FB6F894DEBF0FBECDBFCF91DF911F91C4
:101560000F91FF90EF9008955F926F927F928F920C
:101570009F92AF92BF92CF92DF92EF92FF920F9322
:101580001F93DF93CF93CDB7DEB76C970FB6F89468
:10159000DEBF0FBECDBF0E946A12582E80E00E94AF
:1015A000851280E090E060E040E050E00E94B944A5
:1015B000FE01319686E0DF011D928A95E9F710E081
:1015C000FE2E0F2F812F67E04F2D502F0E94BE70EF
:1015D00084E190E00E94F5191F5F103499F70E9492
:1015E000F63A1E861D86A12C10E4B12EBDE0EB2E2E
:1015F000F12CEC0EFD1E30C0C50168E0A70120E013
:101600000E94E2818D859E85BFEF8F3F9B0701F190
:101610000E94B33C8C010097D9F06B896F70FC017C
:10162000808191810E94043E8F859889D80113960C
:101630009C938E93129789899A89A0E0B0E0F80173
:1016400084839583A683B7838B899C8990FD1086BC
:1016500088E090E0A80EB91E8D859E858F5F9F4F14
:1016600059F61D8A1E8A1F8A188EA5E16A2E712CD2
:101670006C0E7D1EF7E08F2E912C8C0E9D1EC7C028
:10168000C50168E0A30120E00E94E2818D899E8966
:10169000AF89B88D80509040A040B14008F0B3C0F1
:1016A000E98CFA8CE114F10409F4ADC0F0E0EF1616
:1016B000F0E4FF0608F0A7C08B8D9C8DD92EDD1CB1
:1016C000DD24DD1CDD0C009711F4870111C08C01B5
:1016D0001F77C80160E070E040E050E00E941A8689
:1016E000E816F90619F421E0D22A02C0098D1A8DF4
:1016F0002D893E894F89588DCD2CDD24211531054A
:101700004105510509F044C00E943C3E7C01C0FEE9
:1017100009C0AC014C5D5F4FC80160E070E00E9401
:101720001A868C01C8010E94B8388C01009711F10B
:10173000DC0114964D915C9115978D919C911197B8
:1017400018966C910E94B944F801818560E070E0C0
:101750000E949844D80112968D919C9113970E94F3
:10176000B838FC01009731F06481758180819181E6
:101770000E94DB3EC1FE04C0F701848D8160848F2E
:10178000D7015C968C915C9782605C968C933BC091
:10179000802F8F778F83000F012F001F110B119562
:1017A000802F8F778887822F8F77898777E056956C
:1017B0004795379527957A95D1F7822F8F778A8726
:1017C00067E056954795379527956A95D1F7822F0B
:1017D0008F778B8793E0CC0CDD1C9A95E1F787E03F
:1017E00056954795379527958A95D1F7822F87701B
:1017F0008C298C878FEF6CE0A4010E94BE700E9440
:10180000AC788823E1F3E8E0F0E0AE0EBF1E8D89EE
:101810009E89AF89B88D80509040A040B14008F4B7
:101820002FCF0CEB1DE0C50168E0A80120E00E946D
:10183000E28188E090E0A80EB91E085F1F4F9EE08D
:101840000C3B190781F783E00E94851284E690E043
:101850000E94F5198F8598890E944B90852D0E94D2
:1018600085126C960FB6F894DEBF0FBECDBFCF9138
:10187000DF911F910F91FF90EF90DF90CF90BF907D
:10188000AF909F908F907F906F905F9008958F9210
:101890009F92AF92BF92CF92DF92EF92FF920F93FF
:1018A0001F93DF93CF93CDB7DEB728970FB6F89489
:1018B000DEBF0FBECDBF00E010E4FF248BE0882E1A
:1018C000912C5E010894A11CB11C2FC08F2D90E0BB
:1018D000889DF001899DF00D989DF00D1124EB5825
:1018E000F64FC080D180A281B38144815581668149
:1018F00077818185282F30E02F70307038872F83D3
:10190000808587FD03C0316038872F835E834D83D8
:10191000BC83AB83DA82C982C80168E0A50121E0FB
:101920000E94E281F394085F1F4F8091350CF816F6
:1019300068F20E947C6C2FEF3FEF3A832983FC0111
:10194000858596859C838B83C80168E0AE014F5FD7
:101950005F4F21E00E94E2810E943C3EFC01085F53
:101960001F4F109312060093110642A153A1848DBC
:101970004115510531F080FD02C021E009C023E08E
:1019800007C04081518180FD02C020E001C022E0FB
:1019900060E070E080E090E00E945E8A10E0812FBD
:1019A0006BE040E050E00E94BE701F5F1034B9F75A
:1019B00010E00E94AC788823E1F31F5F1630C9F76E
:1019C0006FEF7FEF8FEF9FEF4FEF5FEF20E00E9411
:1019D0005E8AE0901106F0901206109212061092A4
:1019E00011060CEB1DE0C70168E0A80121E00E9490
:1019F000E28188E090E0E80EF91E085F1F4F9EE04C
:101A00000C3B190781F728960FB6F894DEBF0FBE7E
:101A1000CDBFCF91DF911F910F91FF90EF90DF909D
:101A2000CF90BF90AF909F908F900895E3E1F6E044
:101A30008FEF9FEF91838083379626E0E33FF20795
:101A4000C9F708950F931F938C018CEB9DE0B801AB
:101A50000E948392482F9801220F331F442311F0D4
:101A60002F5F3F4FE3E1F6E080819181821793077A
:101A700049F4868180FF0CC0442311F487E40DC033
:101A800082E50BC086E0EC3EF80711F03796ECCF0C
:101A9000442311F487E601C082E71F910F91089556
:101AA0000F931F932FE0803F920718F02FEF3FEF27
:101AB00024C09C013695279543E02D3F3407D8F488
:101AC0008901169507951695079526E096958795B1
:101AD0002A95E1F78452904F0E94F9AC90E007708C
:101AE000107002C0959587950A95E2F780FD03C0B6
:101AF00021E030E002C023E030E0C9011F910F91E6
:101B00000895EF92FF920F931F93CF93DF937B0182
:101B10002FE0803F920708F03DC06330710519F057
:101B200061307105B9F59C013695279543E02D3F4D
:101B3000340780F589011695079516950795EC01F0
:101B400056E0D695C7955A95E1F7C452D04FCE01CD
:101B50000E94F9AC482F98012770307083E0E81696
:101B6000F10451F481E090E002C0880F991F2A959A
:101B7000E2F7642F682B0AC081E090E002C0880F72
:101B8000991F2A95E2F7682F60956423A895CE01E6
:101B90000E940BADDF91CF911F910F91FF90EF90BD
:101BA00008951F93CF93DF93039711F010E001C0C6
:101BB0001FEFCCEDDFE0A895CE01612F0E940BADA9
:101BC00021968FE0CC3FD807B1F7DF91CF911F91DD
:101BD0000895CF93DF93EC01662331F08CEB9DE009
:101BE000BE010E94589205C08CEB9DE0BE010E9490
:101BF0006D92CC0FCD2FCC1FDD0BD19581E090E005
:101C000002C0880F991FCA95E2F72091F306309120
